:020000040800F2
:10000000F0FF012035600008CD430008D54300080B
:10001000DD430008E5430008ED4300080000000050
:10002000000000000000000000000000D11B0108DB
:10003000F543000800000000211E0108FDF700083C
:10004000A9600008A9600008A9600008A96000086C
:10005000A9600008A9600008A9600008A96000085C
:10006000A9600008A9600008A9600008A96000084C
:10007000A9600008A9600008A9600008A96000083C
:10008000A9600008A9600008A9600008A96000082C
:10009000A9600008A9600008A9600008A96000081C
:1000A000A9600008A9600008A9600008A96000080C
:1000B0002D440008A9600008A9600008A960000894
:1000C000A9600008A9600008A9600008A9600008EC
:1000D000A9600008A9600008A9600008A9600008DC
:1000E000A9600008A9600008A9600008A9600008CC
:1000F000A9600008A9600008A9600008A9600008BC
:10010000A9600008A9600008A9600008A9600008AB
:10011000A9600008A960000805440008A96000085B
:10012000A9600008A9600008A9600008A96000088B
:10013000A96000080000000000000000A96000089D
:10014000A9600008A9600008A96000081944000817
:10015000A9600008A9600008A9600008A96000085B
:10016000A9600008A9600008A9600008A96000084B
:10017000A9600008A9600008A9600008000000004C
:1001800000000000A960000800000000000000005E
:10019000A96000080000000000000000A96000083D
:1001A000000000000000000000000000A96000083E
:1001B000A9600008A9600008A9600008A9600008FB
:0401C000A96000082A
:1001D00010B5054C237833B9044B13B10448AFF381
:1001E00000800123237010BD500300200000000098
:1001F000B061010808B5034B1BB103490348AFF3D5
:10020000008008BD0000000054030020B061010818
:1002100010F8012B11F8013B012A28BF9A42F7D0B0
:10022000D01A7047034613F8012B002AFBD1181A85
:1002300001387047000000000000000000000000CE
:1002400001F0FF01102A2BDB10F0070F08D010F887
:10025000013B013A8B422DD010F0070F42B3F6D18B
:10026000F0B441EA012141EA014122F007047FF0A4
:1002700000070023F0E80256083C85EA010586EAFB
:10028000010685FA47F5A3FA87F586FA47F6A5FA37
:1002900087F68EB9EED1F0BC01F0FF0102F0070243
:1002A00032B110F8013B013A83EA010313B1F8D1EE
:1002B0000020704701387047002D06BF35460338CF
:1002C000073815F0010F07D1013015F4807F02BF08
:1002D000013015F4C03F0130F0BC0138704700BF59
:1002E00081F0004102E000BF83F0004330B54FEAE7
:1002F00041044FEA430594EA050F08BF90EA020F54
:100300001FBF54EA000C55EA020C7FEA645C7FEAE6
:10031000655C00F0E2804FEA5454D4EB5555B8BF09
:100320006D420CDD2C4480EA020281EA030382EA7A
:10033000000083EA010180EA020281EA0303362D0C
:1003400088BF30BD11F0004F4FEA01314FF4801CDF
:100350004CEA113102D0404261EB410113F0004FF1
:100360004FEA03334CEA133302D0524263EB4303A8
:1003700094EA050F00F0A780A4F10104D5F1200E46
:100380000DDB02FA0EFC22FA05F2801841F10001A1
:1003900003FA0EF2801843FA05F359410EE0A5F175
:1003A00020050EF1200E012A03FA0EFC28BF4CF0A6
:1003B000020C43FA05F3C01851EBE37101F000455C
:1003C00007D54FF0000EDCF1000C7EEB00006EEB69
:1003D0000101B1F5801F1BD3B1F5001F0CD34908F3
:1003E0005FEA30004FEA3C0C04F101044FEA44524A
:1003F00012F5800F80F09A80BCF1004F08BF5FEAD1
:10040000500C50F1000041EB045141EA050130BDB0
:100410005FEA4C0C404141EB0101013C28BFB1F5C2
:10042000801FE9D291F0000F04BF01460020B1FA0D
:1004300081F308BF2033A3F10B03B3F120020CDAE0
:100440000C3208DD02F1140CC2F10C0201FA0CF0BE
:1004500021FA02F10CE002F11402D8BFC2F1200C23
:1004600001FA02F120FA0CFCDCBF41EA0C019040D9
:10047000E41AA2BF01EB0451294330BD6FEA040422
:100480001F3C1CDA0C340EDC04F11404C4F120020D
:1004900020FA04F001FA02F340EA030021FA04F31F
:1004A00045EA030130BDC4F10C04C4F1200220FA76
:1004B00002F001FA04F340EA0300294630BD21FAB4
:1004C00004F0294630BD94F0000F83F4801306BF7A
:1004D00081F480110134013D4EE77FEA645C18BF6E
:1004E0007FEA655C29D094EA050F08BF90EA020F05
:1004F00005D054EA000C04BF1946104630BD91EAFD
:10050000030F1EBF0021002030BD5FEA545C05D1FF
:100510004000494128BF41F0004130BD14F580043E
:100520003CBF01F5801130BD01F0004545F0FE41B2
:1005300041F470014FF0000030BD7FEA645C1ABFE7
:10054000194610467FEA655C1CBF0B46024650EA1E
:10055000013406BF52EA033591EA030F41F400214A
:1005600030BD00BF90F0000F04BF0021704730B5D0
:100570004FF4806404F132044FF000054FF00001A5
:1005800050E700BF90F0000F04BF0021704730B566
:100590004FF4806404F1320410F0004548BF40423B
:1005A0004FF000013EE700BF42004FEAE2014FEA90
:1005B00031014FEA02701FBF12F07F4393F07F4F6B
:1005C00081F06051704732F07F4208BF704793F06E
:1005D0007F4F04BF41F40021704730B54FF4607481
:1005E00001F0004521F000411CE700BF50EA010284
:1005F00008BF704730B54FF000050AE050EA01022D
:1006000008BF704730B511F0004502D5404261EB9C
:1006100041014FF4806404F132045FEA915C3FF4DD
:10062000D8AE4FF003025FEADC0C18BF03325FEA7A
:10063000DC0C18BF033202EBDC02C2F1200300FA2B
:1006400003FC20FA02F001FA03FE40EA0E0021FA50
:1006500002F11444BDE600BF70B54FF0FF0C4CF43E
:10066000E06C1CEA11541DBF1CEA135594EA0C0FF0
:1006700095EA0C0F00F0DEF82C4481EA030621EA2B
:100680004C5123EA4C5350EA013518BF52EA033566
:1006900041F4801143F4801338D0A0FB02CE4FF018
:1006A0000005E1FB02E506F00042E0FB03E54FF048
:1006B0000006E1FB03569CF0000F18BF4EF0010E40
:1006C000A4F1FF04B6F5007F64F5407404D25FEA3C
:1006D0004E0E6D4146EB060642EAC62141EA5551EF
:1006E0004FEAC52040EA5E504FEACE2EB4F1FD0C31
:1006F00088BFBCF5E06F1ED8BEF1004F08BF5FEAAF
:10070000500E50F1000041EB045170BD06F0004660
:1007100046EA010140EA020081EA0301B4EB5C040D
:10072000C2BFD4EB0C0541EA045170BD41F4801105
:100730004FF0000E013C00F3AB8014F1360FDEBF2A
:10074000002001F0004170BDC4F10004203C35DA06
:100750000C341BDC04F11404C4F1200500FA05F389
:1007600020FA04F001FA05F240EA020001F000422A
:1007700021F0004110EBD37021FA04F642EB0601A0
:100780005EEA430E08BF20EAD37070BDC4F10C04CA
:10079000C4F1200500FA04F320FA05F001FA04F28E
:1007A00040EA020001F0004110EBD37041F100017A
:1007B0005EEA430E08BF20EAD37070BDC4F1200585
:1007C00000FA05F24EEA020E20FA04F301FA05F2ED
:1007D00043EA020321FA04F001F0004121FA04F295
:1007E00020EA020000EBD3705EEA430E08BF20EA65
:1007F000D37070BD94F0000F0FD101F0004640009F
:1008000041EB010111F4801F08BF013CF7D041EA20
:10081000060195F0000F18BF704703F00046520024
:1008200043EB030313F4801F08BF013DF7D043EAF5
:100830000603704794EA0C0F0CEA135518BF95EAAB
:100840000C0F0CD050EA410618BF52EA4306D1D132
:1008500081EA030101F000414FF0000070BD50EA51
:10086000410606BF1046194652EA430619D094EADB
:100870000C0F02D150EA013613D195EA0C0F05D1C5
:1008800052EA03361CBF104619460AD181EA030119
:1008900001F0004141F0FE4141F470014FF00000D1
:1008A00070BD41F0FE4141F4780170BD70B54FF06C
:1008B000FF0C4CF4E06C1CEA11541DBF1CEA1355EC
:1008C00094EA0C0F95EA0C0F00F0A7F8A4EB0504CE
:1008D00081EA030E52EA03354FEA013100F08880C5
:1008E0004FEA03334FF0805545EA131343EA12638E
:1008F0004FEA022245EA111545EA10654FEA002643
:100900000EF000419D4208BF964244F1FD0404F5FB
:10091000407402D25B084FEA3202B61A65EB030557
:100920005B084FEA32024FF480104FF4002CB6EB14
:10093000020E75EB030E22BFB61A754640EA0C0094
:100940005B084FEA3202B6EB020E75EB030E22BFD4
:10095000B61A754640EA5C005B084FEA3202B6EB15
:10096000020E75EB030E22BFB61A754640EA9C00D4
:100970005B084FEA3202B6EB020E75EB030E22BFA4
:10098000B61A754640EADC0055EA060E18D04FEA62
:10099000051545EA16754FEA06164FEAC30343EA02
:1009A00052734FEAC2025FEA1C1CC0D111F4801FCF
:1009B0000BD141EA00014FF000004FF0004CB6E7C8
:1009C00011F4801F04BF01430020B4F1FD0C88BF67
:1009D000BCF5E06F3FF6AFAEB5EB030C04BFB6EB72
:1009E000020C5FEA500C50F1000041EB045170BD65
:1009F0000EF0004E4EEA113114EB5C04C2BFD4EB92
:100A00000C0541EA045170BD41F480114FF0000E15
:100A1000013C90E645EA060E8DE60CEA135594EA91
:100A20000C0F08BF95EA0C0F3FF43BAF94EA0C0F94
:100A30000AD150EA01347FF434AF95EA0C0F7FF409
:100A400025AF104619462CE795EA0C0F06D152EA5D
:100A500003353FF4FDAE1046194622E750EA410641
:100A600018BF52EA43067FF4C5AE50EA41047FF452
:100A70000DAF52EA43057FF4EBAE12E74FF0FF3CB7
:100A800006E000BF4FF0010C02E000BF4FF0010C88
:100A90004DF804CD4FEA410C7FEA6C5C4FEA430C01
:100AA00018BF7FEA6C5C1BD001B050EA410C0CBF50
:100AB00052EA430C91EA030F02BF90EA020F0020B2
:100AC000704710F1000F91EA030F58BF994208BF19
:100AD00090422CBFD8176FEAE37040F001007047D6
:100AE0004FEA410C7FEA6C5C02D150EA013C07D12D
:100AF0004FEA430C7FEA6C5CD6D152EA033CD3D078
:100B00005DF8040B704700BF8446104662468C4671
:100B10001946634600E000BF01B5FFF7B7FF0028A4
:100B200048BF10F1000F01BD4DF808EDFFF7F4FFCD
:100B30000CBF012000205DF808FB00BF4DF808ED58
:100B4000FFF7EAFF34BF012000205DF808FB00BF7B
:100B50004DF808EDFFF7E0FF94BF012000205DF89D
:100B600008FB00BF4DF808EDFFF7CEFF94BF012052
:100B700000205DF808FB00BF4DF808EDFFF7C4FF4B
:100B800034BF012000205DF808FB00BF4FEA410C94
:100B90007FEA6C5C02D150EA013C0AD14FEA430C77
:100BA0007FEA6C5C02D152EA033C02D14FF00000B4
:100BB00070474FF0010070474FEA410212F50012F2
:100BC00015D211D56FF47873B3EB625212D94FEA94
:100BD000C12343F0004343EA505311F0004F23FA7E
:100BE00002F018BF404270474FF00000704750EAD3
:100BF000013005D111F0004008BF6FF00040704790
:100C00004FF00000704700BF4A0011D212F50012E9
:100C100011D20DD56FF47873B3EB62520ED44FEA54
:100C2000C12343F0004343EA505323FA02F07047D4
:100C30004FF00000704750EA013002D14FF0FF3012
:100C400070474FF0000070474FEA4102B2F1E043B5
:100C500024BFB3F5001CDCF1FE5C0DD901F0004CA3
:100C60004FEAC0024CEA5070B2F1004F40EB8300F3
:100C700008BF20F00100704711F0804F21D113F11F
:100C80003872BCBF01F00040704741F480114FEA58
:100C90005252C2F11802C2F1200C10FA0CF320FAE1
:100CA00002F018BF40F001004FEAC1234FEAD323FE
:100CB00003FA0CFC40EA0C0023FA02F34FEA430368
:100CC000CCE77FEA625307D150EA01331EBF4FF0F1
:100CD000FE4040F44000704701F0004040F0FE400C
:100CE00040F40000704700BF53B94AB9002908BF5B
:100CF00000281CBF4FF0FF314FF0FF3000F0BEB9AD
:100D0000ADF1080C6DE904CE00F03CF8DDF804E02C
:100D1000DDE9022304B0704738B500220023044601
:100D20000D46FFF70BFF28B920462946BDE838409D
:100D300000F00AB8204605F1004100F005F84042F5
:100D400061EB410138BD00BFD0B50C4B0022064617
:100D50000F46FFF781FCFFF757FF0446FFF702FC41
:100D6000074B0022FFF778FC02460B463046394617
:100D7000FFF7BAFAFFF748FF2146D0BD0000F03D6B
:100D80000000F0412DE9F047089D8E460446884654
:100D9000002B4AD18A42174662D9B2FA82F64EB186
:100DA000C6F1200301FA06F820FA03F3B74043EA3C
:100DB0000808B4404FEA174E1FFA87FCB8FBFEF153
:100DC000230C0EFB118843EA084301FB0CF29A4204
:100DD00009D9FB1801F1FF3080F0EA809A4240F215
:100DE000E78002393B449A1AA3B2B2FBFEF00EFB35
:100DF000102243EA024300FB0CFC9C4509D9FB1876
:100E000000F1FF3280F0D6809C4540F2D3803B4415
:100E1000023840EA0140A3EB0C0300211DB1F3406E
:100E20000022C5E90032BDE8F0878B4205D90DB13B
:100E3000C5E9000100210846F5E7B3FA83F100296E
:100E400046D1734502D3824200F20581841A6EEBCB
:100E5000030201209046002DE5D0C5E90048E2E7F5
:100E6000002A00F09080B2FA82F6002E40F0A480B2
:100E70008A1A030C4FEA174E80B2BCB20121B2FBB2
:100E8000FEFC0EFB1C2243EA024304FB0CF29A42D6
:100E900007D9FB180CF1FF3802D29A4200F2E08029
:100EA000C4469B1AB3FBFEF20EFB123340EA034327
:100EB00002FB04F49C4207D9FB1802F1FF3002D276
:100EC0009C4200F2CA8002461B1B42EA0C40A5E786
:100ED000C1F120068B4022FA06F71F430EFA01F4F7
:100EE00020FA06F32EFA06FE4FEA1749234300FACA
:100EF00001F81FFA87FCBEFBF9F01C0C09FB10EE91
:100F000044EA0E4400FB0CFEA64502FA01F209D9A0
:100F10003C1900F1FF3A80F09C80A64540F2998090
:100F200002383C44A4EB0E041FFA83FEB4FBF9F331
:100F300009FB13444EEA044403FB0CFCA44508D906
:100F40003C1903F1FF3E80F08280A4457FD9023B2B
:100F50003C4443EA0040A4EB0C04A0FB02EC6445D3
:100F60007346E14662D35FD05DB1B8EB030264EB38
:100F7000090404FA06F622FA01F31E43CC40C5E93F
:100F8000006400214FE7B1FBF2FC010C41EA0E4185
:100F900080B240EA01423B4638463C46B846BE462F
:100FA0002026B1FBF7F1A2EB080241EA0C4166E70B
:100FB000014618E710462CE7C6F120022EFA02F38C
:100FC000B740B14020FA02F24FEA174E0A43B3FB92
:100FD000FEF8BCB20EFB1833110C41EA034108FBCA
:100FE00004F9B04089454FEA104380B23ED97918E0
:100FF00008F1FF3C01D289451FD8A1EB0901B1FBE3
:10100000FEF909FB04F80EFB191192B242EA014203
:10101000424529D2BA1809F1FF31C4D24245C2D2A1
:10102000A9F102013A44BEE7F0459DD2BEEB0203AE
:101030006CEB070C0138E14696E7A7EB0909494438
:10104000A8F1020CB1FBFEF909FB04F8DBE77346DB
:101050007FE7504666E70846FDE63B44023A33E741
:10106000ACF1020C3B441CE749469CE7A1EB0901AB
:10107000C446B1FBFEF909FB04F8C4E7704700BFA2
:1010800080B483B000AF0346FB71044AFB79137050
:1010900000BF0C37BD465DF8047B70476C03002031
:1010A00080B586B000AF3A601A460346FB710B4626
:1010B000BB7113467B710223BB750023FB73FF23B7
:1010C0003B74FF237B74FB79BB7497F820303B752E
:1010D0003B68002B10D07A79BB7D1344DBB201331F
:1010E000BB75BB7DFB74BB797B7507F110030621D3
:1010F000184600F01BFA07E0BB7DFB7407F11003F4
:101100000521184600F012FAFA79BB7D1344DAB2D1
:1011100097F820301344DAB2BB791344DBB2FB7387
:101120003B68002B16D00023FB750AE0FB7D3A6874
:1011300013441A78FB7B1344DBB2FB73FB7D013352
:10114000FB75FA7D7B799A42F0D37B791946386832
:1011500000F0ECF9FB7BDB43DBB2FB7307F10F0321
:101160000121184600F0E2F900BF1837BD4680BDE6
:1011700080B584B002AF3A601A460346FB710B4655
:10118000BB7113467B7100F0FDF97B79B979F87971
:10119000032200923A68FFF783FF00F0FBF9FB7926
:1011A000184600F04BF9034618460837BD4680BD87
:1011B00080B584B002AF0346FB710B46BB7113468A
:1011C0007B7100F0DFF97A1DB979F8790323009378
:1011D0000123FFF765FF00F0DDF9FB79184600F009
:1011E0002DF9034618460837BD4680BD80B588B046
:1011F00002AF3A601A460346FB710B46BB711346B9
:101200007B7100F0BFF97A1DB979F8790223009358
:101210000123FFF745FF00F0BDF93E4B00221A7095
:1012200000F0E2F80346002B04D13A4B01221A7079
:1012300000236BE007F10C030321184600F05AF974
:101240000346032B04D0334B01221A7000235DE0C8
:101250003B7BFA799A4207D0FB79FE2B04D02D4BC9
:1012600003221A70002351E07B7B1A467B790233FC
:101270009A4204D0274B04221A70002346E07B795F
:101280001946386800F036F938617B791A463B69AF
:10129000934204D01F4B01221A70002336E007F15D
:1012A0000C0303330121184600F024F90346012BF7
:1012B00004D0184B01221A70002327E03A7B7B7B75
:1012C0001344DAB2BB7B1344FB750023BB7509E002
:1012D000BB7D3A6813441A78FB7D1344FB75BB7DD4
:1012E0000133BB75BB7D3A699A42F1DCFB7DDB4380
:1012F000FB75FB7BFA7D9A4204D0064B02221A70E2
:10130000002303E0BA7B044B1A703B691846183778
:10131000BD4680BD6E0300206D03002080B586B001
:1013200002AF0346FB7100F02DF9F8790123009319
:10133000002300220021FFF7B3FE00F02BF9284B19
:1013400000221A7000F050F80346002B05D1254BFF
:1013500001221A704FF0FF333EE0224B00221A7038
:1013600007F108030421184600F0C4F80346042BD3
:1013700005D01C4B01221A704FF0FF332CE03B7A52
:10138000FA799A4208D0FB79FE2B05D0154B03223F
:101390001A704FF0FF331FE07B7A022B05D0114B00
:1013A00004221A704FF0FF3316E03A7A7B7A134426
:1013B000DAB2BB7A1344DBB2DB43FB73FB7AFA7B12
:1013C0009A4205D0074B02221A704FF0FF3303E018
:1013D000BA7A034B1A703B7A18461037BD4680BD67
:1013E0006D0300206E03002080B582B000AF0023A3
:1013F000BB800023FB71BB1D0121184600F07AF869
:101400000346002B01D1002313E03B797B71BB79AC
:101410003B713B79FF2B02D17B79FF2B07D0FB7906
:101420000133FB71FB790A2BE5D9002301E000BFF2
:10143000012318460837BD4680BD000080B584B042
:1014400000AF0346FB71284B00221A70FB79FE2B7C
:1014500044D0264B1B78002B40D0FFF7C5FF034636
:10146000002B04D1204B01221A70002337E0204BBF
:1014700000221A7007F108030421184600F03AF818
:101480000346042B04D0184B01221A70002326E0D7
:101490003B7AFA799A4204D0134B03221A70002344
:1014A0001DE07B7A022B04D00F4B04221A7000231C
:1014B00015E03A7A7B7A1344DAB2BB7A1344DBB292
:1014C000DB43FB73FB7AFA7B9A4204D0064B022281
:1014D0001A70002303E0BA7A054B1A7001231846EC
:1014E0001037BD4680BD00BF6E0300200000002005
:1014F0006D03002080B582B000AF786039600A4883
:101500000AF014FA3B689AB24FF0FF337968064844
:101510000AF041F90346002B01D0002300E03B68AC
:1015200018460837BD4680BDC404002080B483B08F
:1015300000AF7860396014E0104B1B785BB2002B71
:101540000FDB0E4B1B781A467B6819780C4B9954AD
:101550000A4B1B780133DAB2084B1A707B680133EF
:101560007B603B685A1E3A60002BE5D1034B1B7829
:1015700018460C37BD465DF8047B7047F003002029
:101580007003002080B500AF012004F0A1FE00BF71
:1015900080BD000080B500AF0A4B1B78002B0ED039
:1015A00009480AF08FF9074B1B781A464FF0FF33B2
:1015B000064905480AF064F8024B00221A7000BF81
:1015C00080BD00BFF0030020C40400207003002091
:1015D00080B400AFBFF34F8F00BF064BDB6803F44E
:1015E000E0620449044B1343CB60BFF34F8F00BF4D
:1015F00000BFFDE700ED00E00400FA0580B582B011
:1016000000AF04F023FE00237B604C4B1B6C4B4A65
:1016100043F080531364494B1B6C03F080537B6091
:101620007B6807F083F9454B5B6F444A43F0010345
:10163000536700BF414B5B6F03F00203002BF9D0EF
:101640003E4B1B6F3D4A23F4004313673B4B1B6F1C
:1016500023F40343394A43F402431367384B5B6D69
:10166000B3F1A53F04D1364B00225A65FFF7B0FF16
:1016700000F08CF800F008FA00F0F4F800F044F9FB
:1016800000F0D8FA10F080FE03F0ACFB02F048F94D
:10169000642004F01DFE02F049F90EF0C9F8294A51
:1016A000002129480EF00EF90346284A1360284A03
:1016B000002128480EF006F90346274A1360274AFE
:1016C000002127480EF0FEF80346264A1360264AFA
:1016D000002126480EF0F6F80346254A1360254AF5
:1016E000002125480EF0EEF80346244A1360244AF0
:1016F000002124480EF0E6F80346234A13600EF05A
:10170000BBF800220121012001F060FB40F24D10E6
:101710000EF06AF901220021012001F057FB40F28E
:101720004D100EF061F901220121002001F04EFB65
:1017300040F24D100EF058F900BFE2E700380240C9
:101740000028004024720108153B00080C05002009
:1017500048720108592D0008780500206C720108B4
:10176000692300087C0500209072010841210008CF
:1017700080050020B4720108A11D00088405002026
:10178000D8720108791D00088805002080B594B042
:1017900000AF07F11C0334220021184612F0B4FCFC
:1017A00007F1080300221A605A609A60DA601A6131
:1017B00000237B60294B1B6C284A43F08053136441
:1017C000264B1B6C03F080537B607B6800233B60DF
:1017D000234B1B68224A43F440431360204B1B6891
:1017E00003F440433B603B680123FB614FF48033CB
:1017F0003B6202237B634FF48003BB630423FB63E0
:10180000A2233B6402237B640823BB640223FB64A2
:1018100007F11C03184607F043FF0346002B01D0D5
:1018200002F0EEF90F23BB600223FB6000233B6153
:101830004FF4A0537B614FF48053BB6107F1080361
:101840000521184607F086F80346002B01D002F068
:10185000D7F900BF5037BD4680BD00BF00380240F9
:101860000070004080B584B000AF3B4600221A6093
:101870005A609A60DA60214B214A1A601F4B4FF47C
:1018800080325A601D4B00229A601C4B00221A6164
:101890001A4B01221A76194B002283F82020174B8D
:1018A0000022DA62154B174A9A62144B0022DA6062
:1018B000124B0122DA61114B002283F830200F4BCA
:1018C00001225A610D4804F027FD0346002B01D088
:1018D00002F096F90A233B6001237B600023BB6082
:1018E0003B461946054804F0F9FE0346002B01D09B
:1018F00002F086F900BF1037BD4680BD34040020D9
:10190000002001400100000F80B58CB000AF07F14E
:101910001C0300221A605A609A60DA601A6107F1AB
:101920000C0300221A605A609A60DA603B1D0022A4
:101930001A605A603C4B4FF080421A603A4B532277
:101940005A60394B00229A60374B4FF0FF32DA6011
:10195000354B00221A61344B00229A61324808F05C
:1019600073FB0346002B01D002F04AF90423FB610C
:1019700050233B6200237B620023BB620023FB6297
:1019800007F11C031946284809F000F80346002B0C
:1019900001D002F035F90023FB6001233B610023F5
:1019A0007B610023BB6107F10C03002219461E482E
:1019B00008F08EFE0346002B01D002F021F902232D
:1019C000FB6002233B6107F10C0304221946164811
:1019D00008F07EFE0346002B01D002F011F900232F
:1019E0007B600023BB603B1D19460F4809F02EFDAC
:1019F0000346002B01D002F003F900210A4808F049
:101A00004FFC0346002B01D002F0FAF804210648EF
:101A100008F06AFB0346002B01D002F0F1F800BF8A
:101A20003037BD4680BD00BF7C04002080B500AFCC
:101A3000124808F0ECF9124B124A1A60104B4FF49E
:101A400096325A600E4B00229A600D4B0022DA60EB
:101A50000B4B00221A610A4B0C225A61084B0022E0
:101A60009A61074B0022DA61054809F07FFD0346C1
:101A7000002B01D002F0C4F800BF80BD1405002087
:101A8000C4040020004C004080B58AB000AF07F1CC
:101A9000140300221A605A609A60DA601A61002307
:101AA0003B615F4B1B6B5E4A43F0040313635C4B6B
:101AB0001B6B03F004033B613B690023FB60584B45
:101AC0001B6B574A43F080031363554B1B6B03F0AA
:101AD0008003FB60FB680023BB60514B1B6B504ACB
:101AE00043F0010313634E4B1B6B03F00103BB6018
:101AF000BB6800237B604A4B1B6B494A43F00203DF
:101B00001363474B1B6B03F002037B607B6800236E
:101B10003B60434B1B6B424A43F008031363404B4B
:101B20001B6B03F008033B603B68002247F6404113
:101B30003C4805F0B5FB00224CF2F8313A4805F07C
:101B4000AFFB00224FF40041384805F0A9FB00220A
:101B50000421374805F0A4FB47F640437B6101238D
:101B6000BB610023FB6100233B6207F114031946AC
:101B70002C4805F0F5F81E237B610023BB61002390
:101B8000FB6107F114031946284805F0E9F8202302
:101B90007B610023BB610023FB6107F1140319463D
:101BA000204805F0DDF843F201037B610023BB61AF
:101BB0000023FB6107F1140319461B4805F0D0F818
:101BC0004CF2F8337B610123BB610023FB610023EE
:101BD0003B6207F114031946134805F0C1F84FF4AE
:101BE00000437B610123BB610023FB6100233B6257
:101BF00007F1140319460D4805F0B2F804237B6180
:101C00000123BB610023FB6100233B6207F1140346
:101C10001946074805F0A4F800BF2837BD4680BD27
:101C20000038024000080240000402400000024068
:101C3000000C024080B588B000AF464809F0EEFCC9
:101C400007F1180300221A605A60434B434A1A6096
:101C5000414B00225A60404B00229A603E4B404A62
:101C6000DA603D4B00221A613B4B00229A613A48F0
:101C700008F07EF80346002B01D001F0C1FF0023DD
:101C8000BB610023FB6107F118031946324809F0D4
:101C9000DDFB0346002B01D001F0B2FF314B602287
:101CA0001A602D4BDB6801331846FEF75BFC4FF0E2
:101CB00033322D4BFEF7D0FC02460B461046194638
:101CC0004FF00002294BFEF70FFB02460B46104671
:101CD0001946FEF799FF0346224A5360214B002222
:101CE0009A60204B00221A6100221E491A4808F00F
:101CF0008BFD0346002B01D001F082FF3B1D00222B
:101D00001A605A609A60DA601A6100233B60184BCF
:101D10001B6B174A43F001031363154B1B6B03F056
:101D200001033B603B6801237B600223BB6000230F
:101D3000FB6003233B6102237B613B1D19460D4879
:101D400005F00EF80021044808F0B6F800BF20376F
:101D5000BD4680BDC404002014050020000C0040D6
:101D60007FA219005C0500203333B33F0000F03F31
:101D7000003802400000024080B582B000AF7860B9
:101D8000054B1B78DBB2002B01D101F0CFFA1420F8
:101D90000DF02AFEF4E700BFF6030020000000006B
:101DA00080B58CB000AF7860002387F82F30002317
:101DB00087F82E30002387F82D30002387F82C3049
:101DC000002387F82B30002387F82A30002387F878
:101DD0002930002387F82830CB4B1B78DBB2002B4F
:101DE0000AD0C94B00221A70C8480CF007FAC7483D
:101DF0000CF092F901F0BAFD4FF40051C44805F01F
:101E000037FA0346002B73D197F82E30002B72D18E
:101E1000012387F82E3097F82F30072B57D801A2CF
:101E200052F823F0451E00085F1E0008831E0008BC
:101E3000A71E0008AF1E0008B71E0008BF1E00083E
:101E4000C71E0008B34B00221A70B34B01221A7050
:101E5000B24B01221A70B24B00221A703BE0AD4B1C
:101E600005221A70AF489FED9E0B00F041FBAA4B74
:101E700001221A70A94B00221A70A94B00221A7075
:101E800029E0A44B04221A70A7489FED950B00F09F
:101E90002FFBA14B00221A70A04B00221A70A04BFE
:101EA00001221A7017E09B4B01221A7013E0994B24
:101EB00002221A700FE0974B03221A700BE0954B29
:101EC00006221A7007E0934B07221A7003E00023E2
:101ED00087F82F3000BF97F82F3001335A4203F0B4
:101EE000070302F0070258BF534287F82F3002E081
:101EF000002387F82E300121854805F0B9F9034603
:101F0000002B14D197F82D30002B13D1012387F823
:101F10002D30804B1B78052B02D100F07DFF09E0AE
:101F20007C4B1B78042B05D100F086FF02E00023D8
:101F300087F82D304FF48051754805F099F9034624
:101F4000002B11D197F82930002B10D1012387F8ED
:101F50002930DFED762A9FED762A9FED631B9FEDFA
:101F6000640B00F0C1FF02E0002387F82930202134
:101F7000704805F07DF90346002B11D197F8283001
:101F8000002B10D1012387F82830DFED682A9FED60
:101F9000682A9FED591B9FED5A0B00F0A5FF02E048
:101FA000002387F828300221634805F061F90346D1
:101FB000002B27D10821604805F05AF90346002B71
:101FC00020D197F82A30002B40F08380012387F836
:101FD0002A30DFED562A9FED562A9FED431B9FEDD9
:101FE000440B00F081FF554B01221A7001F0A8FF4D
:101FF000524B00221A70012387F82C30012387F8F6
:102000002B3066E0002387F82A3002214A4805F089
:102010002FF90346002B27D197F82C30002B26D11F
:10202000012387F82C3000F045FF87ED090A97ED72
:10203000090A00F0CBFF87ED060B97ED060B01F0C8
:102040000FF84FF4C8700DF0CFFC3C4B01221A7012
:1020500001F066FF394B00221A7097ED091A97EDCF
:10206000060B01F055F802E0002387F82C30082118
:10207000314805F0FDF80346002B27D197F82B30A7
:10208000002B26D1012387F82B3000F013FF87EDBA
:10209000050A97ED050A00F099FF87ED020B97ED11
:1020A000020B00F0DDFF4FF4C8700DF09DFC234BD8
:1020B00001221A7001F03CFF204B00221A7097EDAC
:1020C000051A97ED020B01F09BF802E0002387F858
:1020D0002B3032200DF088FC7EE600BFAFF300808D
:1020E000000000000000F87F000000000000294010
:1020F0000000000000000440000000000000244038
:102100000000000000001240100500200C14012007
:1021100000040240FD030020F1030020F203002030
:10212000F303002020620108286201080000C84271
:10213000000000000008024000000240F6030020FA
:1021400080B58CB000AF78600023BB6200237B6257
:1021500000233B6207F10C0300221A605A609A6068
:10216000DA600023FB85FB8D322B40F08A800A2346
:10217000FB6001233B6100237B6107F10C031946DF
:10218000714804F0ABFA704804F00AF94FF0FF31DF
:102190006D4804F00AFA6C4804F092FAB8626A4892
:1021A00004F0D0F9B86AFEF7DDF95DA3D3E90023A6
:1021B000FEF752FA02460B46104619465AA3D3E9D7
:1021C0000023FEF773FB02460B4610461946FEF746
:1021D0003BFD0346FB61F869FEF7E6F954A3D3E93A
:1021E0000023FEF781F802460B461046194652A31B
:1021F000D3E90023FEF75AFB02460B461046194668
:10220000FEF722FD0346514A13600B23FB6007F1E2
:102210000C0319464C4804F061FA4B4804F0C0F82E
:102220004FF0FF31484804F0C0F9474804F048FA3D
:102230007862454804F086F9786AFEF793F938A386
:10224000D3E90023FEF708FA02460B46104619466A
:1022500035A3D3E90023FEF729FB02460B461046BF
:10226000194637A3D3E90023FEF7F6F902460B46D9
:1022700010461946FEF7E8FC0346354A1360002372
:10228000FB850C23FB6007F10C0319462E4804F074
:1022900025FA2D4804F084F84FF0FF312A4804F065
:1022A00084F9294804F00CFA3862274804F04AF906
:1022B0003B6A07EE903AF8EE677A9FED267A27EEB2
:1022C000877ADFED256AC7EE267A244BC3ED007AC4
:1022D000234BD3ED007AF5EEC07AF1EE10FA13DB62
:1022E0001E4B93ED007A1E4BD3ED007A77EE677AA2
:1022F000F0EEE77AB6EE007AF4EEC77AF1EE10FA75
:1023000002DD184B00221A70144B1B68144A13602C
:10231000FB8D0133FB8514200DF066FB23E700BF26
:102320006666666666660A400000000000FEAF4012
:102330001F85EB51B81ED53F4C37894160E5D03F32
:102340007CF0C1071F7C2E403404002000040020D4
:10235000040400200000C84200F07F45080400206B
:10236000040000202804002080B584B000AF78600D
:10237000554B00221A700023FB730023BB810023FE
:10238000FB72514B1B78002B1AD1BB89B3F57A7FB6
:1023900013D1FB7A002B07D14C489FED490B00F07D
:1023A000A7F80123FB7206E049489FED450B00F0BA
:1023B0009FF80023FB720023BB81BB890133BB81E3
:1023C000414B1B78012B0BD1424B1B681846FEF783
:1023D000EBF802460B46002043EC102B00F088F887
:1023E000394B1B78022B0BD13B4B1B681846FEF771
:1023F000DBF802460B46002043EC102B00F078F887
:10240000314B1B78032B0DD100F054FD10EE103A28
:102410001846FEF7C9F802460B46002043EC102B85
:1024200000F066F8284B1B78062B17D103F044FF09
:1024300002462A4B1B68D31A632B05D928489FED07
:10244000200B00F055F809E0264B93ED007B0020AF
:10245000B0EE470AF0EE670A00F04AF81A4B1B7814
:10246000072B19D103F028FF02461C4B1B68D31A17
:10247000632B05D91A489FED120B00F039F80BE0D9
:10248000194B1B881846FEF76DF802460B460020D4
:1024900043EC102B00F02CF8FB7B184600F09CFB63
:1024A000FB7B01335A4203F0030302F0030258BFDF
:1024B0005342FB7301200DF097FA62E7AFF30080FF
:1024C000000000000000F87FFD03002030620108DA
:1024D00038620108000400200404002020040020C9
:1024E00040620108180400201004002000000000D1
:1024F000F0B591B000AF87ED020B78607B68002BE0
:102500004DD00023FB6343E0FB6B7A6813441B78D8
:10251000002B05D18A4AFB6B13440B221A7034E05E
:10252000FB6B7A6813441B782F2B11D9FB6B7A68ED
:1025300013441B78392B0BD8FB6B7A6813441B7838
:10254000303BD9B27E4AFB6B13440A461A701CE03A
:10255000FB6B7A6813441B78402B11D9FB6B7A68AC
:1025600013441B785A2B0BD8FB6B7A6813441B78E7
:10257000353BD9B2724AFB6B13440A461A7004E029
:102580006F4AFB6B13440B221A70FB6B0133FB6326
:10259000FB6B032BB8DD6B4B00221A7011E3D7E9FC
:1025A0000223D7E90201FEF7F1FA0346002B40F0BF
:1025B00008835FA3D3E90023D7E90201FEF7BEFA3F
:1025C0000346002B09D15CA3D3E90023D7E902011C
:1025D000FEF7D2FA0346002B11D00023BB6307E0BD
:1025E000574ABB6B13440A221A70BB6B0133BB639F
:1025F000BB6B032BF4DD534B00221A70E1E2012385
:102600001E464FF000024FF00003D7E90201FEF72B
:1026100095FA0346002B01D100231E4687F8376048
:1026200097F83730002B05D0BC68FB6883F0004575
:10263000C7E90245D7E90201FEF7BEFA03463B634C
:10264000386BFDF79FFF02460B46D7E90201FDF705
:102650004BFE02460B46C7E90A233B6B092B77DC8E
:1026600097F8373083F00103DBB2002B70D0354B85
:1026700001221A703A6B344B83FB02139910D31763
:10268000C91A0B469B000B445B00D11ACAB22C4BF3
:102690001A704FF000022D4BD7E90A01FDF7DCFF5D
:1026A00002460B46C7E90A23D7E90A01FEF784FA76
:1026B00003467B627A6A244B83FB02139910D3177B
:1026C000C91A0B469B000B445B00D11ACAB21C4BC3
:1026D000DA707B6A1C4A82FB03129210DB17D31A52
:1026E0007B627A6A184B83FB02139910D317C91ABD
:1026F0000B469B000B445B00D11ACAB2104B9A7078
:102700007B6A114A82FB03129210DB17D31A7B6299
:102710007A6A0D4B83FB02139910D317C91A0B4623
:102720009B000B445B00D11ACAB2054B5A7048E2B9
:102730000000000000388FC0000000008087C34008
:10274000F8030020FC0300206766666600408F40A7
:102750003B6B092B50DC97F83730002B4CD0864B65
:1027600002221A70854B0A221A703A6B844B83FB43
:1027700002139910D317C91A0B469B000B445B0038
:10278000D11ACAB27D4B5A704FF000027D4BD7E987
:102790000A01FDF761FF02460B46C7E90A23D7E9A4
:1027A0000A01FEF709FA03463B623A6A744B83FB5F
:1027B00002139910D317C91A0B469B000B445B00F8
:1027C000D11ACAB26D4BDA703B6A6D4A82FB0312B2
:1027D0009210DB17D31A3B623A6A694B83FB0213F0
:1027E0009910D317C91A0B469B000B445B00D11AF2
:1027F000CAB2624B9A70E4E13B6B632B67DC97F8DB
:10280000373083F00103DBB2002B60D05A4B022239
:102810001A703A6B5A4B83FB02139910D317C91ADB
:102820000B469B000B445B00D11ACAB2534B5A7043
:102830003B6B534A82FB03129210DB17D31A3B63A4
:102840003A6B4F4B83FB02139910D317C91A0B46EF
:102850009B000B445B00D11ACAB2484B1A704FF070
:102860000002484BD7E90A01FDF7F6FE02460B4687
:10287000C7E90A23D7E90A01FEF79EF90346FB617F
:10288000FA693F4B83FB02139910D317C91A0B4601
:102890009B000B445B00D11ACAB2384BDA70FB695B
:1028A000374A82FB03129210DB17D31AFB61FA69D5
:1028B000334B83FB02139910D317C91A0B469B00A5
:1028C0000B445B00D11ACAB22C4B9A7079E13B6B76
:1028D000632B5BDC97F83730002B57D0264B042254
:1028E0001A70264B0A221A703A6B254B83FB02138F
:1028F0009910D317C91A0B469B000B445B00D11AE1
:10290000CAB21E4B9A703B6B1D4A82FB0312921097
:10291000DB17D31A3B633A6B194B83FB02139910F5
:10292000D317C91A0B469B000B445B00D11ACAB2DD
:10293000124B5A704FF00002134BD7E90A01FDF712
:102940008BFE02460B46C7E90A23D7E90A01FEF7C8
:1029500033F90346BB61BA69094B83FB0213991033
:10296000D317C91A0B469B000B445B00D11ACAB29D
:10297000024BDA7025E100BFFC030020F8030020C1
:102980006766666600005940000024403B6BB3F563
:102990007A7F67DA97F8373083F00103DBB2002BD8
:1029A00060D0894B04221A703A6B884B83FB021368
:1029B0009910D317C91A0B469B000B445B00D11A20
:1029C000CAB2834B9A703B6B804A82FB031292100F
:1029D000DB17D31A3B633A6B7C4B83FB02139910D2
:1029E000D317C91A0B469B000B445B00D11ACAB21D
:1029F000774B5A703B6B754A82FB03129210DB17C0
:102A0000D31A3B633A6B714B83FB02139910D317B4
:102A1000C91A0B469B000B445B00D11ACAB26C4B1F
:102A20001A704FF000026B4BD7E90A01FDF714FE54
:102A300002460B46C7E90A23D7E90A01FEF7BCF8AC
:102A400003467B617A69614B83FB02139910D317AC
:102A5000C91A0B469B000B445B00D11ACAB25C4BEF
:102A6000DA70AEE03B6BB3F57A7F47DA97F8373030
:102A7000002B43D0544B00221A703A6B534B83FB0C
:102A800002139910D317C91A0B469B000B445B0025
:102A9000D11ACAB24E4BDA703B6B4C4A82FB03121E
:102AA0009210DB17D31A3B633A6B484B83FB02133C
:102AB0009910D317C91A0B469B000B445B00D11A1F
:102AC000CAB2434B9A703B6B404A82FB031292108E
:102AD000DB17D31A3B633A6B3C4B83FB0213991011
:102AE000D317C91A0B469B000B445B00D11ACAB21C
:102AF000374B5A70364B0A221A7062E03B6B42F237
:102B00000F7293425DDC97F8373083F00103DBB23C
:102B1000002B56D02C4B00221A703A6B2B4B83FBA8
:102B200002139910D317C91A0B469B000B445B0084
:102B3000D11ACAB2264BDA703B6B244A82FB0312CD
:102B40009210DB17D31A3B633A6B204B83FB0213C3
:102B50009910D317C91A0B469B000B445B00D11A7E
:102B6000CAB21B4B9A703B6B184A82FB031292103D
:102B7000DB17D31A3B633A6B144B83FB0213991098
:102B8000D317C91A0B469B000B445B00D11ACAB27B
:102B90000F4B5A703B6B0D4A82FB03129210DB17EE
:102BA000D31A3B633A6B094B83FB02139910D3177B
:102BB000C91A0B469B000B445B00D11ACAB2044BE6
:102BC0001A704437BD46F0BDFC0300206766666698
:102BD000F80300200000244080B584B000AF034615
:102BE000FB7100224FF40041544804F059FB0022CD
:102BF0000421534804F054FB00222021514804F0E2
:102C00004FFB00224FF400514F4804F049FBFB7981
:102C10004E4AD35CDBB21A464D4B9B5CFB73FB7B8D
:102C200003F00103DBB21A460821464804F038FBE2
:102C3000FB7B5B10DBB203F00103DBB21A464FF4FF
:102C40008061414804F02CFBFB7B9B10DBB203F05E
:102C50000103DBB21A4610213A4804F021FBFB7B4A
:102C6000DB10DBB203F00103DBB21A464FF48051F4
:102C7000354804F015FBFB7B1B11DBB203F00103AD
:102C8000DBB21A4640212F4804F00AFBFB7B5B11A4
:102C9000DBB203F00103DBB21A464FF4807129481E
:102CA00004F0FEFAFB7B9B11DBB203F00103DBB205
:102CB0001A464FF40061244804F0F2FA254B1B78C1
:102CC000DBB21A46FB7942FA03F303F00103002B4F
:102CD00014BF01230023DBB21A464FF400711948D8
:102CE00004F0DEFAFB79032B24D801A252F823F07A
:102CF000012D00080F2D00081B2D0008272D0008AE
:102D000001224FF400410D4804F0CAFA12E00122FA
:102D100004210B4804F0C4FA0CE0012220210948E8
:102D200004F0BEFA06E001224FF40051064804F018
:102D3000B7FA00BF00BF1037BD4680BD000002409B
:102D4000000C02400004024000080240F80300208A
:102D5000FC710108FC03002080B582B000AF7860F0
:102D6000154B01221A70154B01221A70144B0022C8
:102D70001A70144BFA221A70134BFA221A700E4B67
:102D80001B780E4A11780E4A1278184600F01EF889
:102D90000C4B1B7818460CF027FE0B4B1B78082BAE
:102DA000EDD901220121012000F010F8064B1B781B
:102DB00018460CF019FEE2E7F1030020F2030020B0
:102DC000F3030020F4030020F503002080B582B057
:102DD00000AF0346FB710B46BB7113467B71FB7959
:102DE0001A4640210A4804F05BFABB791A464FF4B0
:102DF0000041084804F054FA7B791A464FF48041A8
:102E0000044804F04DFA00BF0837BD4680BD00BF3E
:102E1000000802400004024080B500AF054B0122CB
:102E20001A7000F001FFFEF705FF024B00221A7036
:102E300000BF80BDF603002080B500AF054B012226
:102E40001A7000F069FFFEF7F5FE024B00221A70BF
:102E500000BF80BDF603002080B483B000AF87EDD3
:102E6000010AD7ED017AF5EEC07AF1EE10FA02D53B
:102E70004FF000037B60D7ED017A9FED0A7AF4EE04
:102E8000C77AF1EE10FA01DD074B7B60074A7B68D9
:102E90001360074B01221A7000BF0C37BD465DF866
:102EA000047B70470000C8420000C8422404002090
:102EB0002804002080B400AF084B1B78002B02D000
:102EC000074B1B6801E0074B1B6807EE903AB0EE1A
:102ED000670ABD465DF8047B704700BF28040020E8
:102EE000240400200804002080B586B000AF87EDE0
:102EF000040B87ED021B87ED012AC7ED002A4FF076
:102F000000024FF00003D7E90401FDF717FE034666
:102F1000002B47D14FF00002244BD7E90201FDF707
:102F20002BFE0346002B3DD1D7E90223D7E904014C
:102F3000FDF718FE0346002B34D11D49D7E90423C1
:102F4000C1E900231B49D7E90223C1E9002397ED1A
:102F5000007AD7ED017AB4EEE77AF1EE10FA16DDD9
:102F6000D7ED017AF5EEC07AF1EE10FA0FDBD7ED6E
:102F7000007A9FED117AF4EEC77AF1EE10FA06D8D6
:102F80000E4A7B6813600E4A3B68136006E00B4BE9
:102F90004FF000021A600A4B0A4A1A600A4B0122DB
:102FA0001A7000E000BF1837BD4680BD00005940D0
:102FB00008000020100000200000C8422C0400205F
:102FC000180000200000C8423004002080B582B004
:102FD00000AF87ED010AD7ED017AF5EEC07AF1EE88
:102FE00010FA02D54FF000037B60D7ED017A9FED18
:102FF000177AF4EEC77AF1EE10FA01DD144B7B601C
:103000007868FDF7D1FA4FF00002124BFDF74EFC45
:1030100002460B46104619464FF000020E4BFDF7D4
:103020001BFB02460B46104619464FF000020B4BA5
:10303000FDF75CF902460B4643EC172BB0EE470A4E
:10304000F0EE670A0837BD4680BD00BF0000C842E9
:103050000000C84200005940000024400000044025
:1030600080B586B000AF87ED000BD7E90023C7E934
:1030700004234FF000024FF00003D7E90401FDF7ED
:103080005DFD0346002B05D04FF000024FF000031A
:10309000C7E904234FF000021B4BD7E90401FDF7F9
:1030A0006BFD0346002B04D04FF00002164BC7E91E
:1030B0000423164BDB680133BB60B868FDF752FA96
:1030C000D7E90423FDF7C8FA02460B461046194615
:1030D0004FF000020C4BFDF7E9FB02460B46104691
:1030E0001946FDF791FD0346FB60FA68BB689A42FA
:1030F00001D9BB68FB60054B1B68FA685A6300BFC7
:103100001837BD4680BD00BF00005940140500209F
:1031100080B584B000AF87ED020B87ED011A2F490F
:10312000D7E90223C1E900232D4A7B6813602B4BAA
:10313000D3E900012B4BD3E90023FDF713FD034630
:10314000002B43D0254BD3E900014FF00002264B62
:10315000FDF7CCF802460B462249C1E90023214B7A
:10316000D3E900014FF00002204BFDF705FD0346B7
:10317000002B05D01B494FF000021C4BC1E9002376
:103180001B4B93ED007A164BD3ED007AB4EEE77A41
:10319000F1EE10FA03DD164BD3ED007A06E0104B8A
:1031A000D3ED007AB7EE007A77EE877A104BC3ED55
:1031B000007A0F4BD3ED007A9FED0E7AF4EEC77ACA
:1031C000F1EE10FA02DD0A4B0B4A1A600B4B01229A
:1031D0001A7000BF1037BD4680BD00BF0800002038
:1031E0002C040020100000200000E03F00005940A7
:1031F000180000200000C8420000C842300400202F
:1032000080B584B000AF87ED020B87ED011A2F491E
:10321000D7E90223C1E900232D4A7B6813602B4BB9
:10322000D3E900012B4BD3E90023FDF791FC0346C2
:10323000002B44D0254BD3E900014FF00002264B70
:10324000FDF752F802460B462249C1E90023214B03
:10325000D3E900014FF000024FF00003FDF76EFCD0
:103260000346002B06D01B494FF000024FF000032D
:10327000C1E90023194B93ED007A154BD3ED007A89
:10328000B4EEE77AF1EE10FA03D5144BD3ED007AE1
:1032900006E00F4BD3ED007AB7EE007A77EEC77AEF
:1032A0000E4BC3ED007A0D4BD3ED007AF5EEC07AEC
:1032B000F1EE10FA03D5094B4FF000021A60084BEB
:1032C00001221A7000BF1037BD4680BD10000020DB
:1032D00018000020080000200000E03F2C0400201F
:1032E0003004002080B400AF064BD3E9002343EC48
:1032F000172BB0EE470AF0EE670ABD465DF8047B77
:10330000704700BF0800002080B400AF064BD3E92F
:10331000002343EC172BB0EE470AF0EE670ABD46D8
:103320005DF8047B704700BF10000020B0B586B088
:1033300000AF01F017FA0346002B2CD001F066FA1B
:1033400010EE103A1846FDF72FF902460B46C7E972
:1033500004234FF000024FF00003D7E90401FDF70A
:10336000EDFB0346002B05D04FF000024FF00003A9
:10337000C7E904234FF00002824BD7E90401FDF7AF
:10338000FBFB0346002B00F0AA804FF000027D4BB0
:10339000C7E90423A3E07C4B1B78002B29D07B4B8F
:1033A0001B681846FDF700F902460B46C7E90423DF
:1033B0004FF000024FF00003D7E90401FDF7BEFB18
:1033C0000346002B05D04FF000024FF00003C7E981
:1033D00004234FF000026B4BD7E90401FDF7CCFB4F
:1033E0000346002B7BD04FF00002664BC7E9042355
:1033F00075E0674B1B78002B4DD0664B93ED007A40
:10340000654BD3ED007A77EE677AB7EE007AF4EE8B
:10341000C77AF1EE10FA3EDB604B93ED007A5E4B1B
:10342000D3ED007A77EE676A5A4B93ED007A5A4BE8
:10343000D3ED007A37EE677AC6EE877A9FED587A39
:1034400067EE877A17EE900AFDF7AEF802460B4654
:10345000C7E904234FF000024FF00003D7E904014D
:10346000FDF76CFB0346002B05D04FF000024FF038
:103470000003C7E904234FF00002424BD7E90401DF
:10348000FDF77AFB0346002B29D04FF000023D4B9D
:10349000C7E9042323E0414BD3ED007AB0EE007A74
:1034A000F4EEC77AF1EE10FA03D53C4B4FF0000270
:1034B0001A603A4BD3ED007A9FED3A7AF4EEC77A70
:1034C000F1EE10FA02DD354B374A1A60334B1B68B8
:1034D0001846FDF769F802460B46C7E90423334B4B
:1034E000DB6801333B60284B1B78002B64D001F074
:1034F00039F9034683F00103DBB2002B5CD0234B88
:103500001B681846FDF750F84FF000021D4BFDF701
:10351000CDF902460B46104619464FF00002244BE7
:10352000FDF79AF802460B46104619464FF0000286
:10353000204BFCF7DBFE02460B46C7E902234FF0A7
:1035400000024FF00003D7E90201FDF7F7FA034646
:10355000002B05D04FF000024FF00003C7E9022313
:103560004FF00002074BD7E90201FDF705FB0346C8
:10357000002B00F0AF804FF00002024BC7E902239E
:10358000A8E000BF000059402804002024040020C7
:1035900030040020180000202C0400200804002023
:1035A0000000C8420000C4420000C84214050020C8
:1035B0000000244000000440594B1B78002B6CD0C5
:1035C00001F0D0F8034683F00103DBB2002B64D096
:1035D000544BD3E90001544BD3E90023FCF784FE9C
:1035E00002460B4614461D464FF000024F4BD7E9EA
:1035F0000401FDF75BF902460B4620462946FDF71C
:103600002BF802460B4610461946474BD3E90023D8
:10361000FCF76CFE02460B46C7E90223424BD3E996
:103620000023D7E90201FDF789FA0346002B04D0F5
:103630003D4BD3E90023C7E902233A4BD3E90023EA
:10364000D7E90201FDF798FA0346002B04D0354B69
:10365000D3E90023C7E902234FF000024FF0000333
:10366000D7E90201FDF76AFA0346002B05D04FF0B7
:1036700000024FF00003C7E902234FF000022B4B7A
:10368000D7E90201FDF778FA0346002B22D04FF06C
:103690000002264BC7E902231CE04FF00002234B37
:1036A000D7E90401FDF702F902460B461046194618
:1036B0004FF000021E4BFCF7CFFF02460B461046B0
:1036C00019464FF000021B4BFCF710FE02460B465A
:1036D000C7E902233868FCF745FFD7E90223FCF766
:1036E000BBFF02460B46104619464FF000020F4B37
:1036F000FDF7DCF802460B4610461946FDF784FA42
:1037000003467B607A683B689A4201D93B687B60DC
:10371000094B1B687A685A6300BF1837BD46B0BDB5
:103720003004002010000020080000200000594054
:1037300000002440000004401405002080B400AFC5
:10374000034B1B781846BD465DF8047B704700BFED
:10375000FD0300200000000080B582B000AF78605B
:103760007B68002B44DB7B68072B41DC7B68DAB28B
:10377000254B1A707B68072B3CD801A252F823F026
:10378000A1370008F5370008F5370008F5370008BD
:10379000D3370008B5370008F5370008F5370008BB
:1037A0001A4B01221A701A4B01221A70194B00226F
:1037B0001A7020E018489FED120BFEF799FE134B8C
:1037C00001221A70124B00221A70124B00221A703A
:1037D00011E012489FED0A0BFEF78AFE0B4B002208
:1037E0001A700B4B00221A700A4B01221A7002E069
:1037F00000BF00E000BF0837BD4680BDAFF30080CA
:10380000000000000000F87FFD030020F10300200D
:10381000F2030020F303002020620108286201085F
:1038200080B500AF054B1B781A46054B53F8223084
:103830001846FFF791FF00BF80BD00BFFD030020C9
:10384000FC72010880B400AF034B01221A7000BF64
:10385000BD465DF8047B70471005002080B588B038
:1038600000AF07F1080300221A605A609A60DA601C
:103870001A61284BD3F8C832FB61F86904F0A0FB49
:1038800024480AF0BBFC23480AF046FC224B5B6943
:10389000214A43F08003536100237B6002E07B6890
:1038A00001337B607B6842F20F729342F7D91A4B67
:1038B0005B69194A23F080035361174B5B6B164A0F
:1038C00023F08003536300233B60134B1B6B124AAE
:1038D00043F001031363104B1B6B03F001033B60C8
:1038E0003B684FF4C053BB600123FB6000233B6186
:1038F00000237B6107F108031946084803F030FAFA
:1039000000224FF4C051054803F0CAFC00BF203725
:10391000BD4680BD0C14012000380240000002406A
:1039200080B500AFFFF79AFF00BF80BD80B582B0C1
:1039300000AF0D4B5B6B0C4A43F0800353630023D5
:103940007B60094B5B6C084A43F480435364064B2D
:103950005B6C03F480437B607B680EF015FD00BF59
:103960000837BD4680BD00BF0038024080B582B038
:1039700000AF00237B60244B1B6C234A43F0805331
:103980001364214B1B6C03F080537B607B6804F055
:10399000CDFF1D4B5B6F1C4A43F00103536700BF13
:1039A000194B5B6F03F00203002BF9D0164B1B6F12
:1039B000154A23F400431367134B1B6F23F403438F
:1039C000114A43F402431367104B4FF0A5325A6576
:1039D000FFF744FFC82002F07BFC72B600BF0C4B1F
:1039E00000221A600A4B00225A60094B00229A609A
:1039F000084B094A1A60BFF34F8F00BFBFF36F8FA8
:103A000000BFFDF7E5FD00BF003802400028004080
:103A100010E000E0F0FF0120EFBEADDEB0B582B0F7
:103A200000AF78607B681B68B3F1804F5FD17B6823
:103A30001B7F012B5BD10021786806F0E9FF03466C
:103A40009AB22D4B1A800421786806F0E1FF0346F4
:103A50009AB22A4B1A80284B1B88002B38D0274B50
:103A60001B881846FCF77EFD4FF00002244BFCF744
:103A7000F3FD02460B4614461D461F4B1B88184695
:103A8000FCF780FD02460B4620462946FCF70EFF58
:103A900002460B461B49C1E900231A4BD3E900013A
:103AA0004FF00002164BFDF767F80346002B05D0D8
:103AB00014494FF00002124BC1E900230E4B1B8842
:103AC0001A46114B93FBF2F39AB2104B1A8009E09D
:103AD0000C494FF000024FF00003C1E900230B4BEB
:103AE00000221A8002F0E8FB0346094A136000BF77
:103AF0000837BD46B0BD00BF0C0400200E040020F6
:103B0000000059401804002040420F00100400201B
:103B10002004002080B588B000AF78600023FB61EE
:103B200001F098F900F002FE0346002B1FD002F0CE
:103B3000C3FBB861FB69002B02D1BB69132B07D80B
:103B4000FB69002B06D0BA69FB69D31A632B01D934
:103B5000012300E000237B617B69002B07D001F08B
:103B60009FF80346002B02D002F0A6FBF86100F09C
:103B7000F9FD0346002B27D000F048FE87ED040A2C
:103B80003869FCF711FD4FF00002114BFCF78EFE77
:103B900002460B46104619464FF000020D4BFCF74B
:103BA0005BFD02460B46104619464FF000020A4BD9
:103BB000FCF79CFB02460B46C7E9022397ED021B6C
:103BC00097ED040A00F02CFF01200BF00DFFA7E792
:103BD00000005940000024400000044080B582B03D
:103BE00000AF78607B681B68044A934201D102F001
:103BF0004FFB00BF0837BD4680BD00BF001000402E
:103C000080B400AF72B600BF00BFFDE780B500AF63
:103C1000FDF7B8FC06210348FDF788FCFDF7BAFC68
:103C200000BF80BD7C73010880B582B000AFFDF796
:103C3000FDFE0020FDF724FA2F4B64221A702F4B53
:103C400064221A70FE20FDF769FB0346002B06DA9A
:103C5000294BFA221A70294BFA221A7042E0FA1DF7
:103C6000012315210120FDF7C1FA00223421012092
:103C7000FDF79EFA2D23224A06210120FDF778FA4E
:103C80000346002B0BD1012234210120FDF790FACD
:103C9000194BFA221A70194BFA221A7022E00122EB
:103CA00034210120FDF784FAFFF7B0FF124BFA220E
:103CB0001A70124B00221A7012489FED0D0BFEF77E
:103CC00017FC114B01221A70104B00221A70104B76
:103CD00001221A70084BFA221A70084BFA221A7045
:103CE000FDF7A8FF0837BD4680BD00BFAFF30080D9
:103CF000000000000000F87FF4030020F50300201E
:103D00001C73010850620108F1030020F203002037
:103D1000F30300200000000080B582B000AFFDF783
:103D200085FE0020FDF7ACF92F4B64221A702F4B53
:103D300064221A70FE20FDF7F1FA0346002B06DA22
:103D4000294BFA221A70294BFA221A7042E0FA1D06
:103D5000012315210120FDF749FA00223421012019
:103D6000FDF726FA2D23224A06210120FDF700FA4D
:103D70000346002B0BD1012234210120FDF718FA54
:103D8000194BFA221A70194BFA221A7022E00122FA
:103D900034210120FDF70CFAFFF738FF124BFA220D
:103DA0001A70124B00221A7012489FED0D0BFEF78D
:103DB0009FFB114B01221A70104B00221A70104BFE
:103DC00001221A70084BFA221A70084BFA221A7054
:103DD000FDF730FF0837BD4680BD00BFAFF3008060
:103DE000000000000000F87FF4030020F50300202D
:103DF0004C73010850620108F1030020F203002017
:103E0000F303002080B584B000AF0346FB71FDF7DB
:103E10000DFE0020FDF734F93F4B64221A703F4B32
:103E200064221A70FE20FDF779FA0346002B02DAAD
:103E30004FF0FF336CE007F1080202233821012024
:103E4000FDF7D4F90346022B02D04FF0FF335FE0B9
:103E50003B7A1A467B7A1B021343FB600022342113
:103E60000120FDF7A5F9FB79092B24D1FB68DBB212
:103E70001A4609210120FDF79BF90346002B07DABA
:103E8000012234210120FDF793F94FF0FF333FE089
:103E9000FB681B12DBB21A460A210120FDF788F9E4
:103EA0000346002B2CDA012234210120FDF780F992
:103EB0004FF0FF332CE0FB68DBB21A460B210120E8
:103EC000FDF776F90346002B07DA012234210120A1
:103ED000FDF76EF94FF0FF331AE0FB681B12DBB2FF
:103EE0001A460C210120FDF763F90346002B07DA7F
:103EF000012234210120FDF75BF94FF0FF3307E089
:103F0000012234210120FDF753F9FDF793FE002330
:103F100018461037BD4680BDF4030020F50300208D
:103F200080B500AF0920FFF76DFF0346184680BD3E
:103F300080B500AF0B20FFF765FF0346184680BD34
:103F400080B500AFFDF772FD0020FDF799F82F4B0B
:103F500064221A702E4B64221A70FE20FDF7DEF9DF
:103F60000346002B02DA4FF0FF334CE000223421ED
:103F70000120FDF71DF9002209210120FDF718F9A4
:103F80000346002B07DA012234210120FDF710F946
:103F90004FF0FF3337E000220A210120FDF708F936
:103FA0000346002B07DA012234210120FDF700F936
:103FB0004FF0FF3327E0FF220B210120FDF7F8F837
:103FC0000346002B07DA012234210120FDF7F0F827
:103FD0004FF0FF3317E003220C210120FDF7E8F832
:103FE0000346002B07DA012234210120FDF7E0F817
:103FF0004FF0FF3307E0012234210120FDF7D8F80C
:10400000FDF718FE0023184680BD00BFF403002012
:10401000F503002080B582B000AF00237B60124B17
:104020005B6C114A43F4804353640F4B5B6C03F4A5
:1040300080437B607B6800233B600B4B1B6C0A4A10
:1040400043F080531364084B1B6C03F080533B60B8
:104050003B6800220F216FF0010002F049FE00BF13
:104060000837BD4680BD00BF0038024080B58AB029
:1040700000AF786007F1140300221A605A609A605A
:10408000DA601A617B681B68174A934227D10023C4
:104090003B61164B5B6C154A43F480735364134BBE
:1040A0005B6C03F480733B613B690023FB600F4B47
:1040B0001B6B0E4A43F0040313630C4B1B6B03F0A2
:1040C0000403FB60FB6807237B610323BB610023C0
:1040D000FB6107F114031946054802F041FE00BFD9
:1040E0002837BD4680BD00BF002001400038024097
:1040F0000008024080B58AB000AF786007F1140371
:1041000000221A605A609A60DA601A617B681B6844
:10411000B3F1804F33D100233B611B4B1B6C1A4A18
:1041200043F001031364184B1B6C03F001033B6164
:104130003B690023FB60144B1B6B134A43F00103E4
:104140001363114B1B6B03F00103FB60FB6820231F
:104150007B610223BB610023FB6100233B620123DF
:104160007B6207F114031946084802F0F9FD0022AA
:1041700005211C2002F0BCFD1C2002F0D5FD00BF73
:104180002837BD4680BD00BF003802400000024015
:1041900080B58AB000AF786007F1140300221A607E
:1041A0005A609A60DA601A617B681B68194A934208
:1041B0002BD100233B61184B1B6C174A43F400239F
:1041C0001364154B1B6C03F400233B613B69002314
:1041D000FB60114B1B6B104A43F0010313630E4B42
:1041E0001B6B03F00103FB60FB6801237B6112235F
:1041F000BB610123FB6103233B6208237B6207F160
:1042000014031946054802F0ABFD00BF2837BD4630
:1042100080BD00BF004C004000380240000002405A
:1042200080B582B000AF78607B681B68084A934213
:1042300009D1084B1B6C074A23F4002313640121A6
:10424000054802F021FF00BF0837BD4680BD00BF12
:10425000004C0040003802400000024080B485B0AD
:1042600000AF78607B681B680B4A93420DD1002336
:10427000FB600A4B1B6C094A43F008031364074BAD
:104280001B6C03F00803FB60FB6800BF1437BD46DE
:104290005DF8047B704700BF000C0040003802400E
:1042A00080B483B000AF78607B681B68074A934294
:1042B00005D1074B1B6C064A23F00803136400BFAB
:1042C0000C37BD465DF8047B704700BF000C004012
:1042D0000038024080B58EB000AF78600023FB62EA
:1042E0000023BB620023FB60334B1B6C324A43F05C
:1042F00010031364304B1B6C03F01003FB60FB686E
:1043000007F1100207F114031146184604F03CFCB3
:104310003B6AFB62FB6A002B03D104F00DFC78635F
:1043200004E004F009FC03465B007B637B6B234ADB
:10433000A2FB03239B0C013BBB62214B214A1A6069
:104340001F4B40F2E732DA601D4ABB6A53601C4BD8
:1043500000221A611A4B00229A60194B00229A61BE
:10436000174805F03BFC034687F8333097F83330A5
:10437000002B1BD1124805F08BFC034687F8333025
:1043800097F83330002B11D1362002F0CDFC7B683A
:104390000F2B08D800227968362002F0A9FC0A4ABF
:1043A0007B68136002E0012387F8333097F83330DD
:1043B00018463837BD4680BD0038024083DE1B43B7
:1043C0008C050020001000407800002080B400AF71
:1043D00000BFFDE780B400AF00BFFDE780B400AFD1
:1043E00000BFFDE780B400AF00BFFDE780B400AFC1
:1043F00000BFFDE780B400AF00BFBD465DF8047BA1
:104400007047000080B500AF024806F071F800BFA9
:1044100080BD00BF8C05002080B500AF024803F0CE
:1044200001F900BF80BD00BFE828012080B500AFC2
:10443000024806F05DF800BF80BD00BF7C0400208C
:1044400080B400AF01231846BD465DF8047B704779
:1044500080B582B000AF786039600FF055FF034639
:1044600016221A604FF0FF3318460837BD4680BD4C
:1044700080B582B000AF78604FF0FF317868FFF709
:10448000E7FF00BFFDE780B586B000AFF860B96018
:104490007A6000237B610AE0AFF300800146BB68CD
:1044A0005A1CBA60CAB21A707B6901337B617A699F
:1044B0007B689A42F0DB7B6818461837BD4680BDA2
:1044C00080B586B000AFF860B9607A6000237B6188
:1044D00009E0BB685A1CBA601B781846AFF300802D
:1044E0007B6901337B617A697B689A42F1DB7B6887
:1044F00018461837BD4680BD80B483B000AF7860E1
:104500004FF0FF3318460C37BD465DF8047B70470B
:1045100080B483B000AF786039603B684FF40052DC
:104520005A60002318460C37BD465DF8047B70477F
:1045300080B483B000AF7860012318460C37BD46C5
:104540005DF8047B704780B485B000AFF860B96057
:104550007A60002318461437BD465DF8047B704727
:1045600080B586B000AF7860144A154BD31A7B61D2
:104570007B693B61134B1B68002B02D1114B124A24
:104580001A60104B1A687B6813443A699A4207D242
:104590000FF0BAFE03460C221A604FF0FF3309E019
:1045A000084B1B68FB60074B1A687B681344054A7D
:1045B0001360FB6818461837BD4680BDF0FF012028
:1045C00000040000D40500203831012080B400AF81
:1045D000064BD3F88830054A43F47003C2F888309C
:1045E00000BFBD465DF8047B704700BF00ED00E0F2
:1045F00080B483B000AF78607B68002B02DB7B68FF
:10460000072B01DD054B03E0054A7B6852F8233098
:1046100018460C37BD465DF8047B7047DC62010824
:10462000380000200FB480B5B2B000AF154B1B7836
:10463000DBB283F00103DBB2002B1CD107F1D40302
:104640003B60381D3B68D7F8D020C0210FF04EFDED
:10465000C7F8C400D7F8C430002B0DDDD7F8C4303C
:10466000BF2B09D8D7F8C4309AB23B1D1146184663
:104670000DF054FF00E000BFC837BD46BDE88040E4
:1046800004B070475C06002080B58AB004AFFEF726
:1046900029FE87ED040BFEF737FE87ED020B4FF086
:1046A00000021F4BD7E90401FBF7D6FF02460B4679
:1046B000104619464FF000021A4BFBF717FE024650
:1046C0000B4610461946FCF79FFA03467B604FF0F5
:1046D0000002134BD7E90201FBF7BEFF02460B466F
:1046E000104619464FF000020E4BFBF7FFFD024645
:1046F0000B4610461946FCF787FA03463B603B68B9
:1047000003937B680293D7E90223CDE90023D7E91D
:1047100004230548FFF786FF00BF1837BD4680BD5C
:10472000000069400000E03FE462010880B400AF8F
:104730000A4B1B78002B08D0094B1B7883F0010330
:10474000DBB2002B01D0012300E0002303F00103C2
:10475000DBB21846BD465DF8047B70475D0600205D
:104760005E06002080B400AF034B1B781846BD46A0
:104770005DF8047B704700BF5E06002080B500AF87
:10478000144B01221A70144B4FF000021A6001F012
:1047900093FD0346114A1360114B00221A60114920
:1047A0004FF00002104BC1E9002310494FF0000206
:1047B0000F4BC1E900230F4B0F4A1A600F4B104AF1
:1047C0001A60104B00221A600F4B00221A7000BFB3
:1047D00080BD00BF5E060020600600206406002049
:1047E00068060020200000200040594028000020DA
:1047F0000000F0BF300000200000CA42340000205A
:10480000000080BF6C0600207006002080B400AF5E
:10481000044B1B6807EE903AB0EE670ABD465DF8A0
:10482000047B704760060020B0B590B008AF6F4BB6
:1048300000221A706E48FFF7F5FE6E4BD3E90001B7
:104840004FF000026C4BFCF783F90346002B03D0BA
:10485000684BD3E9002302E04FF00002674BC7E941
:104860000623674BD3E900014FF000024FF000032D
:10487000FCF778F90346002B03D0614BD3E9002302
:1048800002E04FF000025D4BC7E904235D4BD3ED1E
:10489000007A9FED5D7AF4EEC77AF1EE10FA02D855
:1048A000584B1B6800E0594BFB60594BD3ED007A25
:1048B000F5EEC07AF1EE10FA02DB554B1B6800E012
:1048C000524BBB604FF000024FF00003D7E90601E6
:1048D000FCF748F90346002B17D04FF000024D4B70
:1048E000D7E90601FBF7B8FE02460B46104619460B
:1048F0004FF00002484BFBF7F9FC02460B4610460E
:104900001946FCF781F9034600E000237B604FF075
:1049100000024FF00003D7E90401FCF723F9034636
:10492000002B17D04FF000023A4BD7E90401FBF7F8
:1049300093FE02460B46104619464FF00002364BD6
:10494000FBF7D4FC02460B4610461946FCF75CF90F
:10495000034600E000233B60F868FBF725FE0446B1
:104960000D46B868FBF720FE02460B4639680791F2
:1049700079680691CDE90423CDE90245D7E90423FE
:10498000CDE90023D7E906232448FFF74BFE4FF07B
:1049900000024FF00003D7E90601FCF7E3F80346F5
:1049A000002B00D11EE04FF00002134BD7E90401A9
:1049B000FCF7CEF80346002B00D113E0D7E904231F
:1049C000D7E90601FCF7BAF80346002B00D109E04D
:1049D000D7ED022A97ED032A97ED041B97ED060BFE
:1049E000FEF782FA00BF2037BD46B0BD5E0600204C
:1049F0001863010820000020000059400000F0BFAB
:104A000028000020300000200000C842000080BFC5
:104A100034000020000069400000E03F2C630108E2
:104A200080B58AB004AF87ED030A87ED001B534BB6
:104A30001B7883F00103DBB2002B40F09980504BD0
:104A40001B78DBB283F00103DBB2002B40F09080D7
:104A500001F032FC78614B4BD3E90023D7E9000128
:104A6000FCF76CF80346002B08D04649D7E9002331
:104A7000C1E90023444B1B68444A1360444BD3E90B
:104A80000023D7E90001FCF777F80346002B08D094
:104A90003F49D7E90023C1E900233B4B1B683D4A4E
:104AA00013603D4B1B68002B26D03B4B1B687A697B
:104AB000D31A4F2B20D9344BD3ED007AB0EE007AC5
:104AC00077EE877A304BC3ED007A2F4BD3ED007A27
:104AD0009FED327AF4EEC77AF1EE10FA08DB2A4B3A
:104AE0002F4A1A602C4A7B691360FFF79DFE42E053
:104AF000294A7B69136006E0274B1B68002B02D113
:104B0000254A7B691360274B1B78002B09D0264B65
:104B10001B68002B05D0244B1B687A69D31A312BF4
:104B200028D9194B1B681846FBF73EFDD7E900232F
:104B3000CDE90223CDE900011C4A40211C480FF0B9
:104B40002DFA38613B69002B15DD3B693F2B12DCE8
:104B50003B699BB2194616480DF0E0FC0346012B59
:104B600009D0114A7B6913600E4B01221A7002E0D2
:104B700000BF00E000BF1837BD4680BD5E060020C4
:104B80005C0600202000002060060020300000208D
:104B90002800002034000020680600200000C842E1
:104BA0000000C842700600206C060020B0630108B7
:104BB0007406002080B483B000AF78607B68002B5F
:104BC00007DB7B68072B04DC054A7B6852F823303F
:104BD00000E0044B18460C37BD465DF8047B704777
:104BE00058000020C863010880B584B000AF87ED8D
:104BF000000B4FF00002264BD7E90001FBF774FBD6
:104C000002460B46104619464FF00002214BFBF7B7
:104C10004DFE02460B46104619464FF000021E4B51
:104C2000FBF71AFD02460B46C7E902234FF00002CC
:104C30004FF00003D7E90201FBF780FF0346002B8A
:104C400005D04FF000024FF00003C7E902234FF0F8
:104C50000002114BD7E90201FBF78EFF0346002B40
:104C600004D04FF000020C4BC7E902234FF00002C2
:104C70000A4BD7E90201FBF739FB02460B46104607
:104C80001946FBF799FF034618461037BD4680BD0D
:104C90000000044000002440000059400000E03FB4
:104CA00080B596B008AF444B1B78DBB283F00103AC
:104CB000DBB2002B06D1414B1B7883F00103DBB242
:104CC000002B01D0002373E0FEF738FD78633C4BE6
:104CD000D3ED007A9FED3B7A67EE877AFDEEE77AB7
:104CE00017EE903A3B63384BD3ED007A9FED377A5D
:104CF00067EE877AFDEEE77A17EE903AFB62FEF7F1
:104D0000D9F8F0EE407AFDEEE77A17EE903ABB6202
:104D10002F4BD3E900014FF000022E4BFBF79CFC18
:104D200002460B4610461946FBF746FF03467B62D8
:104D3000FEF7D8FA87ED060BFEF7E6FA87ED040BCF
:104D400097ED060BFFF750FFF86097ED040BFFF7A8
:104D50004BFFB860786BFFF72DFF02461E4B1B8898
:104D60001946BB680693FB68059304917B6A03931D
:104D70000292BB6A0193FB6A00933B6B174A502176
:104D800017480FF00BF978607B68002B02DD7B6819
:104D90004F2B01DD00230BE07B689BB219461048C6
:104DA0000DF0BCFB0346012B14BF01230023DBB233
:104DB00018463837BD4680BD5C0600205D060020E1
:104DC0000004002000007A44040400200000C842CF
:104DD000180400200000244010040020CC630108C7
:104DE000B406002080B500AF4022002103480FF038
:104DF0008BF9034B00221A7000BF80BDD80500203C
:104E00001806002080B582B000AF786039603B683A
:104E1000002B15D00C4B01221A703B683F2B01D997
:104E20003F233B603A68796808480FF097FA074AD1
:104E30003B68134400221A70054B01221A7000E0EF
:104E400000BF0837BD4680BD5C0600201C06002060
:104E50001806002080B500AF0E4B1B78DBB283F044
:104E60000103DBB2002B13D10A4B00221A703F2240
:104E700009490A480FF080F9084B002283F83F20C7
:104E800000F052F84022002104480FF03DF900E004
:104E900000BF80BD180600201C060020D805002099
:104EA00080B588B000AFF860B9607A600023FB611C
:104EB0002C21F8680FF030F978617B69002B01D163
:104EC00000232AE07B6900221A707B690133BB61F1
:104ED00015E0FB695A1CFA619B00BA681344BA6971
:104EE0001A602C21B8690FF017F978617B69002BE3
:104EF00011D07B6900221A707B690133BB61FA69AA
:104F00007B689A4208DABB69002B05D0BB691B7825
:104F1000002BDED100E000BFFB6918462037BD46FC
:104F200080BD0000000000002DE9F04FF1B010AF8F
:104F3000002387F87F3107F5C073A3F594731846F3
:104F400020231A4600210FF0DFF80023C7F8443170
:104F500007F118033F22C34918460FF00DF907F572
:104F6000C073A3F5B473002283F83F2007F1580102
:104F700007F1180308221846FFF792FFC7F844010B
:104F80000023C7F8783101F02BB8B74AD7F8783149
:104F900052F833301846FBF745F9C7F84001B24ADA
:104FA000D7F8783152F8331007F11803D7F84021B9
:104FB00018460FF0CFF80346002B1FD107F5C0733A
:104FC000A3F5B472D7F8403113441B78002B13D0EB
:104FD00007F5C073A3F5B472D7F8403113441B78BA
:104FE000202B09D007F5C073A3F5B472D7F8403170
:104FF00013441B782C2B01D1012300E00023C7F8B8
:105000003C31D7F83C31002B00F0E587964AD7F8C1
:105010007831DB0013441B79013B0E2B00F2D38760
:1050200001A252F823F000BF655000086D5000083F
:1050300091510008F95100085352000877540008B4
:1050400095540008035200080D520008855E0008C0
:105050009F5400087755000857560008855B0008E4
:105060001D5D0008FEF7EEFB00F0B1BFFEF766FB2A
:10507000C7F89400FEF736F987ED220B07F180039D
:105080001C46FEF741F984ED000B4FF00002774B10
:10509000D7E92201FBF7E0FA02460B461046194613
:1050A0004FF00002724BFBF721F902460B4607F561
:1050B000C071A1F5827410461946FBF7A5FD0346A1
:1050C000236007F1800319464FF00002674BD1E9D6
:1050D0000001FBF7C1FA02460B46104619464FF095
:1050E0000002634BFBF702F902460B4607F5C0715D
:1050F000A1F5847410461946FBF786FD034623602C
:105100005C4B1B681846FBF74FFA82468B465A4B9E
:105110001B681846FBF748FA04460D46FDF7CAFE21
:1051200010EE103A1846FBF73FFA80468946D7F84A
:105130009400FFF75DFA0646504BD3E9002350492F
:105140000988796007F5C071A1F5847109680F912C
:1051500007F5C071A1F5827109680E9107F1800110
:10516000D1E90001CDE90C01D7E92201CDE90A011D
:1051700079680891CDE906230496CDE90289CDE945
:10518000004552465B463F48FFF74CFA00F01FBF10
:10519000D7F84431002B04DC3B48FFF743FA00F01A
:1051A00016BF07F5C073A3F594731B6837491846FB
:1051B000FBF72EF80346002B06D1FDF72DFE3448F1
:1051C000FFF730FA00F003BF07F5C073A3F594733F
:1051D0001B6830491846FBF71BF80346002B06D125
:1051E000FDF72AFE2C48FFF71DFA00F0F0BE2B4811
:1051F000FFF718FA00F0EBBE2948FFF713FA00F0AA
:10520000E6BE2848FFF70EFA00F0E1BE264B1B6809
:10521000C7F8A430254B1B68C7F8A030244B1B6887
:10522000C7F89C30FEF78AFAC7F89800D7F89800BC
:10523000FFF7DEF903460193D7F89C300093D7F8C7
:10524000A030D7F8A4201B491B48FFF7EBF900F06A
:10525000BEBED7F84431002B32DC1848FFF7E2F924
:1052600000F0B5BED80500209C730108000069401D
:105270000000E03F00040020040400201804002087
:1052800010040020F463010874640108B864010884
:10529000C4640108E8640108F464010818650108A1
:1052A0005065010858650108107AFF1F147AFF1F26
:1052B000187AFF1F6865010870650108A465010878
:1052C0004FF0FF33C7F8743107F5C073A3F594733B
:1052D0001B68C7491846FAF79BFF0346002B03D10A
:1052E0000023C7F87431AEE007F5C073A3F59473DB
:1052F0001B68C0491846FAF78BFF0346002B03D101
:105300000123C7F874319EE007F5C073A3F59473C9
:105310001B68B9491846FAF77BFF0346002B03D1F7
:105320000223C7F874318EE007F5C073A3F59473B8
:105330001B68B2491846FAF76BFF0346002B03D1EE
:105340000323C7F874317EE007F5C073A3F59473A7
:105350001B68AB491846FAF75BFF0346002B03D1E5
:105360000423C7F874316EE007F5C073A3F5947396
:105370001B68A4491846FAF74BFF0346002B03D1DC
:105380000423C7F874315EE007F5C073A3F5947386
:105390001B689D491846FAF73BFF0346002B03D1D3
:1053A0000523C7F874314EE007F5C073A3F5947375
:1053B0001B6896491846FAF72BFF0346002B03D1CA
:1053C0000523C7F874313EE007F5C073A3F5947365
:1053D0001B688F491846FAF71BFF0346002B03D1C1
:1053E0000623C7F874312EE007F5C073A3F5947354
:1053F0001B6888491846FAF70BFF0346002B03D1B8
:105400000623C7F874311EE007F5C073A3F5947343
:105410001B6881491846FAF7FBFE0346002B03D1AF
:105420000723C7F874310EE007F5C073A3F5947332
:105430001B687A491846FAF7EBFE0346002B02D1A7
:105440000723C7F87431D7F87431002B0EDBD7F877
:105450007401FEF781F9D7F87401FFF7C9F8034624
:1054600019466F48FFF7DEF800F0B1BD6D48FFF751
:10547000D9F800F0ACBDFEF7D3F9FEF75FF90346AB
:105480001846FFF7B5F8034619466748FFF7CAF80C
:1054900000F09DBD6548FFF7C5F800F098BDD7F84E
:1054A0004431002B04DC6248FFF7BCF800F08FBDEC
:1054B00007F5C073A3F594731B68C7F8703104E057
:1054C000D7F870310133C7F87031D7F870311B78D5
:1054D000202BF5D05749D7F870010EF02AFE02466E
:1054E000D7F870311344C7F8B430D7F8B4301B780C
:1054F000002B03D0D7F8B43000221A7007F5C07320
:10550000A3F5B67300221A6007F114030A221946A4
:10551000D7F870010EF076FCC7F8B00007F5C0733D
:10552000A3F5B6731B68002B0FD007F5C073A3F566
:10553000B6731B681B78002B07D1D7F8B030002B4F
:1055400003DBD7F8B030642B04DD3B48FFF76AF883
:1055500000F03DBDD7F8B03007EE903AF8EEE77AAC
:10556000B0EE670AFDF778FCD7F8B0103348FFF7C4
:1055700059F800F02CBDD7F84431002B64DD07F555
:10558000C073A3F594731B68C7F86C3104E0D7F8B7
:105590006C310133C7F86C31D7F86C311B78202B94
:1055A000F5D02449D7F86C010EF0C3FD0246D7F8B8
:1055B0006C311344C7F8B830D7F8B8301B78002BDB
:1055C00003D0D7F8B83000221A701D49D7F86C0103
:1055D000FAF71EFE0346002B03D1FFF725F900F072
:1055E000F6BCFFF7CBF81748FFF71CF800F0EFBC4C
:1055F000FC650108046601080C66010814660108D0
:105600001866010820660108346601083C66010836
:105610004C66010854660108606601086866010866
:105620007466010888660108D4660108EC66010802
:10563000386C0108606C0108646C0108806C01081A
:10564000B06C0108B86C0108FFF798F8C448FEF781
:10565000E9FF00F0BCBCD7F84431002B04DCC148A2
:10566000FEF7E0FF00F0B3BC07F5C073A3F5947339
:105670001B68C7F8683104E0D7F868310133C7F810
:105680006831D7F868311B78202BF5D0B649D7F8A8
:1056900068010EF04EFD0246D7F868311344C7F892
:1056A0000831D7F808311B78002B03D0D7F8083120
:1056B00000221A70AD49D7F86801FAF7A9FD034630
:1056C000002B53D1FDF7F6FB87ED320AD7F8C8005F
:1056D000FAF76AFF4FF00002A54BFBF7E7F8024626
:1056E0000B46104619464FF00002A24BFAF7B4FFE2
:1056F00002460B46104619464FF000029E4BFAF741
:10570000F5FD02460B46C7E9302397ED300BFDF758
:10571000A7FC4FF4C87000F0DBFD984B01221A7013
:10572000FEF7FEFBC7F8BC00944B00221A7097ED01
:10573000321A97ED300BFDF7EBFCD7F8C800FAF7FB
:1057400033FF02460B46D7F8BC10002901D18C4923
:1057500000E08C490291CDE90023D7E930238A4843
:10576000FEF760FFFEF790FF00F031BC8749D7F8E5
:105770006801FAF74DFD0346002B52D1FDF79AFB65
:1057800087ED370AD7F8DC00FAF70EFF4FF000027A
:10579000774BFBF78BF802460B46104619464FF045
:1057A0000002744BFAF758FF02460B4610461946A2
:1057B0004FF00002704BFAF799FD02460B46C7E91D
:1057C000342397ED340BFDF74BFC4FF4C87000F019
:1057D0007FFD6A4B01221A70FEF7AAFBC7F8CC00C6
:1057E000664B00221A7097ED371A97ED340BFDF7D0
:1057F00007FDD7F8DC00FAF7D7FE02460B46D7F8CC
:10580000CC10002901D15E4900E05E490291CDE94A
:105810000023D7E934235E48FEF704FFFEF734FF88
:10582000D5E35C49D7F86801FAF7F2FC0346002B90
:1058300021D1DFED592A9FED592A9FED451B9FEDA0
:10584000460BFDF751FB4D4B01221A70FEF778FB1A
:10585000C7F8E000494B00221A70D7F8E030002B5F
:1058600001D1474B00E0474B19464D48FEF7DAFEA1
:10587000FEF70AFFABE307F5C073A3F5B873002288
:105880001A6007F110031946D7F868010EF034FAD0
:1058900087ED400B07F5C073A3F5B8731B68002BA9
:1058A0000CD007F5C073A3F5B8731B68D7F868214F
:1058B0009A4203D0D7F84431012B03DC3948FEF774
:1058C000B1FE84E307F5C073A3F594735B68C7F872
:1058D000643104E0D7F864310133C7F86431D7F894
:1058E00064311B78202BF5D01F49D7F864010EF0E6
:1058F00020FC0246D7F864311344C7F8FC30D7F8CF
:10590000FC301B78002B03D0D7F8FC3000221A7033
:1059100007F110031946D7F864010EF0EDF987ED91
:105920003C0B07F5C073A3F5B8731B68002B08D0B8
:1059300007F5C073A3F5B8731B68D7F864219A42C2
:1059400034D11948FEF76EFE41E300BFAFF300808B
:10595000000000000000294000000000000004409A
:10596000B86C0108206D0108606C0108AC6D01087D
:10597000000059400000244000000440F6030020CD
:10598000B06D0108C46D0108C86D0108F46D01080F
:10599000F86D0108246E01080000C84200000000F4
:1059A0002C6E0108586E0108BC6E01084FF0000310
:1059B000C7F86031A64BC7F85C31D7F84431032BE8
:1059C0007ADD07F5C073A3F594739B68C7F8583167
:1059D00007F5C073A3F59473DB68C7F8543104E08E
:1059E000D7F858310133C7F85831D7F858311B78F8
:1059F000202BF5D004E0D7F854310133C7F85431E7
:105A0000D7F854311B78202BF5D09249D7F858019C
:105A10000EF08FFB0246D7F858311344C7F8EC302C
:105A2000D7F8EC301B78002B03D0D7F8EC300022ED
:105A30001A708849D7F854010EF07BFB0246D7F85C
:105A400054311344C7F8E830D7F8E8301B78002BFE
:105A500003D0D7F8E83000221A7007F11003194676
:105A6000D7F858010EF048F953EC102B10461946A0
:105A7000FBF7EAF80346C7F8603107F5C073A3F5F2
:105A8000B8731B68002B17D007F5C073A3F5B87364
:105A90001B681B78002B0FD107F110031946D7F8AC
:105AA00054010EF029F953EC102B10461946FBF760
:105AB000CBF80346C7F85C31D7ED572A97ED582A43
:105AC00097ED3C1B97ED400BFDF70EFA4FF00002EF
:105AD000614BD7E94001FBF73BF80346002B35D07B
:105AE0004FF000025D4BD7E93C01FBF73BF8034662
:105AF000002B2BD05A4B01221A70FEF721FAC7F85F
:105B0000E400574B00221A70D7F86001FAF74CFDF9
:105B100004460D46D7F85C01FAF746FD02460B46EF
:105B2000D7F8E410002901D14E4900E04E49069112
:105B3000CDE90423CDE90245D7E93C23CDE9002393
:105B4000D7E940234948FEF76DFD18E0D7F860011A
:105B5000FAF72AFD04460D46D7F85C01FAF724FD52
:105B600002460B46CDE90423CDE90245D7E93C23A3
:105B7000CDE90023D7E940233D48FEF753FDFEF76A
:105B800083FD24E2D7F84431002B03DC3948FEF7CB
:105B900049FD1CE207F5C073A3F594731B68C7F8B1
:105BA000503104E0D7F850310133C7F85031D7F8FD
:105BB00050311B78202BF5D02649D7F850010EF034
:105BC000B8FA0246D7F850311344C7F82031D7F855
:105BD00020311B78002B03D0D7F8203100221A7017
:105BE00007F5C073A3F5BA7300221A6007F10C031E
:105BF0001946D7F850010EF07FF887ED460B07F5F0
:105C0000C073A3F5BA731B68002B1DD007F5C073D2
:105C1000A3F5BA731B68D7F850219A4214D04FF0FD
:105C200000024FF00003D7E94601FAF787FF034669
:105C3000002B09D14FF000020F4BD7E94601FAF7CC
:105C40009BFF0346002B1BD00C48FEF7EBFCBEE18C
:105C50000000C842606C01080000044000002940B8
:105C6000F6030020E46E0108C46D0108006F01080E
:105C7000346F0108686F010800005940AC6F0108DB
:105C80004FF00002B64BD7E94601FAF70FFE024685
:105C90000B46104619464FF00002B24BFAF7DCFCF7
:105CA00002460B46104619464FF00002AE4BFAF77B
:105CB0001DFB02460B46C7E9442397ED440BFDF755
:105CC000CFF94FF4C87000F003FBA84B01221A7003
:105CD000FEF726F9C7F80C01A44B00221A70D7E989
:105CE0004601FAF7B1FF034601EE103A97ED440B77
:105CF000FDF70EFAD7F80C31002B01D19C4B00E0D8
:105D00009C4B0293D7E94423CDE90023D7E94623EE
:105D10009948FEF787FCFEF7B7FC58E1D7F8443105
:105D2000002B03DC9548FEF77DFC50E107F5C073BE
:105D3000A3F594731B68C7F84C3104E0D7F84C31D5
:105D40000133C7F84C31D7F84C311B78202BF5D0F4
:105D50008B49D7F84C010EF0ECF90246D7F84C31DC
:105D60001344C7F83831D7F838311B78002B03D0EB
:105D7000D7F8383100221A7007F5C073A3F5BC7349
:105D800000221A6007F108031946D7F84C010DF0FC
:105D9000B3FF87ED4C0B07F5C073A3F5BC731B680D
:105DA000002B1DD007F5C073A3F5BC731B68D7F893
:105DB0004C219A4214D04FF000024FF00003D7E973
:105DC0004C01FAF7BBFE0346002B09D14FF000024D
:105DD000634BD7E94C01FAF7CFFE0346002B03D003
:105DE0006848FEF71FFCF2E04FF000025C4BD7E979
:105DF0004C01FAF75BFD02460B46104619464FF080
:105E00000002584BFAF728FC02460B46104619468A
:105E10004FF00002544BFAF769FA02460B46C7E905
:105E20004A2397ED4A0BFDF71BF94FF4C87000F0B9
:105E30004FFA4E4B01221A70FEF77AF8C7F8240188
:105E40004A4B00221A70D7E94C01FAF7FDFE0346CF
:105E500001EE103A97ED4A0BFDF7D2F9D7F824314D
:105E6000002B01D1424B00E0424B0293D7E94A2379
:105E7000CDE90023D7E94C234348FEF7D3FBFEF7D7
:105E800003FCA4E00023C7F84831D7F84431002BC5
:105E900007DD07F5C073A3F594731B68C7F8483195
:105EA0001CE007F11803202118460EF035F9C7F859
:105EB000AC00D7F8AC30002B10D0D7F8AC300133A1
:105EC0001B78002B0AD0D7F8AC300133C7F8483123
:105ED00004E0D7F848310133C7F84831D7F84831E2
:105EE000002B04D0D7F848311B78202BF1D0D7F8FD
:105EF0004831002B04D0D7F848311B78002B03D150
:105F00002248FEF78FFB62E01D49D7F848010EF0EA
:105F100010F90246D7F848311344C7F8A830D7F82B
:105F2000A8301B78002B03D0D7F8A83000221A70B5
:105F30001749D7F84801FAF76BF90346002B2FD120
:105F4000144B1B78002B03D01348FEF76BFB3EE08D
:105F5000104B01221A702F2110480CF0DFFA36E0A6
:105F6000000059400000244000000440F6030020D7
:105F7000B06D0108C46D0108D86F0108FC6F0108FD
:105F8000606C010844700108707001089470010889
:105F9000DC7001085D060020E0700108147401083F
:105FA0001D49D7F84801FAF733F90346002B06D10B
:105FB0001A4B00221A701A48FEF734FB07E0194802
:105FC000FEF730FB03E01848FEF72CFB00BF01236F
:105FD00087F87F3109E0D7F878310133C7F8783195
:105FE000D7F878310E2B7EF6D0AF97F87F3183F05B
:105FF0000103DBB2002B08D007F1180319460B4848
:10600000FEF710FB0A48FEF70DFB00BF07F5C2774D
:10601000BD46BDE8F08F00BFFC7001085D060020A2
:1060200000710108147101083C71010858710108E0
:10603000707101081348016800220260124A9142FF
:1060400008D0DFF848D0FEF7C1FA11481149124ACA
:10605000002307E0114BD3F800D0D3F804F0D45854
:10606000C4500433C4188C42F9D30D4A0D4C00239C
:1060700001E013600432A242FBD30EF04BF9FBF7B0
:10608000BDFA7047F0FF0120EFBEADDEF0FF01204A
:10609000000000204C030020107801080000FF1FC2
:1060A0005003002034310120FEE780B584B000AFFA
:1060B00078607B68002B05D172B600BFFDF7A0FDAC
:1060C00000BFFDE70023FB6007E07B68FA68002162
:1060D00043F82210FB680133FB60FB68012BF4D905
:1060E0007B6800221A7200BF1037BD4680BD80B5A4
:1060F00084B000AF78607B68002B05D172B600BF1A
:10610000FDF77EFD00BFFDE77B681B7A012B05D9FB
:1061100072B600BFFDF774FD00BFFDE77B681B7A18
:106120005A1CD1B27A6811721946EFF311824FF0FE
:10613000500383F31188BFF36F8FBFF34F8FFA6063
:10614000BB60FA687B6843F8212000BF1037BD466A
:1061500080BD80B584B000AF78607B68002B05D12E
:1061600072B600BFFDF74CFD00BFFDE77B681B7AF0
:10617000013BDAB27B681A727B681B7A012B05D966
:1061800072B600BFFDF73CFD00BFFDE77B681B7AE0
:106190001A467B6853F82230FB60FB6883F3118852
:1061A00000BF00BF1037BD4680BD80B582B000AFD4
:1061B00078607B68002B05D10EF0A6F80346162206
:1061C0001A6016E00C200CF0DDFE03461A467B68D0
:1061D0001A607B681B68002B05D07B681B6818461B
:1061E000FFF763FF05E072B600BFFDF709FD00BFD2
:1061F000FDE70837BD4680BD80B582B000AF78604E
:106200007B68002B05D172B600BFFDF7F9FC00BF1B
:10621000FDE77B681846FFF76AFF00BF0837BD46F9
:1062200080BD80B582B000AF78607B68002B05D15F
:1062300072B600BFFDF7E4FC00BFFDE77B681846BF
:10624000FFF787FF00BF0837BD4680BD80B500AFB0
:106250000E4B1B680D4A43F4007313600B4B1B6815
:106260000A4A43F480631360084B1B68074A43F4EF
:1062700080731360032000F030FD0F20FEF72AF832
:10628000FDF7C8FE0023184680BD00BF003C024059
:1062900080B400AF064B1B781A46064B1B681344AC
:1062A000044A136000BFBD465DF8047B704700BF21
:1062B0007C0000201C07002080B400AF034B1B684B
:1062C0001846BD465DF8047B704700BF1C070020E0
:1062D00080B584B000AF7860FFF7EEFFB8607B68F0
:1062E000FB60FB68B3F1FF3F05D00A4B1B781A46F1
:1062F000FB681344FB6000BFFFF7DEFF0246BB688C
:10630000D31AFA689A42F7D800BF00BF1037BD46CB
:1063100080BD00BF7C00002080B584B000AF7860F5
:106320000023FB737B68002B01D1012333E07B68E2
:106330001B6C002B09D17868FDF798FE7B68002262
:106340005A647B68002283F83C207B681B6C03F056
:106350001003002B18D17B681B6C23F4885323F0A7
:10636000020343F002027B681A64786800F0E8FADE
:106370007B6800225A647B681B6C23F0030343F0A4
:1063800001027B681A6401E00123FB737B68002231
:1063900083F83C20FB7B18461037BD4680BD0000CB
:1063A00080B485B000AF78600023BB607B6893F851
:1063B0003C30012B01D10223B2E07B68012283F83B
:1063C0003C207B681B689B6803F00103012B18D0FD
:1063D0007B681B689A687B681B6842F001029A60C0
:1063E000524B1B68524AA2FB03239A0C13465B00D4
:1063F0001344BB6002E0BB68013BBB60BB68002B81
:10640000F9D17B681B689B6803F00103012B7AD1EB
:106410007B681B6C23F4E06323F0010343F4807278
:106420007B681A647B681B685B6803F48063002BDD
:1064300007D07B681B6C23F4405343F480527B6885
:106440001A647B681B6C03F48053B3F5805F06D13C
:106450007B685B6C23F006027B685A6402E07B6811
:1064600000225A647B68002283F83C20314BFB6099
:106470007B681B686FF022021A60FB685B6803F0A0
:106480001F03002B2AD17B681B682B4A934215D02F
:106490007B681B68294A934205D1264B5B6803F051
:1064A0001F03002B0AD07B681B68254A934236D114
:1064B000204B5B6803F01003002B30D17B681B6816
:1064C0009B6803F04053002B29D17B681B689A68B6
:1064D0007B681B6842F080429A6020E07B681B6802
:1064E000154A93421BD17B681B689B6803F040539D
:1064F000002B14D17B681B689A687B681B6842F08C
:1065000080429A600BE07B681B6C43F010027B6852
:106510001A647B685B6C43F001027B685A64002359
:1065200018461437BD465DF8047B70471C000020F8
:1065300083DE1B4300230140002001400021014075
:106540000022014080B483B000AF78607B6893F88C
:106550003C30012B01D1022321E07B68012283F82A
:106560003C207B681B689A687B681B6822F00102EC
:106570009A607B681B689B6803F00103002B09D1BC
:106580007B681B6C23F4885323F0010343F0010262
:106590007B681A647B68002283F83C20002318463D
:1065A0000C37BD465DF8047B704780B584B000AF02
:1065B000786039600023FB607B681B689B6803F48C
:1065C0008063B3F5806F13D17B681B689B6803F40D
:1065D0008073B3F5807F0BD17B681B6C43F0200286
:1065E0007B681A647B68002283F83C20012363E007
:1065F000FFF762FEF86021E03B68B3F1FF3F1DD07A
:106600003B68002B07D0FFF757FE0246FB68D31A02
:106610003A689A4212D27B681B681B6803F0020337
:10662000022B0BD07B681B6C43F004027B681A645E
:106630007B68002283F83C2003233DE07B681B68D5
:106640001B6803F00203022BD6D17B681B686FF036
:1066500012021A607B681B6C43F400727B681A6438
:106660007B681B689B6803F04053002B23D17B6839
:106670001B7E002B1FD17B681B68DB6A03F4700351
:10668000002B06D07B681B689B6803F48063002B9B
:1066900011D17B681B6C23F480727B681A647B6861
:1066A0001B6C03F48053002B05D17B681B6C43F0FB
:1066B00001027B681A64002318461037BD4680BD6E
:1066C00080B483B000AF78607B681B68DB6C1846D1
:1066D0000C37BD465DF8047B7047000080B485B080
:1066E00000AF786039600023BB607B6893F83C3072
:1066F000012B01D1022313E17B68012283F83C20A6
:106700003B681B68092B25D97B681B68D9683B68E7
:106710001B689BB21A4613465B0013441E3B0722BC
:1067200002FA03F3DA437B681B680A40DA607B688D
:106730001B68D9683B689A683B681B689BB218461F
:1067400003465B0003441E3B9A407B681B680A4378
:10675000DA6022E07B681B6819693B681B689BB2A2
:106760001A4613465B001344072202FA03F3DA4386
:106770007B681B680A401A617B681B6819693B6863
:106780009A683B681B689BB2184603465B0003444B
:106790009A407B681B680A431A613B685B68062B5A
:1067A00024D87B681B68596B3B685A6813469B006A
:1067B0001344053B1F2202FA03F3DA437B681B688C
:1067C0000A405A637B681B68596B3B681B689BB225
:1067D00018463B685A6813469B001344053B00FA71
:1067E00003F27B681B680A435A634CE03B685B68B2
:1067F0000C2B24D87B681B68196B3B685A681346BE
:106800009B001344233B1F2202FA03F3DA437B6805
:106810001B680A401A637B681B68196B3B681B681E
:106820009BB218463B685A6813469B001344233BAF
:1068300000FA03F27B681B680A431A6323E07B6853
:106840001B68D96A3B685A6813469B001344413B56
:106850001F2202FA03F3DA437B681B680A40DA62FC
:106860007B681B68D96A3B681B689BB218463B680B
:106870005A6813469B001344413B00FA03F27B68BD
:106880001B680A43DA62294BFB607B681B68284A55
:1068900093420FD13B681B68122B0BD1FB685B68DE
:1068A00023F40002FB685A60FB685B6843F48002D3
:1068B000FB685A607B681B681D4A93422BD13B687A
:1068C0001B681C4A934203D03B681B68112B22D1E2
:1068D000FB685B6823F48002FB685A60FB685B68B6
:1068E00043F40002FB685A603B681B68114A9342FC
:1068F00011D1114B1B68114AA2FB03239A0C1346BA
:106900009B0013445B00BB6002E0BB68013BBB60C3
:10691000BB68002BF9D17B68002283F83C20002360
:1069200018461437BD465DF8047B704700230140CC
:1069300000200140120000101C00002083DE1B43D9
:1069400080B485B000AF7860794BFB60FB685B6812
:1069500023F44032FB685A60FB685A687B685B68C6
:106960001A43FB685A607B681B685A687B681B681F
:1069700022F480725A607B681B6859687B681B69C7
:106980001A027B681B680A435A607B681B685A6856
:106990007B681B6822F040725A607B681B685968EC
:1069A0007B689A687B681B680A435A607B681B682F
:1069B0009A687B681B6822F400629A607B681B6897
:1069C00099687B68DA687B681B680A439A607B6811
:1069D0009B6A584A934222D07B681B689A687B68FE
:1069E0001B6822F070629A607B681B6899687B68FC
:1069F0009A6A7B681B680A439A607B681B689A687E
:106A00007B681B6822F040529A607B681B6899681B
:106A10007B68DA6A7B681B680A439A600FE07B68D0
:106A20001B689A687B681B6822F070629A607B68BA
:106A30001B689A687B681B6822F040529A607B68EA
:106A40001B689A687B681B6822F002029A607B6868
:106A50001B6899687B681B7E5A007B681B680A4329
:106A60009A607B6893F82030002B1BD07B681B68F2
:106A70005A687B681B6842F400625A607B681B6836
:106A80005A687B681B6822F460425A607B681B6806
:106A900059687B685B6A013B5A037B681B680A4341
:106AA0005A6007E07B681B685A687B681B6822F4A1
:106AB00000625A607B681B68DA6A7B681B6822F494
:106AC0007002DA627B681B68D96A7B68DB69013B0C
:106AD0001A057B681B680A43DA627B681B689A6840
:106AE0007B681B6822F400729A607B681B68996857
:106AF0007B6893F830305A027B681B680A439A60BF
:106B00007B681B689A687B681B6822F480629A60C5
:106B10007B681B6899687B685B699A027B681B6865
:106B20000A439A6000BF1437BD465DF8047B704786
:106B3000002301400100000F80B485B000AF7860F1
:106B40007B6803F00703FB600C4BDB68BB60BA6833
:106B50004FF6FF031340BB60FB681A02BB68134388
:106B600043F0BF6343F40033BB60044ABB68D360A7
:106B700000BF1437BD465DF8047B704700ED00E0B0
:106B800080B400AF044BDB681B0A03F00703184610
:106B9000BD465DF8047B704700ED00E080B483B033
:106BA00000AF0346FB7197F90730002B0BDBFB7935
:106BB00003F01F02074997F907305B09012000FA2B
:106BC00002F241F8232000BF0C37BD465DF8047B7C
:106BD000704700BF00E100E080B483B000AF03461F
:106BE000FB7197F90730002B12DBFB7903F01F02D2
:106BF0000A4997F907305B09012000FA02F22033B5
:106C000041F82320BFF34F8F00BFBFF36F8F00BF4A
:106C100000BF0C37BD465DF8047B704700E100E023
:106C200080B483B000AF03463960FB7197F9073039
:106C3000002B0ADB3B68DAB20C4997F907301201E6
:106C4000D2B20B4483F800230AE03B68DAB2084969
:106C5000FB7903F00F03043B1201D2B20B441A7606
:106C600000BF0C37BD465DF8047B704700E100E0D3
:106C700000ED00E080B489B000AFF860B9607A60E0
:106C8000FB6803F00703FB61FB69C3F10703042BF7
:106C900028BF0423BB61FB690433062B02D9FB69BF
:106CA000033B00E000237B614FF0FF32BB6902FA37
:106CB00003F3DA43BB681A407B699A404FF0FF3117
:106CC0007B6901FA03F3D9437B680B4013431846F1
:106CD0002437BD465DF8047B704780B582B000AFB5
:106CE00078607868FFF728FF00BF0837BD4680BD91
:106CF00080B586B000AF0346B9607A60FB730023AD
:106D00007B61FFF73DFF78617A68B9687869FFF7C2
:106D1000B1FF024697F90F3011461846FFF780FF82
:106D200000BF1837BD4680BD80B582B000AF0346B6
:106D3000FB7197F907301846FFF730FF00BF08379F
:106D4000BD4680BD80B582B000AF0346FB7197F9A8
:106D500007301846FFF740FF00BF0837BD4680BD2B
:106D600080B489B000AF7860396000237B61002374
:106D70003B610023BB610023FB6165E10122FB69EC
:106D800002FA03F37B613B681B687A6913403B613D
:106D90003A697B699A4240F054813B685B6803F032
:106DA0000303012B05D03B685B6803F00303022B50
:106DB00030D17B689B68BB61FB695B00032202FAF0
:106DC00003F3DB43BA691340BB613B68DA68FB69D4
:106DD0005B0002FA03F3BA691343BB617B68BA69CB
:106DE0009A607B685B68BB610122FB6902FA03F36E
:106DF000DB43BA691340BB613B685B681B0903F066
:106E00000102FB6902FA03F3BA691343BB617B68B1
:106E1000BA695A603B685B6803F00303032B17D021
:106E20007B68DB68BB61FB695B00032202FA03F34A
:106E3000DB43BA691340BB613B689A68FB695B003E
:106E400002FA03F3BA691343BB617B68BA69DA607B
:106E50003B685B6803F00303022B23D1FB69DA086C
:106E60007B68083253F82230BB61FB6903F00703EB
:106E70009B000F2202FA03F3DB43BA691340BB61A4
:106E80003B681A69FB6903F007039B0002FA03F3EE
:106E9000BA691343BB61FB69DA087B680832B969D8
:106EA00043F822107B681B68BB61FB695B0003220F
:106EB00002FA03F3DB43BA691340BB613B685B68CA
:106EC00003F00302FB695B0002FA03F3BA691343A0
:106ED000BB617B68BA691A603B685B6803F4403346
:106EE000002B00F0AE800023FB605D4B5B6C5C4AC6
:106EF00043F4804353645A4B5B6C03F48043FB6060
:106F0000FB68584AFB699B08023352F82330BB6187
:106F1000FB6903F003039B000F2202FA03F3DB4338
:106F2000BA691340BB617B684F4A934225D07B68A6
:106F30004E4A93421FD07B684D4A934219D07B68DA
:106F40004C4A934213D07B684B4A93420DD07B68E6
:106F50004A4A934207D07B68494A934201D10623AB
:106F60000CE007230AE0052308E0042306E00323DE
:106F700004E0022302E0012300E00023FA6902F0AA
:106F8000030292009340BA691343BB613549FB6920
:106F90009B080233BA6941F823203A4B9B68BB61D6
:106FA0003B69DB43BA691340BB613B685B6803F430
:106FB0008013002B03D0BA693B691343BB61314A8C
:106FC000BB6993602F4BDB68BB613B69DB43BA69EC
:106FD0001340BB613B685B6803F40013002B03D0D4
:106FE000BA693B691343BB61264ABB69D360254B31
:106FF0005B68BB613B69DB43BA691340BB613B68BB
:107000005B6803F40033002B03D0BA693B69134378
:10701000BB611C4ABB6953601A4B1B68BB613B696F
:10702000DB43BA691340BB613B685B6803F48033A0
:10703000002B03D0BA693B691343BB61114ABB699A
:107040001360FB690133FB61FB690F2B7FF696AE82
:1070500000BF00BF2437BD465DF8047B704700BF0A
:1070600000380240003801400000024000040240A5
:1070700000080240000C02400010024000140240D0
:1070800000180240003C014080B487B000AF786037
:10709000396000233B610023FB600023BB600023B9
:1070A0007B61C7E001227B6902FA03F33B613A6826
:1070B0003B691340FB60FA683B699A4240F0B78035
:1070C000624A7B699B08023352F82330BB607B69BC
:1070D00003F003039B000F2202FA03F3BA68134084
:1070E000BB607B685A4A934225D07B68594A9342D9
:1070F0001FD07B68584A934219D07B68574A934205
:1071000013D07B68564A93420DD07B68554A934210
:1071100007D07B68544A934201D106230CE0072331
:107120000AE0052308E0042306E0032304E0022329
:1071300002E0012300E000237A6902F003029200DA
:107140009340BA689A4232D1484B1A68FB68DB43D5
:10715000464913400B60454B5A68FB68DB43434983
:1071600013404B60414BDA68FB68DB433F491340F7
:10717000CB603E4B9A68FB68DB433C4913408B6015
:107180007B6903F003039B000F2202FA03F3BB6049
:107190002E4A7B699B08023352F82310BB68DA43FE
:1071A0002A487B699B080A40023340F823207B6809
:1071B0001A687B695B00032101FA03F3DB431A4081
:1071C0007B681A607B69DA087B68083253F8221002
:1071D0007B6903F007039B000F2202FA03F3DB43F2
:1071E0007A69D20819407B68083243F822107B681C
:1071F000DA687B695B00032101FA03F3DB431A4081
:107200007B68DA607B685A6801217B6901FA03F3C5
:10721000DB431A407B685A607B689A687B695B0035
:10722000032101FA03F3DB431A407B689A607B6910
:1072300001337B617B690F2B7FF634AF00BF00BF4A
:107240001C37BD465DF8047B704700BF0038014025
:10725000000002400004024000080240000C02400E
:10726000001002400014024000180240003C01409F
:1072700080B485B000AF78600B467B807B681A696C
:107280007B881340002B02D00123FB7301E0002315
:10729000FB73FB7B18461437BD465DF8047B7047D3
:1072A00080B483B000AF78600B467B8013467B7060
:1072B0007B78002B03D07A887B689A6103E07B8817
:1072C0001A047B689A6100BF0C37BD465DF8047BE9
:1072D000704780B586B002AF78607B68002B01D123
:1072E000012308E17B681B68BB607B6893F89534D9
:1072F000DBB2002B06D17B68002283F894247868E7
:107300000BF066FA7B68032283F89524BB68B3F11F
:10731000A04F02D17B6800229A717B681B681846D7
:1073200004F07FFF7B6818687B681A7C8DF800206A
:1073300004330ECB04F05EFE0346002B05D07B68C1
:10734000022283F895240123D5E07B681B68002185
:10735000184604F077FF0346002B05D07B68022215
:1073600083F895240123C6E00023FB734AE0FA7BEF
:1073700079681346DB0013449B000B44153301224C
:107380001A70FA7B79681346DB0013449B000B44A8
:107390001433FA7B1A70FA7BFB7B98B27968134638
:1073A000DB0013449B000B442E3302461A80FA7B09
:1073B00079681346DB0013449B000B44183300220A
:1073C0001A70FA7B79681346DB0013449B000B4468
:1073D0001C3300221A60FA7B79681346DB001344E1
:1073E0009B000B44203300221A60FA7B7968134615
:1073F000DB0013449B000B44243300221A60FB7B08
:107400000133FB737B681B79FA7B9A42AFD300236D
:10741000FB7344E0FA7B79681346DB0013449B005E
:107420000B4403F2552300221A70FA7B7968134645
:10743000DB0013449B000B4403F51573FA7B1A70B1
:10744000FA7B79681346DB0013449B000B4403F579
:10745000167300221A70FA7B79681346DB00134416
:107460009B000B4403F5177300221A60FA7B7968BE
:107470001346DB0013449B000B4403F518730022F2
:107480001A60FA7B79681346DB0013449B000B44B7
:1074900003F5197300221A60FB7B0133FB737B68D1
:1074A0001B79FA7B9A42B5D37B6818687B681A7C93
:1074B0008DF8002004330ECB04F010FF0346002BA0
:1074C00005D07B68022283F89524012313E07B68B2
:1074D00000225A747B68012283F895247B681B7B09
:1074E000012B02D1786801F0FDF97B681B68184612
:1074F00005F09CFF002318461037BD4680BD80B5BF
:1075000082B000AF78607B68002B01D1012315E0C9
:107510007B68032283F895247B681B68184605F076
:10752000EFFE0346002B01D0012307E078680BF043
:10753000C5F97B68002283F8952400231846083794
:10754000BD4680BD80B584B000AF78607B681B68A5
:10755000FB607B6893F89434012B01D1022322E075
:107560007B68012283F89424FB68DB6803F0400306
:10757000002B09D07B685B7B012B05D1FB689B6BE3
:1075800043F48032FB689A637B681B68184604F0FA
:1075900037FE7B681B68184605F027FF7B680022D2
:1075A00083F89424002318461037BD4680BD80B56B
:1075B00084B000AF78607B681B68FB607B6893F8E1
:1075C0009434012B01D1022328E07B68012283F847
:1075D00094247B681B68184604F023FE7B681B68B4
:1075E000184605F023FF7B681B681021184604F03D
:1075F000D3FFFB68DB6803F04003002B09D07B68F6
:107600005B7B012B05D1FB689B6B23F48032FB680D
:107610009A637B68002283F894240023184610376D
:10762000BD4680BD90B58DB000AF78607B681B68AB
:107630003B623B6AFB617B681B68184605F0AAFF4A
:107640000346002B40F0B9847B681B68184605F0A0
:107650000EFF0346002B00F0AF84FB6903F50063C7
:107660009B681B0AC3F30D027B68C3F8D4247B68B4
:107670001B68184605F0FBFE034603F00203022BCD
:1076800007D17B681B685A697B681B6802F002029D
:107690005A617B681B68184605F0E9FE034603F053
:1076A0001003102B61D17B681B689A697B681B688B
:1076B00022F010029A613B6A1B6ABB61BB6903F04E
:1076C0000F021346DB0013449B0003F514737A6822
:1076D000134404337B61BB6903F4F013B3F5802FCB
:1076E00024D1BA6947F6F0731340002B35D07B697B
:1076F000D968BB691B099BB2C3F30A039BB21A4644
:10770000386A05F0D1FC7B69DA68BB691B09C3F3F1
:107710000A031A447B69DA607B695A69BB691B09F1
:10772000C3F30A031A447B695A6116E0BB6903F488
:10773000F013B3F5402F10D17B6803F29C4308226D
:107740001946386A05F0B0FC7B695A69BB691B09A8
:10775000C3F30A031A447B695A617B681B689A6900
:107760007B681B6842F010029A617B681B681846B0
:1077700005F07DFE034603F40023B3F5002F40F02F
:10778000A78000237B627B681B68184605F082FE99
:10779000B86299E0BB6A03F00103002B00F08E8011
:1077A0007B681B687A6AD2B21146184605F0A6FEBD
:1077B00038613B6903F00103002B0CD07B6A5A014E
:1077C000FB69134403F530631A4601239360796A19
:1077D000786800F001FF3B6903F00803002B0CD030
:1077E0007B6A5A01FB69134403F530631A46082388
:1077F0009360796A786800F0D7FF3B6903F0100363
:10780000002B08D07B6A5A01FB69134403F53063EF
:107810001A46102393603B6903F00203002B30D01B
:107820003B6A5B6903F08003802B09D1FB6903F598
:1078300000635B68FA6902F5006243F48063536099
:107840007A6A1346DB0013449B0003F514737A68CD
:10785000134404337B617B69DB78012B08D17B699E
:107860000022DA707B6ADBB2194678680BF0F8F810
:107870007B6A5A01FB69134403F530631A460223FD
:1078800093603B6903F02003002B08D07B6A5A0108
:10789000FB69134403F530631A46202393603B6968
:1078A00003F40053002B09D07B6A5A01FB6913448F
:1078B00003F530631A464FF4005393607B6A01333B
:1078C0007B62BB6A5B08BB62BB6A002B7FF462AF62
:1078D0007B681B68184605F0CAFD034603F4802345
:1078E000B3F5802F40F0DB807B681B68184605F0FD
:1078F000EBFDB86200237B62CDE0BB6A03F00103BD
:10790000002B00F0C2807B681B687A6AD2B21146F5
:10791000184605F011FE38613B6903F00103002BA6
:1079200057D07B6A03F00F03012202FA03F3FB60D6
:10793000FB6903F500635A6BFB68DB43F96901F5EA
:10794000006113404B637B6A5A01FB69134403F5E2
:1079500010631A46012393607B689B79012B32D117
:1079600079687A6A1346DB0013449B000B4420338A
:10797000196878687A6A1346DB0013449B00034455
:107980001C331B68194478687A6A1346DB00134479
:107990009B000344203319607B6A002B13D1796864
:1079A0007A6A1346DB0013449B000B4424331B68A4
:1079B000002B08D17B6818687B6803F29C431A4649
:1079C000012105F019FE7B6ADBB2194678680AF0DE
:1079D000C2FF3B6903F00803002B08D07B6A5A0101
:1079E000FB69134403F510631A46082393603B694F
:1079F00003F01003002B08D07B6A5A01FB69134483
:107A000003F510631A46102393603B6903F04003AB
:107A1000002B08D07B6A5A01FB69134403F51063FD
:107A20001A46402393603B6903F00203002B23D0E6
:107A3000796A386A04F0B0FD7A6A1346DB001344B1
:107A40009B0010337A68134404337B617B69DB78D5
:107A5000012B08D17B690022DA707B6ADBB2194600
:107A600078680BF00FF87B6A5A01FB69134403F541
:107A700010631A46022393603B6903F08003002BD6
:107A800003D0796A786800F01AFD7B6A01337B6263
:107A9000BB6A5B08BB62BB6A002B7FF42EAF7B68BE
:107AA0001B68184605F0E3FC034603F00043B3F1FE
:107AB000004F22D1FB6903F500635B68FA6902F5A8
:107AC000006223F0010353607B6893F8CC34012BF0
:107AD00008D17B68002283F8CC24002178680BF061
:107AE000BFF902E078680AF0ADFF7B681B685A694D
:107AF0007B681B6802F000425A617B681B6818466D
:107B000005F0B5FC034603F40063B3F5006F12D132
:107B1000FB6903F500639B6803F00103012B02D1AD
:107B200078680AF069FF7B681B685A697B681B6884
:107B300002F400625A617B681B68184605F097FCE6
:107B4000034603F00063B3F1006F21D17B681B682B
:107B50005A697B681B6802F000625A617B6893F87F
:107B6000CC34002B11D17B68012283F8CC247B68B4
:107B70001B685B6D9B0803F00F027B68C3F8D02481
:107B8000012178680BF06CF902E078680AF034FFA4
:107B90007B681B68184605F06AFC034603F48053B3
:107BA000B3F5805F40F0B780FB6903F500635B6865
:107BB000FA6902F5006223F0010353607B681B68D9
:107BC0001021184604F0E8FC0023FB6246E0FB6A43
:107BD0005A01FB69134403F510631A464FF67F33CD
:107BE0009360FB6A5A01FB69134403F510631B6839
:107BF000FA6A5101FA690A4402F5106223F400138B
:107C00001360FB6A5A01FB69134403F530631A469B
:107C10004FF67F339360FB6A5A01FB69134403F507
:107C200030631B68FA6A5101FA690A4402F530624E
:107C300023F400131360FB6A5A01FB69134403F534
:107C400030631B68FA6A5101FA690A4402F530622E
:107C500043F000631360FB6A0133FB627B681B79AE
:107C60001A46FB6A9342B2D3FB6903F50063DB69F2
:107C7000FA6902F5006243F00113D3617B68DB7B94
:107C8000002B16D0FB6903F50063D3F88430FA6942
:107C900002F5006243F00B03C2F88430FB6903F580
:107CA00000635B6CFA6902F5006243F00B035364F6
:107CB00015E0FB6903F500635B69FA6902F5006290
:107CC00043F4005343F02B035361FB6903F5006356
:107CD0001B69FA6902F5006243F00B031361FB694B
:107CE00003F500631B68FA6902F5006223F4FE6382
:107CF00013607B6818687B6899797B6803F29C4302
:107D00001A4605F079FC7B681B685A697B681B681A
:107D100002F480525A617B681B68184605F0A7FB85
:107D2000034603F40053B3F5005F23D17B681B685F
:107D3000184605F03DFC7B681B68184604F0A5FC5E
:107D400003461A467B68DA717B681C6800F0E8FE1F
:107D500001467B68DB791A46204604F0AFF9786863
:107D60000AF021FE7B681B685A697B681B6802F475
:107D700000525A617B681B68184605F078FB034681
:107D800003F00803082B0AD178680AF0FEFD7B682F
:107D90001B685A697B681B6802F008025A617B689D
:107DA0001B68184605F063FB034603F08003802B35
:107DB00023D13B6A9B6923F080023B6A9A610123CD
:107DC0007B6214E079687A6A1346DB0013449B00F7
:107DD0000B4403F257231B78012B05D17B6ADBB2DE
:107DE0001946786800F03AFB7B6A01337B627B6856
:107DF0001B791A467B6A9342E4D37B681B6818465A
:107E000005F035FB034603F48013B3F5801F3CD126
:107E100001237B622BE07B6A5A01FB69134403F563
:107E200010631B68BB6179687A6A1346DB001344F0
:107E30009B000B4418331B78012B15D1BB69002B19
:107E400012DA79687A6A1346DB0013449B000B440C
:107E5000173301221A707B6ADBB263F07F03DBB257
:107E60001946786800F0FAFA7B6A01337B627B6816
:107E70001B791A467B6A9342CDD37B681B685A698B
:107E80007B681B6802F480125A617B681B68184685
:107E900005F0EDFA034603F40013B3F5001F56D1C5
:107EA00001237B6245E07B6A5A01FB69134403F5B9
:107EB00030631B68BB6179687A6A1346DB00134440
:107EC0009B000B4403F516731B78012B2ED1BB6965
:107ED000002B2BDABB6903F480327B68D3F8D434EF
:107EE00003F001039A4221D179687A6A1346DB00D4
:107EF00013449B000B4403F2572301221A703B6A80
:107F00009B6943F080023B6A9A613B6A5B6903F0BC
:107F10008003002B0AD1FB6903F500635B68FA69F3
:107F200002F5006243F40073536008E07B6A01339A
:107F30007B627B681B791A467B6A9342B3D37B686A
:107F40001B685A697B681B6802F400125A617B68DF
:107F50001B68184605F08BFA034603F08043B3F123
:107F6000804F0AD178680AF09FFD7B681B685A69C8
:107F70007B681B6802F080425A617B681B68184668
:107F800005F075FA034603F00403042B15D17B6852
:107F90001B685B68BB61BB6903F00403002B02D064
:107FA00078680AF08FFD7B681B6859687B681B68DE
:107FB000BA690A435A6000E000BF3437BD4690BD3D
:107FC00080B584B000AF78607B681B68FB607B681D
:107FD00093F89434012B01D102231DE07B68012228
:107FE00083F894247B681B68184605F01FFAFB6829
:107FF000DB6803F04003002B09D07B685B7B012B1F
:1080000005D1FB689B6B23F48032FB689A637B6825
:10801000002283F89424002318461037BD4680BD03
:1080200080B582B000AF78600B46FB707B6893F838
:108030009434012B01D1022312E07B68012283F8E2
:1080400094247B68FA785A747B681B68FA78114626
:10805000184605F0A4F97B68002283F894240023D5
:1080600018460837BD4680BD80B584B000AF786043
:10807000084611461A460346FB700B463B801346E2
:10808000BB700023FB7297F90330002B0FDAFB78EB
:1080900003F00F021346DB0013449B0010337A6891
:1080A00013440433FB60FB6801225A700FE0FB7835
:1080B00003F00F021346DB0013449B0003F5147317
:1080C0007A6813440433FB60FB6800225A70FB7823
:1080D00003F00F03DAB2FB681A703B88C3F30A029D
:1080E000FB689A60FB68BA781A71FB685B78002BB2
:1080F00004D0FB681B781A46FB685A83BB78022BB6
:1081000002D1FB6800225A717B6893F89434012BEA
:1081100001D102230EE07B68012283F894247B685E
:108120001B68F968184604F0D5FA7B68002283F8CA
:108130009424FB7A18461037BD4680BD80B584B0C4
:1081400000AF78600B46FB7097F90330002B0FDA15
:10815000FB7803F00F021346DB0013449B0010333F
:108160007A6813440433FB60FB6801225A700FE005
:10817000FB7803F00F021346DB0013449B0003F56A
:1081800014737A6813440433FB60FB6800225A704E
:10819000FB7803F00F03DAB2FB681A707B6893F880
:1081A0009434012B01D102230EE07B68012283F875
:1081B00094247B681B68F968184604F013FB7B68FD
:1081C000002283F89424002318461037BD4680BD52
:1081D00080B586B000AFF8607A603B600B46FB72FA
:1081E000FB7A03F00F021346DB0013449B0003F5F8
:1081F0001473FA68134404337B617B697A68DA602C
:108200007B693A681A617B6900225A617B690022A6
:108210005A70FB7A03F00F03DAB27B691A70FB68BD
:108220009B79012B02D17A687B69DA61FB68186857
:10823000FB689B791A46796904F0B0FB0023184665
:108240001837BD4680BD80B483B000AF78600B4660
:10825000FB70FB7803F00F0279681346DB001344D0
:108260009B000B4403F51A731B6818460C37BD4678
:108270005DF8047B704780B586B000AFF8607A6027
:108280003B600B46FB72FB7A03F00F021346DB00E8
:1082900013449B001033FA68134404337B617B69F9
:1082A0007A68DA607B693A681A617B6900225A61F0
:1082B0007B6901225A70FB7A03F00F03DAB27B6903
:1082C0001A70FB689B79012B02D17A687B69DA61AD
:1082D000FB681868FB689B791A46796904F05EFBB5
:1082E000002318461837BD4680BD80B584B000AF66
:1082F00078600B46FB70FB7803F00F037A68127905
:10830000934201D901234FE097F90330002B0FDA94
:10831000FB7803F00F021346DB0013449B0010337D
:108320007A6813440433FB60FB6801225A700DE045
:10833000FA781346DB0013449B0003F514737A6844
:1083400013440433FB60FB6800225A70FB6801226F
:108350009A70FB7803F00F03DAB2FB681A707B683F
:1083600093F89434012B01D102231DE07B68012294
:1083700083F894247B681B68F968184604F0ECFEC7
:10838000FB7803F00F03002B09D17B6818687B682A
:1083900099797B6803F29C431A4605F02DF97B68B6
:1083A000002283F89424002318461037BD4680BD70
:1083B00080B584B000AF78600B46FB70FB7803F0AB
:1083C0000F037A681279934201D9012342E097F9A9
:1083D0000330002B0FDAFB7803F00F021346DB00AB
:1083E00013449B0010337A6813440433FB60FB682A
:1083F00001225A700FE0FB7803F00F021346DB00F6
:1084000013449B0003F514737A6813440433FB6030
:10841000FB6800225A70FB6800229A70FB7803F018
:108420000F03DAB2FB681A707B6893F89434012B5F
:1084300001D102230EE07B68012283F894247B683B
:108440001B68F968184604F0F5FE7B68002283F883
:108450009424002318461037BD4680BD80B584B0F3
:1084600000AF78600B46FB7097F90330002B0CDAF5
:10847000FB7803F00F021346DB0013449B0010331C
:108480007A6813440433FB600CE0FB7803F00F02BE
:108490001346DB0013449B0003F514737A681344FE
:1084A0000433FB607B681B68F968184604F014FD10
:1084B0000346FB72FB7A18461037BD4680BD80B577
:1084C0008AB002AF786039607B681B687B617B692A
:1084D0003B613A681346DB0013449B0010337A6813
:1084E00013440433FB60FB685A69FB681B699A42BA
:1084F00001D901236BE0FB681A69FB685B69D31A39
:10850000FB61FB689B68FA699A4202D9FB689B6829
:10851000FB61FB6903339B08BB612AE0FB681A69B6
:10852000FB685B69D31AFB61FB689B68FA699A4236
:1085300002D9FB689B68FB61FB6903339B08BB6145
:10854000FB68D9683B68DAB2FB6998B27B689B79B3
:1085500000930346786904F069FDFB68DA68FB69FB
:108560001A44FB68DA60FB685A69FB691A44FB68C5
:108570005A613B685A013B69134403F510639B69D8
:108580009BB2BA699A4209D8FB685A69FB681B69B1
:108590009A4203D2FB681B69002BBFD1FB681A69A2
:1085A000FB685B699A4211D83B6803F00F03012214
:1085B00002FA03F3BB603B6903F500635A6BBB68C7
:1085C000DB43396901F5006113404B630023184612
:1085D0002037BD4680BD000080B588B000AF786010
:1085E00039607B681B68FB61FB69BB61FB693C33DD
:1085F00004331B687B613B685A01BB69134403F574
:1086000030639B683B617B689B79012B7BD13B6925
:1086100003F00803002B15D07B69614A934240F2B6
:10862000B9803B6903F40043002B00F0B3803B6842
:108630005A01BB69134403F530631A464FF40043F3
:108640009360A7E03B6903F02003002B09D03B684F
:108650005A01BB69134403F530631A462023936023
:1086600098E03B6903F02803002B40F093807B697E
:108670004B4A93420FD93B6903F40043002B0AD0C5
:108680003B685A01BB69134403F530631A464FF443
:10869000004393607EE03A681346DB0013449B007E
:1086A00003F514737A6813440433FB60FB681A6A99
:1086B0003B685901BB690B4403F530631B69C3F385
:1086C0001203D21AFB685A613B68002B14D1FB6875
:1086D0001B69002B09D17B6818687B6803F29C43F7
:1086E0001A46012104F088FF06E0FB68DA68FB689F
:1086F0005B691A44FB68DA603B68DBB2194678684C
:108700000AF00EF946E07B69264A934224D13B6980
:1087100003F40043002B0AD03B685A01BB691344A1
:1087200003F530631A464FF40043936032E03B692F
:1087300003F02003002B08D03B685A01BB691344A7
:1087400003F530631A46202393603B68DBB2194679
:1087500078680AF0E5F81DE03B68002B14D17968D1
:108760003A681346DB0013449B000B4403F519736E
:108770001B68002B08D17B6818687B6803F29C4358
:108780001A46002104F038FF3B68DBB219467868CE
:108790000AF0C6F8002318462037BD4680BD00BF4A
:1087A0000A30544F0A31544F80B586B000AF78601C
:1087B00039607B681B687B617B693B617B693C330B
:1087C00004331B68FB603B685A013B69134403F5A3
:1087D00030639B68BB60FB68154A93420ED9BB6847
:1087E00003F40043002B09D03B685A013B69134452
:1087F00003F530631A464FF40043936078680AF03B
:108800007DF8FB680A4A93420CD97B689B79012B5F
:1088100008D17B6818687B6803F29C431A460121E3
:1088200004F0EAFE002318461837BD4680BD00BF9D
:108830000A30544F80B485B000AF78600B46FB70AF
:1088400013463B807B681B685B6ABB60FB78002B30
:1088500007D13B8819047B681B68BA680A439A628F
:1088600028E07B681B689B6A1B0CBA681344BB60DA
:108870000023FB730DE07B681A68FB7B40339B0091
:1088800013445B681B0CBA681344BB60FB7B013369
:10889000FB73FA7BFB78013B9A42ECD33B881804CC
:1088A0007B681968FB78013BBA68024340339B0040
:1088B0000B445A60002318461437BD465DF8047B0C
:1088C000704780B483B000AF78600B467B807B68D4
:1088D0001B687A885A62002318460C37BD465DF83B
:1088E000047B704780B485B000AF78607B681B68FC
:1088F000FB607B680122C3F8D8247B68002283F8E0
:10890000CC24FB689B6943F00062FB689A61FB68BA
:108910005B6D43F0805343F00303FA685365002313
:1089200018461437BD465DF8047B704780B483B0A9
:1089300000AF064B01221A60054B1B687B607B6809
:1089400000BF0C37BD465DF8047B704720000E4227
:108950000070004080B584B000AF786039607B68FB
:10896000002B01D10123CCE0684B1B6803F00F03FF
:108970003A689A420CD9654B3A68D2B21A70634B86
:108980001B6803F00F033A689A4201D00123B8E054
:108990007B681B6803F00203002B20D07B681B68F8
:1089A00003F00403002B05D0594B9B68584A43F44D
:1089B000E05393607B681B6803F00803002B05D02D
:1089C000534B9B68524A43F460439360504B9B68FF
:1089D00023F0F0027B689B684D4913438B607B68F2
:1089E0001B6803F00103002B44D07B685B68012BFC
:1089F00007D1474B1B6803F40033002B19D1012327
:108A00007FE07B685B68022B03D07B685B68032B8D
:108A100007D13F4B1B6803F00073002B09D10123E2
:108A20006FE03B4B1B6803F00203002B01D10123D5
:108A300067E0374B9B6823F003027B685B6834492F
:108A400013438B60FDF738FCF8600AE0FDF734FC57
:108A50000246FB68D31A41F28832934201D90323BC
:108A60004FE02B4B9B6803F00C027B685B689B001C
:108A70009A42EBD1254B1B6803F00F033A689A42E8
:108A80000CD2224B3A68D2B21A70204B1B6803F00A
:108A90000F033A689A4201D0012332E07B681B68D9
:108AA00003F00403002B08D0194B9B6823F4E05219
:108AB0007B68DB68164913438B607B681B6803F097
:108AC0000803002B09D0124B9B6823F460427B689B
:108AD0001B69DB000E4913438B6000F0B1FB0246BB
:108AE0000B4B9B681B0903F00F030A49CB5C22FA6E
:108AF00003F3094A1360094B1B681846FBF7EAFBAE
:108B0000002318461037BD4680BD00BF003C024020
:108B100000380240847301081C0000207800002007
:108B200080B400AF034B1B681846BD465DF8047B5C
:108B3000704700BF1C00002080B500AFFFF7F0FFBA
:108B40000246054B9B689B0A03F007030349CB5C75
:108B500022FA03F3184680BD0038024094730108DE
:108B600080B500AFFFF7DCFF0246054B9B685B0B4F
:108B700003F007030349CB5C22FA03F3184680BDD8
:108B8000003802409473010880B483B000AF78606D
:108B900039607B680F221A60124B9B6803F0030256
:108BA0007B685A600F4B9B6803F0F0027B689A6009
:108BB0000C4B9B6803F4E0527B68DA60094B9B68BE
:108BC000DB0803F4E0527B681A61074B1B6803F073
:108BD0000F023B681A6000BF0C37BD465DF8047B8E
:108BE000704700BF00380240003C024080B58CB0A6
:108BF00000AF786000237B6200233B620023FB61AF
:108C00000023BB6100237B6100233B610023FB60E9
:108C10000023FB620023BB627B681B6803F0010337
:108C2000002B10D06F4BD3F88C3023F0C0627B68E0
:108C30009B6B6C491343C1F88C307B689B6B002B9A
:108C400001D10123FB627B681B6803F00203002B48
:108C500010D0644BD3F88C3023F0C0527B68DB6BB0
:108C600060491343C1F88C307B68DB6B002B01D16A
:108C70000123FB627B681B6803F00403002B17D001
:108C8000584BD3F88C3023F440127B681B6B55494A
:108C90001343C1F88C307B681B6BB3F5801F01D187
:108CA0000123FB627B681B6B002B01D10123BB629C
:108CB0007B681B6803F00803002B17D0494BD3F8DF
:108CC0008C3023F440027B685B6B46491343C1F848
:108CD0008C307B685B6BB3F5800F01D10123FB62A5
:108CE0007B685B6B002B01D10123BB627B681B6837
:108CF00003F02003002B00F08A800023BB60394B77
:108D00001B6C384A43F080531364364B1B6C03F0E2
:108D10008053BB60BB68344B1B68334A43F4807399
:108D20001360FDF7C9FA786208E0FDF7C5FA02465C
:108D30007B6AD31A022B01D9032378E22A4B1B68E2
:108D400003F48073002BF0D0264B1B6F03F44073A9
:108D50003B623B6A002B2FD07B681B6C03F4407393
:108D60003A6A9A4228D01F4B1B6F23F440733B6230
:108D70001E4B01221A601D4B00221A60194A3B6AE1
:108D80001367184B1B6F03F00103012B14D1FDF780
:108D900093FA78620AE0FDF78FFA02467B6AD31AEB
:108DA00041F28832934201D9032340E20D4B1B6FFD
:108DB00003F00203002BEED07B681B6C03F44073BE
:108DC000B3F5407F14D1074B9B6823F4F8127B68FE
:108DD0001B6C23F0704323F44073024913438B60F0
:108DE0000CE000BF0038024000700040400E4742D7
:108DF0004A4B9B68494A23F4F8139360474B1A6F18
:108E00007B681B6CC3F30B03444913430B677B68FC
:108E10001B6803F01003002B04D07B6893F85820E4
:108E20003F4B1A607B681B6803F08003002B0AD05D
:108E30003A4BD3F8943023F440027B68DB6C37491B
:108E40001343C1F894307B681B6803F04003002B88
:108E50000AD0324BD3F8943023F080627B689B6C4D
:108E60002E491343C1F894307B681B6803F4807368
:108E7000002B11D0294BD3F8943023F000627B688B
:108E80005B6D26491343C1F894307B685B6DB3F189
:108E9000006F01D10123BB627B681B6803F4007380
:108EA000002B0AD01D4BD3F8943023F080527B68FE
:108EB0005B6C1A491343C1F894307B681B6803F458
:108EC0008063002B11D0154BD3F8943023F000525F
:108ED0007B681B6D11491343C1F894307B681B6D8F
:108EE000B3F1005F01D10123FB62FB6A012B05D0C6
:108EF0007B681B68B3F5006F40F0FF80094B0022D0
:108F00001A60FDF7D9F978620EE0FDF7D5F902464F
:108F10007B6AD31A022B07D9032388E10038024069
:108F2000E0114742680047427E4B1B6803F0006334
:108F3000002BEAD17B681B6803F00103002B03D0F0
:108F40007B689B6B002B09D07B681B6803F00203D6
:108F5000002B28D07B68DB6B002B24D1714BD3F81E
:108F600084301B0C03F0030301335B00FB616D4B8A
:108F7000D3F884301B0E03F00F03BB617B685A6883
:108F80007B689B689B011A43FB695B08013B1B04E0
:108F90001A43BB691B061A437B685B691B0761495F
:108FA0001343C1F884307B681B6803F00403002B73
:108FB00004D07B681B6BB3F5801F0AD07B681B68ED
:108FC00003F00803002B35D07B685B6BB3F5800F93
:108FD00030D1544BD3F884301B0C03F0030301331E
:108FE0005B00FB614F4BD3F884301B0F03F007038A
:108FF0007B617B685A687B689B689B011A43FB69AD
:109000005B08013B1B041A437B681B691B061A4360
:109010007B691B0743491343C1F88430414BD3F8A4
:109020008C3023F01F027B689B6A013B3D49134350
:10903000C1F88C307B681B6803F48063002B29D057
:109040007B681B6DB3F1005F24D1364BD3F88430BD
:109050001B0C03F0030301335B00BB61314BD3F8FE
:1090600084301B0F03F007037B617B685A687B68C1
:109070009B689B011A437B68DB685B08013B1B0410
:109080001A43BB691B061A437B691B072549134317
:10909000C1F884307B681B6803F40063002B16D092
:1090A0007B685A687B689B689B011A437B68DB6816
:1090B0005B08013B1B041A437B681B691B061A43B0
:1090C0007B685B691B0717491343C1F88430164B53
:1090D00001221A60FDF7F0F8786208E0FDF7ECF87D
:1090E00002467B6AD31A022B01D903239FE00D4B62
:1090F0001B6803F00063002BF0D0BB6A012B40F02B
:1091000095800A4B00221A60FDF7D6F878620FE0CE
:10911000FDF7D2F802467B6AD31A022B08D9032343
:1091200085E000BF003802406800474270004742B7
:10913000414B1B6803F00053B3F1005FE8D07B683C
:109140001B6803F00403002B03D07B681B6B002B10
:1091500009D07B681B6803F00803002B2BD07B68C9
:109160005B6B002B27D1344BD3F888301B0C03F0FA
:10917000030301335B003B617B689A697B68DB69B1
:109180009B011A433B695B08013B1B041A437B6844
:109190005B6A1B0628491343C1F88830264BD3F875
:1091A0008C3023F4F8527B68DB6A013B1B022249B6
:1091B0001343C1F88C307B681B6803F48073002B69
:1091C0001DD07B685B6DB3F1006F18D11A4BD3F8DB
:1091D00088301B0E03F00F03FB607B689A697B6885
:1091E000DB699B011A437B681B6A5B08013B1B041C
:1091F0001A43FB681B0610491343C1F888300F4B14
:1092000001221A60FDF758F8786208E0FDF754F87B
:1092100002467B6AD31A022B01D9032307E0064BCF
:109220001B6803F00053B3F1005FEFD10023184631
:109230003037BD4680BD00BF003802407000474255
:109240002DE9B04FAEB000AF0023C7F8AC3000231B
:10925000C7F8B4300023C7F8A8300023C7F8A430FB
:109260000023C7F8B030CB4B9B6803F00C030C2BEA
:1092700000F2068201A252F823F000BFB19200086A
:10928000819600088196000881960008B99200082E
:10929000819600088196000881960008C192000816
:1092A000819600088196000881960008B194000814
:1092B000B94BC7F8B030E7E1B84BC7F8B030E3E1DD
:1092C000B44B5B6803F03F03C7F8AC30B14B5B684D
:1092D00003F48003002B71D0AE4B5B689B09002226
:1092E000C7F89830C7F89C20D7F89830C3F3080324
:1092F000C7F890300023C7F89430D7E924452246B8
:109300002B464FF000004FF00001590141EAD261B5
:10931000500102460B462146511A3964294663EB37
:1093200001037B644FF000024FF00003D7E910897E
:1093300049468B01414643EA916341468A014146D1
:10934000511AB963494663EB0103FB634FF0000216
:109350004FF00003D7E90E894946CB00414643EA66
:1093600051734146CA0010461946034622469B18CF
:109370003B632B460A4642EB03037B634FF000023C
:109380004FF00003D7E90C4529464B02214643EA3A
:10939000D15321464A0210461946D7F8AC30002274
:1093A000C7F88830C7F88C20D7E92223F7F79CFC50
:1093B00002460B461346C7F8B43067E0754B5B684E
:1093C0009B090022C7F88030C7F88420D7F8803086
:1093D000C3F30803BB670023FB67D7E91E4522469A
:1093E0002B464FF000004FF00001590141EAD261D5
:1093F000500102460B462146511AB962294663EBD9
:109400000103FB624FF000024FF00003D7E90A8925
:1094100049468B01414643EA916341468A014146F0
:10942000B2EB010A494663EB010B4FF000024FF02B
:1094300000034FEACB0343EA5A734FEACA0292464B
:109440009B4623461AEB03033B622B464BEB03037D
:109450007B624FF000024FF00003D7E90845294630
:109460008B02214643EA915321468A02104619464F
:10947000D7F8AC3000223B677A67D7E91C23F7F7AF
:1094800033FC02460B461346C7F8B430414B5B68C9
:109490001B0C03F0030301335B00C7F8A830D7F8B7
:1094A000B420D7F8A830B2FBF3F3C7F8B030EBE044
:1094B000384B5B6803F03F03C7F8AC30354B5B6853
:1094C00003F48003002B6BD0324B5B689B090022B6
:1094D000BB66FA66BB6EC3F308033B6600237B667C
:1094E000D7E9184522462B464FF000004FF0000107
:1094F000590141EAD261500102460B462146511AF8
:10950000B961294663EB0103FB614FF000024FF0A4
:109510000003D7E906AB59468B01514643EA9163F4
:1095200051468A015146B2EB0108594663EB0109E5
:109530004FF000024FF000034FEAC90343EA5873AB
:109540004FEAC80290469946234618EB03033B6155
:109550002B4649EB03037B614FF000024FF0000301
:10956000D7E9044529464B02214643EAD153214617
:109570004A0210461946D7F8AC300022BB65FA659E
:10958000D7E91623F7F7B0FB02460B461346C7F898
:10959000B43065E0003802400024F40000127A0084
:1095A0003D4B5B689B09002218461146C0F3080337
:1095B0003B6500237B65D7E9148942464B464FF053
:1095C00000004FF00001590141EAD261500102460A
:1095D0000B464146511AB960494663EB0103FB60F3
:1095E0004FF000024FF00003D7E902AB59468B0160
:1095F000514643EA916351468A015146541A5946ED
:1096000063EB01054FF000024FF00003EB0043EA6B
:109610005473E20014461D464346E3183B604B4634
:1096200045EB03037B604FF000024FF00003D7E9E6
:10963000004529468B02214643EA915321468A027E
:1096400010461946D7F8AC300022BB64FA64D7E95B
:109650001223F7F749FB02460B461346C7F8B4300E
:109660000D4B5B681B0F03F00703C7F8A430D7F856
:10967000B420D7F8A430B2FBF3F3C7F8B03003E05E
:10968000064BC7F8B03000BFD7F8B0301846B8372F
:10969000BD46BDE8B08F00BF003802400024F40092
:1096A00080B586B000AF78607B68002B01D10123C4
:1096B0008DE27B681B6803F00103002B00F08380C0
:1096C000944B9B6803F00C03042B19D0914B9B68BF
:1096D00003F00C03082B06D18E4B5B6803F4800368
:1096E000B3F5800F0CD08B4B9B6803F00C030C2B55
:1096F00012D1884B5B6803F48003B3F5800F0BD164
:10970000844B1B6803F40033002B5BD07B685B68E1
:10971000002B57D101235AE27B685B68B3F5803F89
:1097200006D17C4B1B687B4A43F4803313601DE0F9
:109730007B685B68B3F5A02F0CD1764B1B68754A2C
:1097400043F480231360734B1B68724A43F48033E5
:1097500013600BE06F4B1B686E4A23F48033136079
:109760006C4B1B686B4A23F4802313607B685B6837
:10977000002B13D0FCF7A0FD386108E0FCF79CFD3E
:1097800002463B69D31A642B01D903231FE2614BC4
:109790001B6803F40033002BF0D014E0FCF78CFDC1
:1097A000386108E0FCF788FD02463B69D31A642B58
:1097B00001D903230BE2574B1B6803F40033002B42
:1097C000F0D100E000BF7B681B6803F00203002BB0
:1097D0006FD0504B9B6803F00C03002B17D04D4B00
:1097E0009B6803F00C03082B05D14A4B5B6803F41C
:1097F0008003002B0BD0474B9B6803F00C030C2B12
:109800001CD1444B5B6803F48003002B16D1414B01
:109810001B6803F00203002B05D07B68DB68012B7B
:1098200001D00123D3E13B4B1B6823F0F8027B6896
:109830001B69DB00374913430B603AE07B68DB6848
:10984000002B20D0344B01221A60FCF735FD386123
:1098500008E0FCF731FD02463B69D31A022B01D91F
:109860000323B4E12B4B1B6803F00203002BF0D061
:10987000284B1B6823F0F8027B681B69DB00254935
:1098800013430B6015E0244B00221A60FCF714FD13
:10989000386108E0FCF710FD02463B69D31A022B41
:1098A00001D9032393E11B4B1B6803F00203002B38
:1098B000F0D17B681B6803F00803002B36D07B686F
:1098C0005B69002B16D0154B01221A60FCF7F4FCE3
:1098D000386108E0FCF7F0FC02463B69D31A022B22
:1098E00001D9032373E10B4B5B6F03F00203002BE1
:1098F000F0D01BE0094B00221A60FCF7DDFC386158
:109900000EE0FCF7D9FC02463B69D31A022B07D9BB
:1099100003235CE10038024000004742800E4742CA
:109920008A4B5B6F03F00203002BEAD17B681B6854
:1099300003F00403002B00F097800023FB75834B9A
:109940001B6C03F08053002B0FD10023BB607F4BB7
:109950001B6C7E4A43F0805313647C4B1B6C03F0FA
:109960008053BB60BB680123FB75794B1B6803F414
:109970008073002B18D1764B1B68754A43F48073B3
:109980001360FCF799FC386108E0FCF795FC02468F
:109990003B69D31A022B01D9032318E16C4B1B68D6
:1099A00003F48073002BF0D07B689B68012B06D1F9
:1099B000664B1B6F654A43F0010313671CE07B682D
:1099C0009B68052B0CD1614B1B6F604A43F004036D
:1099D00013675E4B1B6F5D4A43F0010313670BE097
:1099E0005A4B1B6F594A23F001031367574B1B6FE8
:1099F000564A23F0040313677B689B68002B15D03D
:109A0000FCF75AFC38610AE0FCF756FC02463B6959
:109A1000D31A41F28832934201D90323D7E04B4B4A
:109A20001B6F03F00203002BEED014E0FCF744FCA4
:109A300038610AE0FCF740FC02463B69D31A41F268
:109A40008832934201D90323C1E0404B1B6F03F0DE
:109A50000203002BEED1FB7D012B05D13B4B1B6C90
:109A60003A4A23F0805313647B689B69002B00F013
:109A7000AD80364B9B6803F00C03082B60D07B68ED
:109A80009B69022B45D1334B00221A60FCF714FC72
:109A9000386108E0FCF710FC02463B69D31A022B40
:109AA00001D9032393E0294B1B6803F00073002BBB
:109AB000F0D17B68DA697B681B6A1A437B685B6A52
:109AC0009B011A437B689B6A5B08013B1B041A439A
:109AD0007B68DB6A1B061A437B681B6B1B071B49F1
:109AE00013434B601B4B01221A60FCF7E5FB386106
:109AF00008E0FCF7E1FB02463B69D31A022B01D9CF
:109B0000032364E0114B1B6803F00073002BF0D0BB
:109B10005CE0104B00221A60FCF7CEFB386108E0D5
:109B2000FCF7CAFB02463B69D31A022B01D9032377
:109B30004DE0064B1B6803F00073002BF0D145E0AD
:109B40007B689B69012B07D1012340E0003802406C
:109B500000700040600047421F4B5B68FB607B6801
:109B60009B69012B30D0FB6803F480027B68DB69C2
:109B70009A4229D1FB6803F03F027B681B6A9A4234
:109B800022D1FA6847F6C07313407A68526A92018C
:109B9000934219D1FB6803F440327B689B6A5B08EF
:109BA000013B1B049A420FD1FB6803F070627B6893
:109BB000DB6A1B069A4207D1FB6803F0E0427B6830
:109BC0001B6B1B079A4201D0012300E000231846BB
:109BD0001837BD4680BD00BF0038024080B582B056
:109BE00000AF78607B68002B01D1012341E07B68E6
:109BF00093F83D30DBB2002B06D17B68002283F85E
:109C00003C20786800F039F87B68022283F83D2018
:109C10007B681A687B6804331946104600F05AFFC7
:109C20007B68012283F846207B68012283F83E206E
:109C30007B68012283F83F207B68012283F8402063
:109C40007B68012283F841207B68012283F842204F
:109C50007B68012283F843207B68012283F844203B
:109C60007B68012283F845207B68012283F83D2030
:109C7000002318460837BD4680BD80B483B000AFCE
:109C8000786000BF0C37BD465DF8047B704700006C
:109C900080B485B000AF78607B6893F83D30DBB26C
:109CA000012B01D001234EE07B68022283F83D2086
:109CB0007B681B68DA687B681B6842F00102DA6027
:109CC0007B681B68234A934222D07B681B68B3F1F0
:109CD000804F1DD07B681B681F4A934218D07B6859
:109CE0001B681E4A934213D07B681B681C4A934230
:109CF0000ED07B681B681B4A934209D07B681B68A7
:109D0000194A934204D07B681B68184A934211D1C8
:109D10007B681B689B6803F00703FB60FB68062BEE
:109D200010D07B681B681A687B681B6842F00102D0
:109D30001A6007E07B681B681A687B681B6842F042
:109D400001021A60002318461437BD465DF8047BF3
:109D5000704700BF000001400004004000080040C0
:109D6000000C004000040140004001400018004089
:109D700080B582B000AF78607B68002B01D10123F1
:109D800041E07B6893F83D30DBB2002B06D17B6865
:109D9000002283F83C207868FAF760FA7B68022298
:109DA00083F83D207B681A687B68043319461046A7
:109DB00000F090FE7B68012283F846207B68012238
:109DC00083F83E207B68012283F83F207B680122D4
:109DD00083F840207B68012283F841207B680122C0
:109DE00083F842207B68012283F843207B680122AC
:109DF00083F844207B68012283F845207B68012298
:109E000083F83D20002318460837BD4680BD80B545
:109E100082B000AF78607B68022283F83D207B68C7
:109E20001B681A6A41F211131340002B0FD17B6893
:109E30001B681A6A40F244431340002B07D17B6829
:109E40001B681A687B681B6822F001021A60786838
:109E5000FAF726FA7B68002283F846207B68002206
:109E600083F83E207B68002283F83F207B68002235
:109E700083F840207B68002283F841207B68002221
:109E800083F842207B68002283F843207B6800220D
:109E900083F844207B68002283F845207B680022F9
:109EA00083F83D207B68002283F83C20002318467D
:109EB0000837BD4680BD000080B584B000AF786033
:109EC00039603B68002B09D17B6893F83E30DBB2E8
:109ED000012B14BF01230023DBB222E03B68042BDB
:109EE00009D17B6893F83F30DBB2012B14BF01230B
:109EF0000023DBB215E03B68082B09D17B6893F89F
:109F00004030DBB2012B14BF01230023DBB208E099
:109F10007B6893F84130DBB2012B14BF012300238F
:109F2000DBB2002B01D001237CE03B68002B04D185
:109F30007B68022283F83E2013E03B68042B04D1A7
:109F40007B68022283F83F200BE03B68082B04D19A
:109F50007B68022283F8402003E07B68022283F8BA
:109F600041207B681B6801223968184601F049FAD4
:109F70007B681B682D4A934204D07B681B682C4A7F
:109F8000934201D1012300E00023002B07D07B681E
:109F90001B685A6C7B681B6842F400425A647B68F9
:109FA0001B68224A934222D07B681B68B3F1804F22
:109FB0001DD07B681B681F4A934218D07B681B68C2
:109FC0001D4A934213D07B681B681C4A93420ED0F3
:109FD0007B681B68164A934209D07B681B68184A45
:109FE000934204D07B681B68164A934211D17B6868
:109FF0001B689B6803F00703FB60FB68062B10D00F
:10A000007B681B681A687B681B6842F001021A6053
:10A0100007E07B681B681A687B681B6842F00102D6
:10A020001A60002318461037BD4680BD000001406D
:10A03000000401400004004000080040000C004003
:10A04000004001400018004080B582B000AF786049
:10A050007B68002B01D1012341E07B6893F83D3000
:10A06000DBB2002B06D17B68002283F83C207868A5
:10A07000FAF740F87B68022283F83D207B681A6873
:10A080007B6804331946104600F024FD7B680122EA
:10A0900083F846207B68012283F83E207B680122FA
:10A0A00083F83F207B68012283F840207B680122EF
:10A0B00083F841207B68012283F842207B680122DB
:10A0C00083F843207B68012283F844207B680122C7
:10A0D00083F845207B68012283F83D200023184641
:10A0E0000837BD4680BD000080B584B000AF786001
:10A0F00039603B68002B04D17B6893F83E30DBB2BB
:10A1000013E03B68042B04D17B6893F83F30DBB24B
:10A110000BE03B68082B04D17B6893F84030DBB23E
:10A1200003E07B6893F84130DBB2FB733B68002BA4
:10A1300004D17B6893F84230DBB213E03B68042B18
:10A1400004D17B6893F84330DBB20BE03B68082B0B
:10A1500004D17B6893F84430DBB203E07B6893F86A
:10A160004530DBB2BB73FB7B012B02D1BB7B012BE8
:10A1700001D0012381E03B68002B04D17B680222DF
:10A1800083F83E2013E03B68042B04D17B68022255
:10A1900083F83F200BE03B68082B04D17B68022248
:10A1A00083F8402003E07B68022283F841203B686B
:10A1B000002B04D17B68022283F8422013E03B6825
:10A1C000042B04D17B68022283F843200BE03B6818
:10A1D000082B04D17B68022283F8442003E07B68CB
:10A1E000022283F845207B681B68012239681846E3
:10A1F00001F007F97B681B68224A934222D07B68F2
:10A200001B68B3F1804F1DD07B681B681E4A9342C8
:10A2100018D07B681B681D4A934213D07B681B686B
:10A220001B4A93420ED07B681B681A4A934209D09E
:10A230007B681B68184A934204D07B681B68174AE6
:10A24000934211D17B681B689B6803F00703BB60D6
:10A25000BB68062B10D07B681B681A687B681B687C
:10A2600042F001021A6007E07B681B681A687B688D
:10A270001B6842F001021A60002318461037BD46E1
:10A2800080BD00BF00000140000400400008004005
:10A29000000C004000040140004001400018004054
:10A2A00080B584B000AF786039600023FB733B68F1
:10A2B000002B04D17B6893F83E30DBB213E03B689F
:10A2C000042B04D17B6893F83F30DBB20BE03B6892
:10A2D000082B04D17B6893F84030DBB203E07B6845
:10A2E00093F84130DBB2BB733B68002B04D17B6831
:10A2F00093F84230DBB213E03B68042B04D17B6857
:10A3000093F84330DBB20BE03B68082B04D17B6849
:10A3100093F84430DBB203E07B6893F84530DBB25E
:10A320007B73BB7B012B02D17B7B012B01D00123F3
:10A33000CCE03B68002B04D17B68022283F83E20EE
:10A3400013E03B68042B04D17B68022283F83F2092
:10A350000BE03B68082B04D17B68022283F8402085
:10A3600003E07B68022283F841203B68002B04D184
:10A370007B68022283F8422013E03B68042B04D15F
:10A380007B68022283F843200BE03B68082B04D152
:10A390007B68022283F8442003E07B68022283F872
:10A3A00045203B680C2B41D801A252F823F000BF96
:10A3B000E5A300082DA400082DA400082DA4000882
:10A3C000F7A300082DA400082DA400082DA4000860
:10A3D00009A400082DA400082DA400082DA400083D
:10A3E0001BA400087B681B68DA687B681B6842F066
:10A3F0000202DA601DE07B681B68DA687B681B6814
:10A4000042F00402DA6014E07B681B68DA687B685B
:10A410001B6842F00802DA600BE07B681B68DA68B0
:10A420007B681B6842F01002DA6002E00123FB73D4
:10A4300000BFFB7B002B48D17B681B680122396879
:10A44000184600F0DEFF7B681B68224A934222D048
:10A450007B681B68B3F1804F1DD07B681B681E4A68
:10A46000934218D07B681B681C4A934213D07B68C8
:10A470001B681B4A93420ED07B681B68194A9342A3
:10A4800009D07B681B68184A934204D07B681B681C
:10A49000164A934211D17B681B689B6803F007033F
:10A4A000BB60BB68062B10D07B681B681A687B6892
:10A4B0001B6842F001021A6007E07B681B681A689B
:10A4C0007B681B6842F001021A60FB7B184610375C
:10A4D000BD4680BD0000014000040040000800406F
:10A4E000000C004000040140004001400018004002
:10A4F00080B584B000AF78607B681B68DB68FB6068
:10A500007B681B681B69BB60BB6803F00203002B00
:10A5100020D0FB6803F00203002B1BD07B681B6874
:10A520006FF002021A617B6801221A777B681B6850
:10A530009B6903F00303002B03D07868F9F76EFAE8
:10A5400005E0786800F0A8FA786800F0AFFA7B6858
:10A5500000221A77BB6803F00403002B20D0FB68AD
:10A5600003F00403002B1BD07B681B686FF0040210
:10A570001A617B6802221A777B681B689B6903F467
:10A580004073002B03D07868F9F748FA05E0786843
:10A5900000F082FA786800F089FA7B6800221A7766
:10A5A000BB6803F00803002B20D0FB6803F008030E
:10A5B000002B1BD07B681B686FF008021A617B6858
:10A5C00004221A777B681B68DB6903F00303002B06
:10A5D00003D07868F9F722FA05E0786800F05CFAB1
:10A5E000786800F063FA7B6800221A77BB6803F092
:10A5F0001003002B20D0FB6803F01003002B1BD0AE
:10A600007B681B686FF010021A617B6808221A775A
:10A610007B681B68DB6903F44073002B03D0786808
:10A62000F9F7FCF905E0786800F036FA786800F090
:10A630003DFA7B6800221A77BB6803F00103002B08
:10A640000CD0FB6803F00103002B07D07B681B686C
:10A650006FF001021A617868F9F7C0FABB6803F07D
:10A660008003002B0CD0FB6803F08003002B07D085
:10A670007B681B686FF080021A61786800F06CFFDD
:10A68000BB6803F04003002B0CD0FB6803F04003D1
:10A69000002B07D07B681B686FF040021A61786856
:10A6A00000F00EFABB6803F02003002B0CD0FB680F
:10A6B00003F02003002B07D07B681B686FF020029B
:10A6C0001A61786800F03EFF00BF1037BD4680BDBC
:10A6D00080B586B000AFF860B9607A600023FB7582
:10A6E000FB6893F83C30012B01D1022388E0FB6822
:10A6F000012283F83C207B68002B1BD1FB68186883
:10A70000BB681968BB685A68BB68DB6800F0D0FC9E
:10A71000FB681B689A69FB681B6822F00C029A614F
:10A72000FB681B689969BB689A68FB681B680A43E9
:10A730009A6160E07B68042B1CD1FB681868BB68D9
:10A740001968BB685A68BB68DB6800F054FDFB6899
:10A750001B689A69FB681B6822F440629A61FB6877
:10A760001B689969BB689B681A02FB681B680A43EF
:10A770009A6140E07B68082B1BD1FB681868BB68B6
:10A780001968BB685A68BB68DB6800F0A1FDFB680C
:10A790001B68DA69FB681B6822F00C02DA61FB684F
:10A7A0001B68D969BB689A68FB681B680A43DA6151
:10A7B00021E07B680C2B1CD1FB681868BB6819680A
:10A7C000BB685A68BB68DB6800F0BEFDFB681B68AD
:10A7D000DA69FB681B6822F44062DA61FB681B6877
:10A7E000D969BB689B681A02FB681B680A43DA6177
:10A7F00001E00123FB75FB68002283F83C20FB7D10
:10A8000018461837BD4680BD80B586B000AFF860E9
:10A81000B9607A600023FB75FB6893F83C30012B2C
:10A8200001D10223AEE0FB68012283F83C207B6863
:10A830000C2B00F29F8001A252F823F071A80008AF
:10A8400075A9000875A9000875A90008B1A8000835
:10A8500075A9000875A9000875A90008F3A80008E3
:10A8600075A9000875A9000875A9000833A9000892
:10A87000FB681B68B968184600F0D8F9FB681B68CC
:10A880009A69FB681B6842F008029A61FB681B68C2
:10A890009A69FB681B6822F004029A61FB681B68D6
:10A8A0009969BB681A69FB681B680A439A6164E08E
:10A8B000FB681B68B968184600F028FAFB681B683B
:10A8C0009A69FB681B6842F400629A61FB681B6826
:10A8D0009A69FB681B6822F480629A61FB681B68B6
:10A8E0009969BB681B691A02FB681B680A439A6175
:10A8F00043E0FB681B68B968184600F07DFAFB6806
:10A900001B68DA69FB681B6842F00802DA61FB68C1
:10A910001B68DA69FB681B6822F00402DA61FB68D5
:10A920001B68D969BB681A69FB681B680A43DA614E
:10A9300023E0FB681B68B968184600F0D1FAFB6891
:10A940001B68DA69FB681B6842F40062DA61FB6825
:10A950001B68DA69FB681B6822F48062DA61FB68B5
:10A960001B68D969BB681B691A02FB681B680A432C
:10A97000DA6102E00123FB7500BFFB68002283F867
:10A980003C20FB7D18461837BD4680BD80B582B09F
:10A9900000AF786039607B6893F83C30012B01D1BF
:10A9A000022331E07B68012283F83C207B6802228D
:10A9B00083F83D203968786800F0E8FA0346002BF8
:10A9C00009D07B68012283F83D207B68002283F850
:10A9D0003C20012318E07B681B68DA687B681B68F1
:10A9E00022F04002DA607B681B68DA687B681B68CB
:10A9F00022F48042DA607B68012283F83D207B6884
:10AA0000002283F83C20002318460837BD4680BD4D
:10AA100080B485B000AF786039600023FB603B688C
:10AA20000C2B31D801A252F823F000BF61AA000814
:10AA300089AA000889AA000889AA00086BAA000848
:10AA400089AA000889AA000889AA000875AA00082E
:10AA500089AA000889AA000889AA00087FAA000814
:10AA60007B681B685B6BFB600FE07B681B689B6B04
:10AA7000FB600AE07B681B68DB6BFB6005E07B68C2
:10AA80001B681B6CFB6000E000BFFB6818461437B6
:10AA9000BD465DF8047B704780B483B000AF78603A
:10AAA00000BF0C37BD465DF8047B704780B483B0AF
:10AAB00000AF786000BF0C37BD465DF8047B70477F
:10AAC00080B483B000AF786000BF0C37BD465DF83E
:10AAD000047B704780B485B000AF786039607B68D4
:10AAE0001B68FB607B68464A934213D07B68B3F1D6
:10AAF000804F0FD07B68434A93420BD07B68424A19
:10AB0000934207D07B68414A934203D07B68404A16
:10AB1000934208D1FB6823F07003FB603B685B68DD
:10AB2000FA681343FB607B68354A93422BD07B68FD
:10AB3000B3F1804F27D07B68324A934223D07B68A1
:10AB4000314A93421FD07B68304A93421BD07B68C6
:10AB50002F4A934217D07B682E4A934213D07B68CA
:10AB60002D4A93420FD07B682C4A93420BD07B68CE
:10AB70002B4A934207D07B682A4A934203D07B68D2
:10AB8000294A934208D1FB6823F44073FB603B6879
:10AB9000DB68FA681343FB60FB6823F080023B68C4
:10ABA0005B691343FB607B68FA681A603B689A68CC
:10ABB0007B68DA623B681A687B689A627B68104A35
:10ABC000934203D07B68124A934203D13B681A69CF
:10ABD0007B681A637B6801225A617B681B6903F0FA
:10ABE0000103012B05D17B681B6923F001027B68FF
:10ABF0001A6100BF1437BD465DF8047B704700BF83
:10AC0000000001400004004000080040000C00402B
:10AC10000004014000400140004401400048014060
:10AC200000180040001C00400020004080B487B0A5
:10AC300000AF786039607B681B6A7B617B681B6A48
:10AC400023F001027B681A627B685B683B617B686A
:10AC50009B69FB60FB6823F07003FB60FB6823F0DB
:10AC60000303FB603B681B68FA681343FB607B6966
:10AC700023F002037B613B689B687A6913437B6125
:10AC80007B68204A934203D07B681F4A93420CD1D1
:10AC90007B6923F008037B613B68DB687A691343B7
:10ACA0007B617B6923F004037B617B68154A9342D7
:10ACB00003D07B68144A934211D13B6923F480731B
:10ACC0003B613B6923F400733B613B685B693A6914
:10ACD00013433B613B689B693A6913433B617B6863
:10ACE0003A695A607B68FA689A613B685A687B687F
:10ACF0005A637B687A691A6200BF1C37BD465DF8EB
:10AD0000047B7047000001400004014080B487B01C
:10AD100000AF786039607B681B6A7B617B681B6A67
:10AD200023F010027B681A627B685B683B617B687A
:10AD30009B69FB60FB6823F4E043FB60FB6823F442
:10AD40004073FB603B681B681B02FA681343FB609F
:10AD50007B6923F020037B613B689B681B017A6958
:10AD600013437B617B68224A934203D07B68214A6C
:10AD700093420DD17B6923F080037B613B68DB68E4
:10AD80001B017A6913437B617B6923F040037B617C
:10AD90007B68174A934203D07B68164A934213D1CB
:10ADA0003B6923F480633B613B6923F400633B61AF
:10ADB0003B685B699B003A6913433B613B689B6955
:10ADC0009B003A6913433B617B683A695A607B6830
:10ADD000FA689A613B685A687B689A637B687A690B
:10ADE0001A6200BF1C37BD465DF8047B704700BF88
:10ADF000000001400004014080B487B000AF7860DB
:10AE000039607B681B6A7B617B681B6A23F48072F4
:10AE10007B681A627B685B683B617B68DB69FB600F
:10AE2000FB6823F07003FB60FB6823F00303FB6007
:10AE30003B681B68FA681343FB607B6923F400736B
:10AE40007B613B689B681B027A6913437B617B686B
:10AE5000214A934203D07B68204A93420DD17B69FB
:10AE600023F400637B613B68DB681B027A69134350
:10AE70007B617B6923F480637B617B68164A934224
:10AE800003D07B68154A934213D13B6923F4805366
:10AE90003B613B6923F400533B613B685B691B01E9
:10AEA0003A6913433B613B689B691B013A69134351
:10AEB0003B617B683A695A607B68FA68DA613B6893
:10AEC0005A687B68DA637B687A691A6200BF1C374C
:10AED000BD465DF8047B704700000140000401405E
:10AEE00080B487B000AF786039607B681B6A3B61D3
:10AEF0007B681B6A23F480527B681A627B685B68FC
:10AF00007B617B68DB69FB60FB6823F4E043FB60EB
:10AF1000FB6823F44073FB603B681B681B02FA6804
:10AF20001343FB603B6923F400533B613B689B6820
:10AF30001B033A6913433B617B68124A934203D077
:10AF40007B68114A934209D17B6923F480437B617A
:10AF50003B685B699B017A6913437B617B687A6913
:10AF60005A607B68FA68DA613B685A687B681A64E1
:10AF70007B683A691A6200BF1C37BD465DF8047BE6
:10AF8000704700BF000001400004014080B586B05A
:10AF900000AF786039600023FB757B681B689B6895
:10AFA0003B613B6923F070033B613B685B683A6936
:10AFB00013433B613B6923F007033B613B681B681C
:10AFC0003A6913433B617B681B683A699A603B6846
:10AFD0005B68702B1AD0702B60D8602B54D0602B1C
:10AFE0005CD8502B46D0502B58D8402B19D0402B32
:10AFF00054D8302B55D0302B50D8202B51D0202B6B
:10B000004CD8002B4DD0102B4BD047E07B681868F4
:10B010003B68D9683B689A683B681B6900F0D1F9C6
:10B0200040E03B681B68052B01D101233BE07B68B6
:10B030001B681B6AFB607B681B681A6A7B681B685D
:10B0400022F001021A627B681B689B69BB60BB68C7
:10B0500023F0F003BB603B681B691B01BA68134314
:10B06000BB607B681B68BA689A617B681B68FA687A
:10B070001A6217E07B6818683B6899683B681B692F
:10B080001A4600F089F80DE07B6818683B689968FB
:10B090003B681B691A4600F0EBF803E00123FB75DF
:10B0A00000E000BFFB7D18461837BD4680BD00009C
:10B0B00080B487B000AFF860B9607A603B60FB682D
:10B0C0001B6A3B61FB681B6A23F00102FB681A6282
:10B0D000FB689B697B61FB68284A93421BD0FB6835
:10B0E000B3F1804F17D0FB68254A934213D0FB6819
:10B0F000244A93420FD0FB68234A93420BD0FB684B
:10B10000224A934207D0FB68214A934203D0FB684E
:10B11000204A934201D1012300E00023002B08D0F4
:10B120007B6923F003037B617A697B6813437B614E
:10B1300003E07B6943F001037B617B6923F0F0034B
:10B140007B613B681B01DBB27A6913437B613B691E
:10B1500023F00A033B61BB6803F00A033A69134317
:10B160003B61FB687A699A61FB683A691A6200BFC1
:10B170001C37BD465DF8047B704700BF00000140EE
:10B180000004004000080040000C004000040140A2
:10B19000004001400018004080B487B000AFF86064
:10B1A000B9607A60FB681B6A7B61FB681B6A23F0ED
:10B1B0000102FB681A62FB689B693B613B6923F0F3
:10B1C000F0033B617B681B013A6913433B617B6978
:10B1D00023F00A037B617A69BB6813437B61FB68D8
:10B1E0003A699A61FB687A691A6200BF1C37BD46EA
:10B1F0005DF8047B704780B487B000AFF860B96039
:10B200007A603B60FB681B6A7B61FB681B6A23F00A
:10B210001002FB681A62FB689B693B613B6923F47F
:10B2200040733B617B681B023A6913433B613B6996
:10B2300023F470433B613B681B039BB23A691343A1
:10B240003B617B6923F0A0037B61BB681B0103F0BA
:10B25000A0037A6913437B61FB683A699A61FB68D2
:10B260007A691A6200BF1C37BD465DF8047B7047DF
:10B2700080B487B000AFF860B9607A60FB681B6A81
:10B280007B61FB681B6A23F01002FB681A62FB6893
:10B290009B693B613B6923F470433B617B681B0303
:10B2A0003A6913433B617B6923F0A0037B61BB6870
:10B2B0001B017A6913437B61FB683A699A61FB68F9
:10B2C0007A691A6200BF1C37BD465DF8047B70477F
:10B2D00080B487B000AFF860B9607A603B60FB680B
:10B2E0001B6A7B61FB681B6A23F48072FB681A622D
:10B2F000FB68DB693B613B6923F003033B613A690F
:10B300007B6813433B613B6923F0F0033B613B687F
:10B310001B01DBB23A6913433B617B6923F4206371
:10B320007B61BB681B0203F420637A6913437B6172
:10B33000FB683A69DA61FB687A691A6200BF1C37F8
:10B34000BD465DF8047B704780B487B000AFF860FD
:10B35000B9607A603B60FB681B6A7B61FB681B6AB3
:10B3600023F48052FB681A62FB68DB693B613B692E
:10B3700023F440733B617B681B023A6913433B61D2
:10B380003B6923F470433B613B681B039BB23A6902
:10B3900013433B617B6923F420437B61BB681B0340
:10B3A00003F420437A6913437B61FB683A69DA61ED
:10B3B000FB687A691A6200BF1C37BD465DF8047BE2
:10B3C000704780B487B000AFF860B9607A603B60C6
:10B3D000FB689B687B617B6923F47F437B613B68EF
:10B3E0001A027B681A43BB6813437A6913437B6173
:10B3F000FB687A699A6000BF1C37BD465DF8047B24
:10B40000704780B487B000AFF860B9607A60BB68FD
:10B4100003F01F03012202FA03F37B61FB681A6A3F
:10B420007B69DB431A40FB681A62FB681A6ABB68D7
:10B4300003F01F03796801FA03F31A43FB681A62E9
:10B4400000BF1C37BD465DF8047B704780B485B0F3
:10B4500000AF786039607B6893F83C30012B01D1F4
:10B4600002235AE07B68012283F83C207B68022299
:10B4700083F83D207B681B685B68FB607B681B680A
:10B480009B68BB60FB6823F07003FB603B681B6834
:10B49000FA681343FB607B681B68FA685A607B6834
:10B4A0001B68214A934222D07B681B68B3F1804F0E
:10B4B0001DD07B681B681D4A934218D07B681B68AF
:10B4C0001B4A934213D07B681B681A4A93420ED0E2
:10B4D0007B681B68184A934209D07B681B68174A2F
:10B4E000934204D07B681B68154A93420CD1BB6819
:10B4F00023F08003BB603B685B68BA681343BB60A2
:10B500007B681B68BA689A607B68012283F83D20DB
:10B510007B68002283F83C20002318461437BD4680
:10B520005DF8047B704700BF00000140000400404C
:10B5300000080040000C00400004014000400140B1
:10B540000018004080B483B000AF786000BF0C37B3
:10B55000BD465DF8047B704780B483B000AF78606F
:10B5600000BF0C37BD465DF8047B704780B582B0E4
:10B5700000AF78607B68002B01D101234AE07B6833
:10B5800093F84130DBB2002B06D17B68002283F8B0
:10B5900040207868F8F7FCFD7B68242283F841207E
:10B5A0007B681B68DA687B681B6822F40052DA60EB
:10B5B000786800F0ABFA7B681B681A697B681B68C7
:10B5C00022F490421A617B681B685A697B681B6889
:10B5D00022F022025A617B681B685A697B681B68EB
:10B5E00042F008025A617B681B68DA687B681B6856
:10B5F00042F40052DA607B6800225A647B682022A1
:10B6000083F841207B68202283F842207B68002257
:10B610005A63002318460837BD4680BD80B582B006
:10B6200000AF78607B68002B01D1012324E07B68A8
:10B63000242283F841207B681B68DA687B681B68DA
:10B6400022F40052DA607868F8F7EAFD7B6800229D
:10B650005A647B68002283F841207B68002283F8CB
:10B6600042207B6800221A637B6800225A637B6851
:10B67000002283F84020002318460837BD4680BDCD
:10B6800080B58AB002AFF860B9603B601346FB80BA
:10B6900000237B61FB6893F84130DBB2202B75D12E
:10B6A000BB68002B02D0FB88002B01D101236EE088
:10B6B000FB6800225A64FB68212283F84120FAF7D4
:10B6C000FBFD7861FB68FA889A84FB68FA88DA8463
:10B6D000FB689B68B3F5805F08D1FB681B69002B92
:10B6E00004D10023FB61BB68BB6103E0BB68FB6165
:10B6F0000023BB612EE03B6800937B690022802120
:10B70000F86800F047F90346002B05D0FB682022BB
:10B7100083F8412003233AE0FB69002B0BD1BB697E
:10B720001B881A46FB681B68C2F308025A60BB6993
:10B730000233BB6107E0FB691A78FB681B685A603B
:10B74000FB690133FB61FB68DB8C9BB2013B9AB266
:10B75000FB68DA84FB68DB8C9BB2002BCBD13B68A7
:10B7600000937B6900224021F86800F013F903463A
:10B77000002B05D0FB68202283F84120032306E03C
:10B78000FB68202283F84120002300E002231846B2
:10B790002037BD4680BD80B58AB002AFF860B96081
:10B7A0003B601346FB8000237B61FB6893F84230CB
:10B7B000DBB2202B40F08180BB68002B02D0FB88DD
:10B7C000002B01D1012379E0FB6800225A64FB6859
:10B7D000222283F84220FB6800221A63FAF76CFDEC
:10B7E0007861FB68FA889A85FB68FA88DA85FB68D5
:10B7F0009B68B3F5805F08D1FB681B69002B04D1FF
:10B800000023FB61BB68BB6103E0BB68FB610023F5
:10B81000BB6147E03B6800937B6900222021F86808
:10B8200000F0B8F80346002B05D0FB68202283F80F
:10B830004220032342E0FB69002B0CD1FB681B680C
:10B840005B689BB2C3F308039AB2BB691A80BB69F9
:10B850000233BB611FE0FB689B68B3F5805F07D0D4
:10B86000FB689B68002B0AD1FB681B69002B06D183
:10B87000FB681B685B68DAB2FB691A7008E0FB685A
:10B880001B685B68DBB203F07F03DAB2FB691A70F6
:10B89000FB690133FB61FB68DB8D9BB2013B9AB214
:10B8A000FB68DA85FB68DB8D9BB2002BB2D1FB68AD
:10B8B000202283F84220002300E00223184620378C
:10B8C000BD4680BD80B485B000AF78600023FB60CA
:10B8D0007B6893F84030012B01D1022320E07B6884
:10B8E000012283F840207B68242283F841207B6872
:10B8F0001B68DB68FB60FB6823F00C03FB60FB68E4
:10B9000043F00803FB607B681B68FA68DA607B68B9
:10B91000202283F841207B68002283F84020002306
:10B9200018461437BD465DF8047B704780B485B077
:10B9300000AF78600023FB607B6893F84030012BF8
:10B9400001D1022320E07B68012283F840207B683C
:10B95000242283F841207B681B68DB68FB60FB685E
:10B9600023F00C03FB60FB6843F00403FB607B687F
:10B970001B68FA68DA607B68202283F841207B68C4
:10B98000002283F84020002318461437BD465DF896
:10B99000047B704780B586B000AFF860B9603B604B
:10B9A0001346FB713BE03B6AB3F1FF3F37D0FAF738
:10B9B00083FC02463B68D31A3A6A9A4202D33B6A36
:10B9C000002B01D103233AE0FB681B68DB6803F01E
:10B9D0000403002B23D0BB68802B20D0BB68402BF6
:10B9E0001DD0FB681B681B6803F00803082B16D1E9
:10B9F00000237B61FB681B681B687B61FB681B681D
:10BA00005B687B617B69F86800F01DF8FB680822C1
:10BA10005A64FB68002283F8402001230FE0FB6892
:10BA20001B681A68BB681340BA689A420CBF0123AE
:10BA30000023DBB21A46FB799A42B4D000231846A1
:10BA40001837BD4680BD80B495B000AF78607B6884
:10BA50001B680C337B637B6B53E8003F3B633B6BA2
:10BA600023F49073FB647B681B680C33FA6C3A64B4
:10BA7000FB63F96B3A6C41E80023BB63BB6B002BA3
:10BA8000E5D17B681B6814333B623B6A53E8003F97
:10BA9000FB61FB6923F00103BB647B681B68143303
:10BAA000BA6CFA62BB62B96AFA6A41E800237B6247
:10BAB0007B6A002BE5D17B681B6B012B19D17B685E
:10BAC0001B680C33FB60FB6853E8003FBB60BB683E
:10BAD00023F010037B647B681B680C337A6CBA61BB
:10BAE0007B617969BA6941E800233B613B69002BBE
:10BAF000E5D17B68202283F842207B6800221A630C
:10BB000000BF5437BD465DF8047B70472DE9B04F48
:10BB1000C0B000AFC7F8F400D7F8F4301B681B6959
:10BB200023F44050D7F8F430D968D7F8F4301A68C5
:10BB300040EA01031361D7F8F4309A68D7F8F4307B
:10BB40001B691A43D7F8F4305B691A43D7F8F4300D
:10BB5000DB691343C7F8F830D7F8F4301B68DB68AB
:10BB600023F4164121F00C01D7F8F4301A68D7F805
:10BB7000F8300B43D360D7F8F4301B685B6923F4CB
:10BB80004070D7F8F4309969D7F8F4301A6840EA71
:10BB900001035361D7F8F4301A688F4B9A4205D0ED
:10BBA000D7F8F4301A688D4B9A4204D1FCF7D8FFCD
:10BBB000C7F8FC0003E0FCF7BFFFC7F8FC00D7F8AC
:10BBC000F430DB69B3F5004F40F00C81D7F8FC305E
:10BBD0000022C7F8E830C7F8EC20D7E93A452246FA
:10BBE0002B469118B9655B41FB65D7E916232146C1
:10BBF00012EB0108294643EB01094FF000024FF018
:10BC000000034FEAC90343EA58734FEAC80290465B
:10BC10009946234618EB0303C7F8E0302B4649EB5F
:10BC20000303C7F8E430D7F8F4305B680022C7F8A4
:10BC3000D830C7F8DC20D7E936120B46DB183B6555
:10BC4000134642EB03037B65D7E91423D7E9380198
:10BC5000F5F74AF802460B46614BA3FB02235B094A
:10BC60001C01D7F8FC300022C7F8D030C7F8D42028
:10BC7000D7E9348942464B469118B9645B41FB646D
:10BC8000D7E91223414612EB010A494643EB010B67
:10BC90004FF000024FF000034FEACB0343EA5A7320
:10BCA0004FEACA0292469B4643461AEB0303C7F883
:10BCB000C8304B464BEB0303C7F8CC30D7F8F43011
:10BCC0005B680022C7F8C030C7F8C420D7E930123B
:10BCD0000B46DB183B64134642EB03037B64D7E956
:10BCE0001023D7E93201F4F7FFFF02460B46114655
:10BCF0003B4BA3FB01235B09642202FB03F3CB1A3A
:10BD0000DB0003F13202364BA3FB02235B095B002D
:10BD100003F4F8731C44D7F8FC300022C7F8B8309D
:10BD2000C7F8BC20D7E92E8942464B469118B96323
:10BD30005B41FB63D7E90E234146511839634946FD
:10BD40004B417B634FF000024FF00003D7E90CAB8F
:10BD50005946CB00514643EA51735146CA0010463A
:10BD60001946034642469B18C7F8B0304B460A4670
:10BD700042EB0303C7F8B430D7F8F4305B68002215
:10BD8000C7F8A830C7F8AC20D7E92A120B46DB1851
:10BD9000BB62134642EB0303FB62D7E90A23D7E9F0
:10BDA0002C01F4F7A1FF02460B460D4BA3FB021337
:10BDB0005B09642101FB03F3D31ADB003233084A29
:10BDC000A2FB03235B0903F00702D7F8F4301B68DA
:10BDD00022449A6006E100BF0010014000140140B7
:10BDE0001F85EB51D7F8FC300022C7F8A030C7F808
:10BDF000A420D7E9288942464B46911839625B4115
:10BE00007B62D7E9082341465418494643EB0105B4
:10BE10004FF000024FF00003EB0043EA5473E200DE
:10BE200014461D464346E318C7F898304B4645EB89
:10BE30000303C7F89C30D7F8F4305B680022C7F8DA
:10BE40009030C7F894204FF000024FF00003D7E97C
:10BE5000244529468B00214643EA917321468A00F6
:10BE6000D7E92601F4F740FF02460B46604BA3FBDF
:10BE700002235B091C01D7F8FC300022C7F8883088
:10BE8000C7F88C20D7E9228942464B469118B96100
:10BE90005B41FB61D7E906234146511839614946A8
:10BEA0004B417B614FF000024FF00003D7E904AB38
:10BEB0005946CB00514643EA51735146CA001046D9
:10BEC0001946034642469B18C7F880304B460A463F
:10BED00042EB0303C7F88430D7F8F4305B680022E4
:10BEE000BB67FA674FF000024FF00003D7E91E89E5
:10BEF00049468B00414643EA917341468A00D7E99F
:10BF00002001F4F7F1FE02460B461146384BA3FB25
:10BF100001235B09642202FB03F3CB1A1B013233BA
:10BF2000334AA2FB03235B0903F0F0031C44D7F858
:10BF3000FC3000223B677A67D7E91C8942464B46B2
:10BF40009118B9605B41FB60D7E902234146511863
:10BF5000396049464B417B604FF000024FF00003CF
:10BF6000D7E900AB5946CB00514643EA51735146DD
:10BF7000CA0010461946034642469B18BB664B460C
:10BF80000A4642EB0303FB66D7F8F4305B680022F5
:10BF90003B667A664FF000024FF00003D7E918893C
:10BFA00049468B00414643EA917341468A00D7E9EE
:10BFB0001A01F4F799FE02460B460D4BA3FB021340
:10BFC0005B09642101FB03F3D31A1B013233084AD6
:10BFD000A2FB03235B0903F00F02D7F8F4301B68C0
:10BFE00022449A6000BF07F58077BD46BDE8B08F58
:10BFF0001F85EB5184B080B584B000AF786007F145
:10C000001C0080E80E0097F82130012B23D17B68BB
:10C010009B6B23F480327B689A637B68DB6823F434
:10C02000840323F040037A68D3607B68DB6823F4E1
:10C0300040127B68DA6097F82830012B05D17B68C5
:10C04000DB6843F480127B68DA60786801F032FBC9
:10C050000346FB731BE07B68DB6843F040027B68B0
:10C06000DA60786801F026FB0346FB7397F8253009
:10C07000002B06D17B689B6B43F480327B689A630C
:10C0800005E07B689B6B23F480327B689A63BB7FFF
:10C09000012B0BD17B689B6843F006027B689A609A
:10C0A0007B689B6843F020027B689A60FB7B1846A4
:10C0B0001037BD46BDE8804004B0704780B487B0FB
:10C0C00000AFF860B9601346FB71FB79022B65D1B4
:10C0D000BB68414A934206D9BB68404A934202D2A8
:10C0E0000F237B6162E0BB683C4A934206D3BB6886
:10C0F0003B4A934202D20E237B6157E0BB68384A29
:10C10000934206D3BB68374A934202D20D237B6128
:10C110004CE0BB68334A934206D3BB68324A934231
:10C1200002D80C237B6141E0BB682F4A934206D9B9
:10C13000BB682E4A934202D80B237B6136E0BB6872
:10C140002A4A934206D9BB68294A934202D80A2355
:10C150007B612BE0BB68264A934206D9BB68254A1F
:10C16000934202D209237B6120E0BB68214A9342BB
:10C1700006D3BB68204A934202D808237B6115E0AE
:10C18000BB681D4A934206D9BB681C4A934202D23F
:10C1900007237B610AE006237B6107E0FB79002B24
:10C1A00002D109237B6101E009237B61FB68DB6825
:10C1B00023F47052FB68DA60FB68DA687B699B02E3
:10C1C00003F470531A43FB68DA60002318461C37E7
:10C1D000BD465DF8047B7047BFACD800C0E1E40009
:10C1E0000024F400807306019F491A01FF2C3101DD
:10C1F0003FA44C0100366E011FABA6010048E801C8
:10C2000080B483B000AF78607B689B6843F0010224
:10C210007B689A60002318460C37BD465DF8047BA6
:10C22000704780B483B000AF78607B689B6823F070
:10C2300001027B689A60002318460C37BD465DF802
:10C24000047B704780B584B000AF78600B46FB700C
:10C250000023FB607B68DB6823F0C0427B68DA6008
:10C26000FB78012B15D17B68DB6843F000527B68BB
:10C27000DA600A20FAF72CF8FB680A33FB6078686A
:10C2800001F088F90346012B1ED0FB68C72BF0D9BB
:10C290001AE0FB78002B15D17B68DB6843F0804205
:10C2A0007B68DA600A20FAF713F8FB680A33FB6050
:10C2B000786801F06FF90346002B05D0FB68C72BA7
:10C2C000F0D901E0012305E0FB68C82B01D101236F
:10C2D00000E0002318461037BD4680BD84B080B50D
:10C2E00086B000AF786007F1240080E80E000023DC
:10C2F000FB757B68FB6000233B6109E07A683B6962
:10C3000040339B00134400225A603B6901333B6178
:10C310003B690E2BF2D997F82E30002B1CD1FB680D
:10C3200003F500635B68FA6802F5006243F00203FC
:10C3300053607B689B6B23F400127B689A637B6875
:10C340001B6843F040027B681A607B681B6843F0FF
:10C3500080027B681A6005E07B689B6B43F40012E7
:10C360007B689A63FB6803F560631A4600231360D9
:10C3700097F82930012B0DD197F82730002B04D1E5
:10C380000021786800F068F908E00121786800F081
:10C3900063F903E00321786800F05EF91021786802
:10C3A00000F0FAF80346002B01D00123FB757868F2
:10C3B00000F024F90346002B01D00123FB75FB6834
:10C3C00003F500631A4600231361FB6803F500635D
:10C3D0001A4600235361FB6803F500631A460023E5
:10C3E000D36100233B6143E03B695A01FB6813447E
:10C3F00003F510631B6803F00043B3F1004F18D13D
:10C400003B69002B0AD13B695A01FB68134403F5D1
:10C4100010631A464FF00063136013E03B695A0142
:10C42000FB68134403F510631A464FF09043136002
:10C4300008E03B695A01FB68134403F510631A4690
:10C44000002313603B695A01FB68134403F5106332
:10C450001A46002313613B695A01FB68134403F534
:10C4600010631A464FF67F3393603B6901333B619B
:10C4700097F824301A463B699342B5D300233B61B9
:10C4800043E03B695A01FB68134403F530631B68C2
:10C4900003F00043B3F1004F18D13B69002B0AD1E0
:10C4A0003B695A01FB68134403F530631A464FF0A9
:10C4B0000063136013E03B695A01FB68134403F502
:10C4C00030631A464FF09043136008E03B695A010D
:10C4D000FB68134403F530631A46002313603B697D
:10C4E0005A01FB68134403F530631A4600231361B5
:10C4F0003B695A01FB68134403F530631A464FF653
:10C500007F3393603B6901333B6197F824301A46CF
:10C510003B699342B5D3FB6803F500631B69FA6876
:10C5200002F5006223F4807313617B6800229A6134
:10C530007B686FF080425A6197F82630002B05D156
:10C540007B689B6943F010027B689A617B689A69FB
:10C55000104B13437A68936197F82A30002B05D06B
:10C560007B689B6943F008027B689A6197F82E30DC
:10C57000012B07D17B689B6943F0804343F00403A0
:10C580007A689361FB7D18461837BD46BDE8804048
:10C5900004B0704700383C8080B485B000AF78604C
:10C5A00039600023FB60FB680133FB60FB68B3F17B
:10C5B000706F01D903231BE07B681B69002BF2DA43
:10C5C0000023FB603B689B0143F020027B681A61FB
:10C5D000FB680133FB60FB68B3F1706F01D9032383
:10C5E00006E07B681B6903F02003202BF0D00023BA
:10C5F00018461437BD465DF8047B704780B485B09B
:10C6000000AF78600023FB60FB680133FB60FB68D0
:10C61000B3F1706F01D9032318E07B681B69002B0D
:10C62000F2DA0023FB607B6810221A61FB68013399
:10C63000FB60FB68B3F1706F01D9032306E07B68F0
:10C640001B6903F01003102BF0D000231846143799
:10C65000BD465DF8047B704780B485B000AF78605C
:10C660000B46FB707B68FB60FB6803F500631A6890
:10C67000FB78F96801F5006113430B60002318464D
:10C680001437BD465DF8047B704780B487B000AFB7
:10C6900078607B683B613B6903F500639B6803F04E
:10C6A0000603FB60FB68002B02D10023FB750AE048
:10C6B000FB68022B02D0FB68062B02D10223FB751C
:10C6C00001E00F23FB75FB7D18461C37BD465DF866
:10C6D000047B704780B485B000AF786039607B68B8
:10C6E000FB603B681B78BB603B685B78012B3AD1F1
:10C6F000FB6803F50063DA693B681B7803F00F03FE
:10C70000012101FA03F39BB2F96801F500611343BB
:10C71000CB61BB685A01FB68134403F510631B68C7
:10C7200003F40043002B55D1BB685A01FB68134446
:10C7300003F510631A683B689B68C3F30A013B6802
:10C740001B799B041943BB689B050B431343BA68D1
:10C750005101FA680A4402F5106243F0805343F431
:10C760000043136036E0FB6803F50063DA693B6859
:10C770001B7803F00F03012101FA03F31B04F9688E
:10C7800001F500611343CB61BB685A01FB68134498
:10C7900003F530631B6803F40043002B1AD1BB6818
:10C7A0005A01FB68134403F530631A683B689B68C1
:10C7B000C3F30A013B681B799B040B431343BA681C
:10C7C0005101FA680A4402F5306243F0805343F4A1
:10C7D00000431360002318461437BD465DF8047B00
:10C7E0007047000080B485B000AF786039607B6826
:10C7F000FB603B681B78BB603B685B78012B61D1B9
:10C80000BB685A01FB68134403F510631B6803F00F
:10C810000043B3F1004F1FD1BB685A01FB681344BA
:10C8200003F510631B68BA685101FA680A4402F5FF
:10C83000106243F000631360BB685A01FB68134445
:10C8400003F510631B68BA685101FA680A4402F5DF
:10C85000106243F080431360FB6803F50063DA6BFA
:10C860003B681B7803F00F03012101FA03F39BB22D
:10C87000DB43F96801F500611340CB63FB6803F506
:10C880000063DA693B681B7803F00F03012101FAAA
:10C8900003F39BB2DB43F96801F500611340CB6100
:10C8A000BB685A01FB68134403F510631A68BB6840
:10C8B0005901FB680B4403F510631946354B1340CF
:10C8C0000B6060E0BB685A01FB68134403F53063FA
:10C8D0001B6803F00043B3F1004F1FD1BB685A013E
:10C8E000FB68134403F530631B68BA685101FA68AA
:10C8F0000A4402F5306243F000631360BB685A01DA
:10C90000FB68134403F530631B68BA685101FA6889
:10C910000A4402F5306243F080431360FB6803F57C
:10C920000063DA6B3B681B7803F00F03012101FA07
:10C9300003F31B04DB43F96801F500611340CB638B
:10C94000FB6803F50063DA693B681B7803F00F03AB
:10C95000012101FA03F31B04DB43F96801F50061CF
:10C960001340CB61BB685A01FB68134403F5306385
:10C970001A68BB685901FB680B4403F5306319461C
:10C98000054B13400B60002318461437BD465DF875
:10C99000047B7047007833EC0078F3EF80B58AB001
:10C9A00002AFF860B9601346FB71FB68FB61BB68BE
:10C9B0001B78BB61BB685B78012B40F07F81BB6853
:10C9C0001B69002B32D1BB695A01FB69134403F583
:10C9D00010631B69BA695101FA690A4402F51062D1
:10C9E00023F0FF5323F4C0131361BB695A01FB69A1
:10C9F000134403F510631B69BA695101FA690A44CB
:10CA000002F5106243F400231361BB695A01FB690C
:10CA1000134403F510631B69BA695101FA690A44AA
:10CA200002F51062DB0CDB04136197E0BB695A016D
:10CA3000FB69134403F510631B69BA695101FA6974
:10CA40000A4402F51062DB0CDB041361BB695A0176
:10CA5000FB69134403F510631B69BA695101FA6954
:10CA60000A4402F5106223F0FF5323F4C01313614C
:10CA7000BB69002B1AD1BB681A69BB689B689A42D4
:10CA800003D9BB689A68BB681A61BB695A01FB6924
:10CA9000134403F510631B69BA695101FA690A442A
:10CAA00002F5106243F40023136144E0BB681A6985
:10CAB000BB689B6813445A1EBB689B68B2FBF3F3C8
:10CAC000FB82BB695A01FB69134403F510631A69C1
:10CAD000FB8AD904A44B0B40B9694801F9690144A8
:10CAE00001F5106113430B61BB681B79012B22D147
:10CAF000BB695A01FB69134403F510631B69BA69EA
:10CB00005101FA690A4402F5106223F0C04313612F
:10CB1000BB695A01FB69134403F510631A69FB8A68
:10CB20005B0703F0C043B9694801F969014401F5A5
:10CB3000106113430B61BB695A01FB69134403F590
:10CB400010631A69BB681B69C3F31203B969480112
:10CB5000F969014401F5106113430B61FB79012B65
:10CB60004BD1BB68DB69002B09D0BB695A01FB695B
:10CB7000134403F510631A46BB68DB695361BB6855
:10CB80001B79012B28D1FB6903F500639B6803F433
:10CB90008073002B10D1BB695A01FB69134403F564
:10CBA00010631B68BA695101FA690A4402F5106200
:10CBB00043F0005313600FE0BB695A01FB69134453
:10CBC00003F510631B68BA695101FA690A4402F55A
:10CBD000106243F080531360BB695A01FB69134430
:10CBE00003F510631B68BA695101FA690A4402F53A
:10CBF000106243F00443136066E1BB695A01FB69AC
:10CC0000134403F510631B68BA695101FA690A44B9
:10CC100002F5106243F004431360BB681B79012BDB
:10CC200015D0BB681B69002B00F04E81FB6903F532
:10CC300000635A6BBB681B7803F00F03012101FAF4
:10CC400003F3F96901F5006113434B633CE1FB69B0
:10CC500003F500639B6803F48073002B10D1BB695C
:10CC60005A01FB69134403F510631B68BA6951014B
:10CC7000FA690A4402F5106243F0005313600FE0B2
:10CC8000BB695A01FB69134403F510631B68BA6959
:10CC90005101FA690A4402F5106243F080531360AF
:10CCA000BB68D968BB681A78BB681B6998B2FB7906
:10CCB00000930346F86800F0B9F905E1BB695A0131
:10CCC000FB69134403F530631B69BA695101FA69C2
:10CCD0000A4402F53062DB0CDB041361BB695A01C4
:10CCE000FB69134403F530631B69BA695101FA69A2
:10CCF0000A4402F5306223F0FF5323F4C01313619A
:10CD0000BB69002B32D1BB681B69002B03D0BB6809
:10CD10009A68BB681A61BB689A68BB681A62BB698B
:10CD20005A01FB69134403F530631A69BB681B6A37
:10CD3000C3F31203B9694801F969014401F530618F
:10CD400013430B61BB695A01FB69134403F530635C
:10CD50001B69BA695101FA690A4402F5306243F469
:10CD60000023136162E000BF0000F81FBB681B696D
:10CD7000002B23D1BB695A01FB69134403F53063CF
:10CD80001A69BB689B68C3F31203B9694801F96962
:10CD9000014401F5306113430B61BB695A01FB6922
:10CDA000134403F530631B69BA695101FA690A44F7
:10CDB00002F5306243F40023136137E0BB681A695F
:10CDC000BB689B6813445A1EBB689B68B2FBF3F3B5
:10CDD000FB82BB689B68FA8A03FB02F2BB681A629B
:10CDE000BB695A01FB69134403F530631A69FB8A76
:10CDF000D904384B0B40B9694801F969014401F580
:10CE0000306113430B61BB695A01FB69134403F59D
:10CE100030631A69BB681B6AC3F31203B96948011E
:10CE2000F969014401F5306113430B61FB79012B72
:10CE30000DD1BB68DB68002B09D0BB68D968BB6922
:10CE40005A01FB69134403F530630A465A61BB6813
:10CE50001B79012B28D1FB6903F500639B6803F460
:10CE60008073002B10D1BB695A01FB69134403F591
:10CE700030631B68BA695101FA690A4402F53062ED
:10CE800043F0005313600FE0BB695A01FB69134480
:10CE900003F530631B68BA695101FA690A4402F567
:10CEA000306243F080531360BB695A01FB6913443D
:10CEB00003F530631B68BA695101FA690A4402F547
:10CEC000306243F004431360002318462037BD4608
:10CED00080BD00BF0000F81F80B487B000AF78604D
:10CEE00039600023FB600023FB757B683B613B6876
:10CEF0005B78012B4AD13B681B785A013B6913448C
:10CF000003F510631B6803F00043B3F1004F40F0DA
:10CF100086803B681B785A013B69134403F5106314
:10CF20001B683A68127851013A690A4402F51062A6
:10CF300043F0006313603B681B785A013B6913445C
:10CF400003F510631B683A68127851013A690A4484
:10CF500002F5106243F080431360FB680133FB600D
:10CF6000FB6842F21072934202D90123FB7556E02E
:10CF70003B681B785A013B69134403F510631B6837
:10CF800003F00043B3F1004FE7D048E03B681B7863
:10CF90005A013B69134403F530631B6803F00043F7
:10CFA000B3F1004F3BD13B681B785A013B691344F6
:10CFB00003F530631B683A68127851013A690A44F4
:10CFC00002F5306243F0006313603B681B785A013E
:10CFD0003B69134403F530631B683A6812785101CA
:10CFE0003A690A4402F5306243F080431360FB68FB
:10CFF0000133FB60FB6842F21072934202D90123B5
:10D00000FB750CE03B681B785A013B69134403F540
:10D0100030631B6803F00043B3F1004FE7D0FB7DA2
:10D0200018461C37BD465DF8047B704780B489B054
:10D0300000AFF860B96011461A460B46FB71134603
:10D04000BB80FB687B61BB68FB6197F82830002BD5
:10D0500023D1BB8803339B083B610023BB6118E0ED
:10D06000FB791A037B69134403F580531A46FB6965
:10D070001B681360FB690133FB61FB690133FB61D2
:10D08000FB690133FB61FB690133FB61BB69013360
:10D09000BB61BA693B699A42E2D300231846243740
:10D0A000BD465DF8047B704780B48BB000AFF8607C
:10D0B000B9601346FB80FB68BB61BB687B62FB8881
:10D0C0009B089BB27B61FB8803F00303FB83002377
:10D0D0003B6214E0BB6903F580531A687B6A1A60EF
:10D0E0007B6A01337B627B6A01337B627B6A01333B
:10D0F0007B627B6A01337B623B6A01333B623A6A43
:10D100007B699A42E6D3FB8B002B1ED000233B6247
:10D11000BB6903F580531A4607F1100312681A60C1
:10D120003A693B6ADBB2DB0022FA03F3DAB27B6ACC
:10D130001A703B6A01333B627B6A01337B62FB8B73
:10D14000013BFB83FB8B002BEAD17B6A18462C3713
:10D15000BD465DF8047B704780B485B000AF786051
:10D1600039607B68FB603B681B78BB603B685B7821
:10D17000012B2CD1BB685A01FB68134403F51063E3
:10D180001B68002B12DBBB68002B0FD0BB685A0159
:10D19000FB68134403F510631B68BA685101FA6811
:10D1A0000A4402F5106223F080431360BB685A0101
:10D1B000FB68134403F510631B68BA685101FA68F1
:10D1C0000A4402F5106243F4001313602BE0BB68BD
:10D1D0005A01FB68134403F530631B68002B12DB14
:10D1E000BB68002B0FD0BB685A01FB68134403F5E2
:10D1F00030631B68BA685101FA680A4402F530626C
:10D2000023F080431360BB685A01FB68134403F5A5
:10D2100030631B68BA685101FA680A4402F530624B
:10D2200043F400131360002318461437BD465DF81D
:10D23000047B704780B485B000AF786039607B684C
:10D24000FB603B681B78BB603B685B78012B28D197
:10D25000BB685A01FB68134403F510631B68BA6886
:10D260005101FA680A4402F5106223F400131360B6
:10D270003B681B79032B03D03B681B79022B38D109
:10D28000BB685A01FB68134403F510631B68BA6856
:10D290005101FA680A4402F5106243F080531360AA
:10D2A00027E0BB685A01FB68134403F530631B6831
:10D2B000BA685101FA680A4402F5306223F4001397
:10D2C00013603B681B79032B03D03B681B79022B4F
:10D2D0000FD1BB685A01FB68134403F530631B6828
:10D2E000BA685101FA680A4402F5306243F080538B
:10D2F0001360002318461437BD465DF8047B704761
:10D3000080B586B000AF78607B683B6100237B61AD
:10D3100016E07B695A013B69134403F510631A4612
:10D320004FF67F3393607B695A013B69134403F5E1
:10D3300030631A464FF67F3393607B6901337B611C
:10D340007B690E2BE5D93B6903F500631A46002380
:10D3500013613B6903F500631A46002353613B697F
:10D3600003F500631A460023D3617868FFF746F996
:10D370000346FB73FB7B002B01D0FB7B0BE01021F2
:10D380007868FFF709F90346FB73FB7B002B01D09C
:10D39000FB7B00E0FB7B18461837BD4680BD80B4A0
:10D3A00085B000AF78600B46FB707B68FB60FB6864
:10D3B00003F500631B68FA6802F5006223F4FE635C
:10D3C0001360FB6803F500631A68FB781B0103F424
:10D3D000FE63F96801F5006113430B6000231846F2
:10D3E0001437BD465DF8047B704780B485B000AF4C
:10D3F00078607B68FB60FB6803F560631B68FA6814
:10D4000002F5606223F003031360FB6803F5006319
:10D410005B68FA6802F5006223F0020353600023A0
:10D4200018461437BD465DF8047B704780B485B05C
:10D4300000AF78607B68FB60FB6803F560631B6886
:10D44000FA6802F5606223F003031360FB6803F5DA
:10D4500000635B68FA6802F5006243F00203536000
:10D46000002318461437BD465DF8047B704780B42E
:10D4700085B000AF78607B685B69FB607B689B6907
:10D48000FA681340FB60FB6818461437BD465DF828
:10D49000047B704780B485B000AF78607B68FB6028
:10D4A000FB6803F500639B69BB60FB6803F50063E1
:10D4B000DB69BA681340BB60BB681B0C18461437A5
:10D4C000BD465DF8047B704780B485B000AF7860DE
:10D4D0007B68FB60FB6803F500639B69BB60FB68CE
:10D4E00003F50063DB69BA681340BB60BB689BB29D
:10D4F00018461437BD465DF8047B704780B485B08C
:10D5000000AF78600B46FB707B68FB60FB785A01CC
:10D51000FB68134403F530639B68BB60FB6803F54D
:10D5200000635B69BA681340BB60BB681846143778
:10D53000BD465DF8047B704780B487B000AF78606B
:10D540000B46FB707B687B617B6903F500631B699D
:10D550003B617B6903F500635B6BFB60FB7803F069
:10D560000F03FA6822FA03F3DB01DBB23A691343D3
:10D570003B61FB785A017B69134403F510639B6898
:10D580003A691340BB60BB6818461C37BD465DF85E
:10D59000047B704780B483B000AF78607B685B69C0
:10D5A00003F0010318460C37BD465DF8047B704755
:10D5B00080B485B000AF78607B68FB60FB6803F5E2
:10D5C00010631B68FA6802F5106223F4FF6323F00E
:10D5D00007031360FB6803F500635B68FA6802F5F4
:10D5E000006243F480735360002318461437BD462D
:10D5F0005DF8047B7047000080B487B000AFF8602E
:10D600000B467A60FB72FB687B61FB683C3304333A
:10D610001B683B613B69264A93420AD97B6903F543
:10D6200030631B6803F00043B3F1004F01D10023C6
:10D6300037E07B6903F530631A46002313617B6989
:10D6400003F530631B697A6902F5306243F4002305
:10D6500013617B6903F530631B697A6902F53062F7
:10D6600043F0180313617B6903F530631B697A6922
:10D6700002F5306243F0C0431361FB7A012B0FD1F6
:10D680007B6903F530631A467B6853617B6903F558
:10D6900030631B687A6902F5306243F080231360BF
:10D6A000002318461C37BD465DF8047B704700BF59
:10D6B0000A30544F80B485B000AF78600023FB601F
:10D6C000FB680133FB60FB68B3F1706F01D9032382
:10D6D0001BE07B681B69002BF2DA0023FB607B6890
:10D6E0001B6943F001027B681A61FB680133FB6030
:10D6F000FB68B3F1706F01D9032306E07B681B69F7
:10D7000003F00103012BF0D0002318461437BD4667
:10D710005DF8047B7047000080B584B000AF78608E
:10D720000B46FB704FF4077005F0E8FBF860FB68F0
:10D73000002B09D17B68D3F8D4227B68B03200215A
:10D7400043F822100223D4E04FF407720021F86856
:10D7500006F0DAFC7B68D3F8D4227B68B032F96833
:10D7600043F822107B68D3F8D4227B68B03253F898
:10D7700022207B68C3F8BC227B681B7C002B38D13D
:10D780005E4B19784FF400730222786805F045FA71
:10D790005A4B1B7803F00F02796813469B00134421
:10D7A0009B000B44243301221A80554B19784FF407
:10D7B00000730222786805F030FA514B1B7803F0B1
:10D7C0000F02796813469B0013449B000B4403F53A
:10D7D000B27301221A804B4B1B7803F00F02796859
:10D7E00013469B0013449B000B44263310221A80DF
:10D7F00035E0424B197840230222786805F00DFA93
:10D800003E4B1B7803F00F02796813469B001344CC
:10D810009B000B44243301221A80394B1978402392
:10D820000222786805F0F9F9354B1B7803F00F02F6
:10D83000796813469B0013449B000B4403F5B273B5
:10D8400001221A802F4B1B7803F00F0279681346D0
:10D850009B0013449B000B44263310221A80294B53
:10D86000197808230322786805F0D7F9254B1B782F
:10D8700003F00F02796813469B0013449B000B448E
:10D88000243301221A80FB680022C3F804227B683B
:10D89000D3F8D4327A68B0339B0013445B681B68BA
:10D8A0009847FB680022C3F81422FB680022C3F8E3
:10D8B0001822FB68D3F80432002B01D1022318E0B0
:10D8C0007B681B7C002B0AD10D4B1978FB68D3F8C1
:10D8D00004224FF40073786805F08EFA08E0084BD4
:10D8E0001978FB68D3F804224023786805F084FA9D
:10D8F000002318461037BD4680BD00BF0701002039
:10D90000080100200901002080B582B000AF7860D6
:10D910000B46FB703A4B1B781946786805F0A3F963
:10D92000374B1B7803F00F02796813469B001344B2
:10D930009B000B44243300221A80324B1B7819467B
:10D94000786805F090F92F4B1B7803F00F02796887
:10D9500013469B0013449B000B4403F5B273002253
:10D960001A80294B1B781946786805F07CF9264BFC
:10D970001B7803F00F02796813469B0013449B0049
:10D980000B44243300221A801F4B1B7803F00F0234
:10D99000796813469B0013449B000B4426330022F6
:10D9A0001A807B68D3F8D4227B68B03253F82230D7
:10D9B000002B1FD07B68D3F8D4327A68B0339B0039
:10D9C00013445B685B6898477B68D3F8D4227B6814
:10D9D000B03253F82230184605F09EFA7B68D3F82F
:10D9E000D4227B68B032002143F822107B680022E9
:10D9F000C3F8BC22002318460837BD4680BD00BFCF
:10DA000007010020080100200901002080B586B030
:10DA100000AF786039607B68D3F8D4227B68B0327D
:10DA200053F822303B6100237B7300237B8100236A
:10DA3000FB753B69002B01D10323BFE03B681B78DA
:10DA400003F06003002B50D0202B40F0AF803B68E8
:10DA5000DB88002B3AD03B681B785BB2002B1BDACB
:10DA60007B68D3F8D4327A68B0339B0013445B6888
:10DA70009B683A68507839693A68D28898473B6819
:10DA8000DB88072B28BF0723FB813B69FA891946EE
:10DA9000786801F009FE90E03B685A783B6983F8AA
:10DAA00000223B68DB883F2B03D83B68DB88DAB277
:10DAB00000E040223B6983F8012239693B6993F811
:10DAC00001321A46786801F01BFE76E07B68D3F8D5
:10DAD000D4327A68B0339B0013445B689B683A6821
:10DAE000507800223968984767E03B685B780B2BD9
:10DAF00051D801A252F823F029DB0008A5DB000869
:10DB000097DB000897DB000897DB000897DB00082D
:10DB100097DB000897DB000897DB000897DB00081D
:10DB200053DB00087DDB00087B6893F89C32DBB296
:10DB3000032B07D107F10A0302221946786801F086
:10DB4000B3FD32E03968786801F031FD0323FB75DD
:10DB50002BE07B6893F89C32DBB2032B07D107F1F3
:10DB60000D0301221946786801F09EFD1DE0396819
:10DB7000786801F01CFD0323FB7516E07B6893F8C1
:10DB80009C32DBB2032B0FD03968786801F00FFDAF
:10DB90000323FB7508E03968786801F008FD03236A
:10DBA000FB7502E000BF08E000BF06E03968786856
:10DBB00001F0FDFC0323FB7500BFFB7D1846183701
:10DBC000BD4680BD80B584B000AF78600B46FB7069
:10DBD0007B68D3F8C832FB607B68D3F8D4227B68BB
:10DBE000B03253F82230002B01D1032365E07B686B
:10DBF000D3F8D4227B68B03253F82230BB60FB7874
:10DC000003F00F02796813469B0013449B000B44FA
:10DC100018331B68002B2FD0FB7803F00F027968B4
:10DC200013469B0013449B000B4418331A68FB787F
:10DC300003F00F01F8680B46DB000B449B00034424
:10DC40001C331B68B2FBF3F101FB03F3D31A002B67
:10DC500012D1FB7803F00F02796813469B0013443E
:10DC60009B000B44183300221A60F978002300222D
:10DC7000786805F0A0F81FE0BB680022C3F8142202
:10DC80007B68D3F8D4327A68B0339B0013445B6866
:10DC90001B69002B10D07B68D3F8D4327A68B0337C
:10DCA0009B0013445B681B69BA68D2F80802BA6823
:10DCB00002F50471FA789847002318461037BD46DC
:10DCC00080BD80B584B000AF78600B46FB707B6888
:10DCD000D3F8D4227B68B03253F82230FB607B68E3
:10DCE000D3F8D4227B68B03253F82230002B01D114
:10DCF00003231AE0FB781946786805F09EF802467F
:10DD0000FB68C3F80C227B68D3F8D4327A68B0334E
:10DD10009B0013445B68DB68FA68D2F80402FA6877
:10DD200002F5037211469847002318461037BD4686
:10DD300080BD80B584B000AF78607B68D3F8D42212
:10DD40007B68B03253F82230FB60FB68002B01D1B6
:10DD5000032324E07B68D3F8D4327A68B0339B0085
:10DD600013445B68002B19D0FB6893F80032FF2B3B
:10DD700014D07B68D3F8D4327A68B0339B00134454
:10DD80005B689B68FA6892F80002F968FA6892F892
:10DD900001229847FB68FF2283F8002200231846DF
:10DDA0001037BD4680BD000080B586B000AF7860FA
:10DDB0008221184800F09AFD78610121154800F091
:10DDC00095FD38618121134800F090FDF8607B6972
:10DDD000002B02D07B6910229A713B69002B06D080
:10DDE0003B69002242F040021A7100225A71FB681E
:10DDF000002B06D0FB68002242F040021A7100227C
:10DE00005A717B6843221A80024B18461837BD4668
:10DE100080BD00BFC400002080B586B000AF786030
:10DE20008221184800F062FD78610121154800F058
:10DE30005DFD38618121134800F058FDF8607B6971
:10DE4000002B02D07B6910229A713B69002B06D00F
:10DE50003B6900221A71002242F002025A71FB68EB
:10DE6000002B06D0FB6800221A71002242F0020249
:10DE70005A717B6843221A80024B18461837BD46F8
:10DE800080BD00BFC400002080B586B000AF7860C0
:10DE90008221184800F02AFD78610121154800F020
:10DEA00025FD38618121134800F020FDF8607B6971
:10DEB000002B02D07B6910229A713B69002B06D09F
:10DEC0003B69002242F040021A7100225A71FB683D
:10DED000002B06D0FB68002242F040021A7100229B
:10DEE0005A717B6843221A80024B18461837BD4688
:10DEF00080BD00BFC400002080B483B000AF786054
:10DF00007B680A221A80034B18460C37BD465DF821
:10DF1000047B70478000002080B483B000AF78603D
:10DF200039603B68002B01D1032309E07B68D3F8FB
:10DF3000D4327A68B0339B0013443A685A600023A5
:10DF400018460C37BD465DF8047B704780B487B037
:10DF500000AFF860B9607A60FB68D3F8D422FB6840
:10DF6000B03253F822307B617B69002B01D103234F
:10DF700008E07B69BA68C3F808227B697A68C3F84D
:10DF80001022002318461C37BD465DF8047B7047FD
:10DF900080B485B000AF786039607B68D3F8D42254
:10DFA0007B68B03253F82230FB60FB68002B01D154
:10DFB000032304E0FB683A68C3F8042200231846F0
:10DFC0001437BD465DF8047B7047000080B584B00F
:10DFD00000AF78607B68D3F8D4227B68B03253F806
:10DFE0002230BB600123FB73BB68002B01D10323EC
:10DFF00025E0BB68D3F81432002B1FD1BB68012287
:10E00000C3F81422104B1B7803F00F02BB68D3F83F
:10E010001012786813469B0013449B000344183386
:10E020001960094B1978BB68D3F80822BB68D3F88C
:10E030001032786804F0BFFE0023FB73FB7B1846A8
:10E040001037BD4680BD00BF0701002080B584B0F9
:10E0500000AF78607B68D3F8D4227B68B03253F885
:10E060002230FB607B68D3F8D4227B68B03253F84F
:10E070002230002B01D1032318E07B681B7C002B8E
:10E080000AD10C4B1978FB68D3F804224FF40073C3
:10E09000786804F0B1FE08E0064B1978FB68D3F805
:10E0A00004224023786804F0A7FE002318461037A6
:10E0B000BD4680BD0801002080B586B000AFF86085
:10E0C000B9601346FB71FB68002B01D103231FE0ED
:10E0D000FB680022C3F8B822FB680022C3F8C42200
:10E0E000FB680022C3F8D022BB68002B03D0FB687A
:10E0F000BA68C3F8B422FB68012283F89C22FB684B
:10E10000FA791A70F86804F0EBFC0346FB75FB7DA6
:10E1100018461837BD4680BD80B584B000AF786022
:10E12000786804F05FFD7B68012283F89C227B689D
:10E13000D3F8B832002B09D07B68D3F8B8325B68CB
:10E140007A685268D2B21146786898477B68002294
:10E15000C3F8C4227B680022C3F8B4227B68002283
:10E16000C3F8D022786804F007FD0346FB73FB7BFD
:10E1700018461037BD4680BD80B584B000AF7860CA
:10E1800039600023FB813B68002B01D1032325E08C
:10E190007B683A68C3F8B8227B68D3F8D4227B68DE
:10E1A000AE3253F82230DB6A002B0FD07B68D3F8F5
:10E1B000D4227B68AE3253F82230DB6A07F10E02BC
:10E1C0001046984702467B68C3F8D0227B68D3F894
:10E1D000D8325A1C7B68C3F8D8220023184610375F
:10E1E000BD4680BD80B582B000AF7860786804F02D
:10E1F000DEFC034618460837BD4680BD80B582B0B8
:10E2000000AF7860786804F0EDFC7B68D3F8B83232
:10E21000002B09D07B68D3F8B8325B687A68526803
:10E22000D2B2114678689847002318460837BD4691
:10E2300080BD80B483B000AF7860002318460C37EF
:10E24000BD465DF8047B704780B584B000AF786050
:10E250000B46FB700023FB737B68D3F8B832002BAE
:10E2600009D07B68D3F8B8321B68FA781146786811
:10E2700098470346FB73FB7B18461037BD4680BDAD
:10E2800080B584B000AF78600B46FB700023FB7351
:10E290007B68D3F8B8325B68FA781146786898479B
:10E2A0000346002B01D00323FB73FB7B184610377A
:10E2B000BD4680BD80B584B000AF786039607B68B2
:10E2C00003F2AA233968184601F037F97B68012266
:10E2D000C3F894227B68B3F8B0321A467B68C3F85F
:10E2E00098227B6893F8AA3203F01F03022B1AD0FE
:10E2F000022B22D8002B02D0012B0AD01DE07B6814
:10E3000003F2AA231946786800F064FB0346FB7306
:10E3100020E07B6803F2AA231946786800F0CCFB62
:10E320000346FB7316E07B6803F2AA23194678685C
:10E3300000F02EFC0346FB730CE07B6893F8AA32D6
:10E3400023F07F03DBB21946786804F0ABFC034688
:10E35000FB7300BFFB7B18461037BD4680BD80B500
:10E3600086B000AFF8600B467A60FB720023FB7545
:10E37000FB7A002B6ED1FB6803F5AA733B61FB6847
:10E38000D3F89432032B40F098803B699A683B693C
:10E39000DB689A4213D93B699A683B69DB68D21AF9
:10E3A0003B699A603B69DA683B699B68934228BF86
:10E3B00013461A467968F86801F0BFF97DE0FB68FA
:10E3C00093F8AA3203F01F03022B14D0022B1DD89E
:10E3D000002B02D0012B03D018E00023BB7518E0FE
:10E3E000FB68B3F8AE32DBB21946F86800F064FAA5
:10E3F0000346BB750DE0FB68B3F8AE32DBB21946DD
:10E40000F86800F066FA0346BB7502E00023BB75AE
:10E4100000BFBB7D002B19D1FB6893F89C32DBB2A7
:10E42000032B13D1BA7DFB68AE3253F822301B693F
:10E43000002B0BD0BA7DFB68C3F8D422BA7DFB68F1
:10E44000AE3253F822301B69F8689847F86801F03B
:10E4500085F932E0FB7A03F07F03DBB21946F868F6
:10E4600000F037FA0346BB75BB7DFF2B25D0BB7D83
:10E47000002B22D1FB6893F89C32DBB2032B17D11F
:10E48000BA7DFB68AE3253F822309B69002B0FD067
:10E49000BA7DFB68C3F8D422BA7DFB68AE3253F86C
:10E4A00022309B69FA7A1146F86898470346FB7553
:10E4B000FB7D002B01D0FB7D00E0002318461837C0
:10E4C000BD4680BD80B586B000AFF8600B467A606F
:10E4D000FB72FB7A002B6FD1FB6814333B61FB6846
:10E4E000D3F89432022B5AD13B699A683B69DB68B6
:10E4F0009A4214D93B699A683B69DB68D21A3B6936
:10E500009A603B699B681A467968F86801F0E7F8F9
:10E51000002300220021F86804F06EFC3FE03B6914
:10E52000DA683B699B689A421CD13B695A683B692F
:10E53000DB689A4216D33B695A68FB68D3F8983275
:10E540009A420FD200220021F86801F0C8F8FB6857
:10E550000022C3F89822002300220021F86804F06A
:10E560004BFC1CE0FB6893F89C32DBB2032B0FD111
:10E57000FB68D3F8B832DB68002B09D0FB680022B7
:10E58000C3F8D422FB68D3F8B832DB68F868984740
:10E590008021F86804F086FBF86801F0F2F8FB6867
:10E5A00093F8A032002B3AD0F868FFF742FEFB68E0
:10E5B000002283F8A02232E0FB7A63F07F03DBB213
:10E5C0001946F86800F085F90346FB75FB7DFF2BC3
:10E5D00025D0FB7D002B22D1FB6893F89C32DBB267
:10E5E000032B1CD1FA7DFB68AE3253F822305B69F5
:10E5F000002B14D0FA7DFB68C3F8D422FA7DFB68A7
:10E60000AE3253F822305B69FA7A1146F8689847BF
:10E610000346BB75BB7D002B01D0BB7D00E0002312
:10E6200018461837BD4680BD80B584B000AF78600D
:10E630000023FB737B68012283F89C227B68002205
:10E64000C3F894227B6800225A607B680022C3F8DA
:10E65000A4227B68002283F8A0227B68D3F8B8321A
:10E66000002B14D07B68D3F8B8325B68002B0ED037
:10E670007B68D3F8B8325B687A685268D2B21146C8
:10E68000786898470346002B01D00323FB7340238F
:10E6900000220021786804F0C0FA7B680122A3F808
:10E6A00064217B684022C3F860214023002280213E
:10E6B000786804F0B2FA7B6801229A847B68402271
:10E6C0001A62FB7B18461037BD4680BD80B483B00C
:10E6D00000AF78600B46FB707B68FA781A740023F1
:10E6E00018460C37BD465DF8047B704780B483B094
:10E6F00000AF78607B6893F89C32DBB2042B06D0C5
:10E700007B6893F89C32DAB27B6883F89D227B6841
:10E71000042283F89C22002318460C37BD465DF87E
:10E72000047B704780B483B000AF78607B6893F857
:10E730009C32DBB2042B06D17B6893F89D32DAB2AF
:10E740007B6883F89C22002318460C37BD465DF891
:10E75000047B704780B582B000AF78607B6893F827
:10E760009C32DBB2032B10D17B68D3F8B832002B7C
:10E770000BD07B68D3F8B832DB69002B05D07B68FF
:10E78000D3F8B832DB697868984700231846083711
:10E79000BD4680BD80B582B000AF78600B46FB708F
:10E7A0007B68D3F8D4227B68AE3253F82230002B3A
:10E7B00001D103231CE07B6893F89C32DBB2032B6E
:10E7C00015D17B68D3F8D4227B68AE3253F822305F
:10E7D0001B6A002B0BD07B68D3F8D4227B68AE3247
:10E7E00053F822301B6AFA7811467868984700235C
:10E7F00018460837BD4680BD80B582B000AF78604E
:10E800000B46FB707B68D3F8D4227B68AE3253F89A
:10E810002230002B01D103231CE07B6893F89C324B
:10E82000DBB2032B15D17B68D3F8D4227B68AE32E0
:10E8300053F822305B6A002B0BD07B68D3F8D422CC
:10E840007B68AE3253F822305B6AFA7811467868FA
:10E850009847002318460837BD4680BD80B483B072
:10E8600000AF7860002318460C37BD465DF8047B86
:10E87000704780B584B000AF78600023FB737B687D
:10E88000012283F89C227B68D3F8B832002B0ED08B
:10E890007B68D3F8B8325B687A685268D2B21146A6
:10E8A000786898470346002B01D00323FB73FB7B5A
:10E8B00018461037BD4680BD80B483B000AF786085
:10E8C0000B46FB70002318460C37BD465DF8047BF1
:10E8D000704780B483B000AF78600B46FB700023B4
:10E8E00018460C37BD465DF8047B704780B586B08E
:10E8F00000AF78600B46FB707B687B617B68FB60D8
:10E9000000233B61FB685B889BB2FA6812789342F4
:10E910001FD9FB681B787B8113E007F10A031946B6
:10E92000786900F01BF878617B695B78052B08D16A
:10E930007B693B613B699B78FA789A4208D0002357
:10E940003B61FB685B889AB27B899A42E5D800E01C
:10E9500000BF3B6918461837BD4680BD80B485B0FE
:10E9600000AF786039607B68FB603B681B88FA68A1
:10E97000127813449AB23B681A80FB681B781A46D7
:10E980007B681344FB60FB6818461437BD465DF88E
:10E99000047B704780B487B000AF78607B687B6190
:10E9A0007B691B787B827B6901337B617B691B7888
:10E9B0003B82B7F910301B021AB2B7F91230134379
:10E9C0001BB2FB81FB8918461C37BD465DF8047BF2
:10E9D0007047000080B584B000AF786039600023D4
:10E9E000FB733B681B7803F06003402B05D0402B82
:10E9F00057D8002B0FD0202B53D17B68D3F8D422CB
:10EA00007B68AE3253F822309B6839687868984743
:10EA10000346FB734AE03B685B78092B3BD801A2B5
:10EA200052F823F079EA00088DEA000897EA000816
:10EA300083EA000897EA000857EA00084DEA000850
:10EA400097EA00086FEA000861EA00083968786808
:10EA500000F03CFA24E03968786800F0CBFB1FE056
:10EA60003968786800F00AFC0346FB7318E03968DF
:10EA7000786800F0ADFC13E03968786800F0DEFCDF
:10EA80000EE03968786800F00DFD09E039687868B3
:10EA900000F031FD04E03968786800F088FD00BFBF
:10EAA00004E03968786800F082FD00BFFB7B1846FF
:10EAB0001037BD4680BD00BF80B584B000AF786020
:10EAC00039600023FB733B681B7803F06003402B25
:10EAD00005D0402B52D8002B01D0202B4ED17B6883
:10EAE00093F89C32DBB2013B022B40D83B689B88F9
:10EAF000DBB2012B36D83B689B88DBB219467868BD
:10EB0000FFF7DAFE0346BB73BB7BFF2B1DD0BB7B3D
:10EB1000002B1AD1BA7B7B68AE3253F822309B6847
:10EB2000002B0FD0BA7B7B68C3F8D422BA7B7B68FA
:10EB3000AE3253F822309B683968786898470346AC
:10EB4000FB7304E00323FB7301E00323FB733B68C7
:10EB5000DB88002B10D1FB7B002B0DD1786800F0F7
:10EB6000FDFD09E03968786800F021FD04E03968AE
:10EB7000786800F01CFD00E000BF04E039687868A8
:10EB800000F015FD00BFFB7B18461037BD4680BD69
:10EB900080B584B000AF786039600023FB733B68B8
:10EBA0009B88BB733B681B7803F06003402B07D046
:10EBB000402B00F27F81002B2AD0202B40F07A815D
:10EBC000BB7B19467868FFF784FE03467B737B7B2B
:10EBD000FF2B00F074817B7B002B40F070817A7BEF
:10EBE0007B68C3F8D4227A7B7B68AE3253F822303C
:10EBF0009B68002B00F063817A7B7B68AE3253F810
:10EC000022309B683968786898470346FB7356E161
:10EC10003B685B78032B08D0032B00F34581002B66
:10EC200000F09B80012B3CD03EE17B6893F89C3246
:10EC3000DBB2022B02D0032B16D02CE0BB7B002BC7
:10EC40000DD0BB7B802B0AD0BB7B1946786804F0C3
:10EC500029F88021786804F025F800BF20E03968A1
:10EC6000786800F0A4FC1BE03B685B88002B0ED1A9
:10EC7000BB7B002B0BD0BB7B802B08D03B68DB8899
:10EC8000002B04D1BB7B1946786804F00BF8786838
:10EC900000F064FD04E03968786800F088FC00BF8B
:10ECA00007E17B6893F89C32DBB2022B02D0032B86
:10ECB00016D04BE0BB7B002B0DD0BB7B802B0AD04A
:10ECC000BB7B1946786803F0EDFF8021786803F07C
:10ECD000E9FF00BF40E03968786800F068FC3BE07D
:10ECE0003B685B88002B36D1BB7B03F07F03002B96
:10ECF00004D0BB7B1946786803F0F3FF786800F016
:10ED00002DFDBB7B19467868FFF7E3FD03467B7357
:10ED10007B7BFF2B1FD07B7B002B1CD17A7B7B68FE
:10ED2000C3F8D4227A7B7B68AE3253F822309B68DA
:10ED3000002B10D07A7B7B68AE3253F822309B6870
:10ED40003968786898470346FB7304E03968786847
:10ED500000F02DFC00E000BFABE07B6893F89C3234
:10ED6000DBB2022B02D0032B32D097E0BB7B002B0F
:10ED700007D0BB7B802B04D03968786800F017FC83
:10ED800091E097F90E30002B0BDABB7B03F07F028A
:10ED900013469B0013449B0010337A6813440433DA
:10EDA0000BE0BB7B03F07F0213469B0013449B00E8
:10EDB00003F5A8737A6813440433BB60BB68002270
:10EDC0001A60BB6802221946786800F06DFC6AE0A0
:10EDD00097F90E30002B11DABB7B03F00F02796834
:10EDE00013469B0013449B000B4424331B88002BC9
:10EDF00017D13968786800F0DAFB54E0BB7B03F088
:10EE00000F02796813469B0013449B000B4403F5E3
:10EE1000B2731B88002B04D13968786800F0C7FBF7
:10EE200041E097F90E30002B0BDABB7B03F07F0239
:10EE300013469B0013449B0010337A681344043339
:10EE40000BE0BB7B03F07F0213469B0013449B0047
:10EE500003F5A8737A6813440433BB60BB7B002BB3
:10EE600002D0BB7B802B03D1BB6800221A600EE06E
:10EE7000BB7B1946786803F053FF0346002B03D091
:10EE8000BB6801221A6002E0BB6800221A60BB68FE
:10EE900002221946786800F007FC04E039687868B7
:10EEA00000F085FB00BF04E03968786800F07FFB64
:10EEB00000BF05E03968786800F079FB00E000BF2A
:10EEC000FB7B18461037BD4680BD000080B584B07E
:10EED00000AF7860396000233B810023FB60002392
:10EEE000FB723B685B881B0A9BB2013B0E2B00F256
:10EEF000528101A252F823F069EF000881EF000867
:10EF0000C1EF000897F1000897F1000837F10008F9
:10EF100063F1000897F1000897F1000897F10008E5
:10EF200097F1000897F1000897F1000897F10008A1
:10EF300035EF00087B68D3F8B432DB69002B0BD0C7
:10EF40007B68D3F8B432DB697A68127C07F1080178
:10EF500010469847F86026E13968786800F027FB8A
:10EF6000FB7A0133FB721EE17B68D3F8B4321B6875
:10EF70007A68127C07F1080110469847F86012E1A0
:10EF80007B681B7C002B0DD17B68D3F8B8329B6A61
:10EF900007F1080210469847F860FB680133022227
:10EFA0001A7000E17B68D3F8B832DB6A07F1080217
:10EFB00010469847F860FB68013302221A70F2E0AD
:10EFC0003B685B88DBB2052B00F2AC8001A252F8F3
:10EFD00023F000BFEDEF000821F0000855F0000815
:10EFE00089F00008BDF00008F1F000087B68D3F854
:10EFF000B4325B68002B0BD07B68D3F8B4325B680B
:10F000007A68127C07F1080110469847F86091E091
:10F010003968786800F0CBFAFB7A0133FB7289E03B
:10F020007B68D3F8B4329B68002B0BD07B68D3F895
:10F03000B4329B687A68127C07F108011046984741
:10F04000F86077E03968786800F0B1FAFB7A01334C
:10F05000FB726FE07B68D3F8B432DB68002B0BD017
:10F060007B68D3F8B432DB687A68127C07F1080158
:10F0700010469847F8605DE03968786800F097FAC4
:10F08000FB7A0133FB7255E07B68D3F8B4321B691D
:10F09000002B0BD07B68D3F8B4321B697A68127CE2
:10F0A00007F1080110469847F86043E0396878682E
:10F0B00000F07DFAFB7A0133FB723BE07B68D3F80A
:10F0C000B4325B69002B0BD07B68D3F8B4325B6938
:10F0D0007A68127C07F1080110469847F86029E029
:10F0E0003968786800F063FAFB7A0133FB7221E03B
:10F0F0007B68D3F8B4329B69002B0BD07B68D3F8C4
:10F10000B4329B697A68127C07F10801104698476F
:10F11000F8600FE03968786800F049FAFB7A01334B
:10F12000FB7207E03968786800F041FAFB7A013336
:10F13000FB7200BF37E07B681B7C002B09D17B682A
:10F14000D3F8B8325B6B07F1080210469847F860B5
:10F1500029E03968786800F02AFAFB7A0133FB72FB
:10F1600021E07B681B7C002B0DD17B68D3F8B83283
:10F170001B6B07F1080210469847F860FB680133E3
:10F1800007221A700FE03968786800F010FAFB7AED
:10F190000133FB7207E03968786800F008FAFB7AFF
:10F1A0000133FB7200BFFB7A002B1ED13B68DB886A
:10F1B000002B16D03B89002B0ED03B68DA883B89A8
:10F1C000934228BF13469BB23B813B891A46F9689C
:10F1D000786800F069FA09E03968786800F0E7F9C2
:10F1E00004E0786800F0BAFA00E000BF1037BD46CE
:10F1F00080BD00BF80B584B000AF786039603B68E7
:10F200009B88002B31D13B68DB88002B2DD13B68DC
:10F210005B887F2B29D83B685B88DBB203F07F03D8
:10F22000FB737B6893F89C32DBB2032B04D1396803
:10F23000786800F0BCF91DE07B68FA7B83F89E22B9
:10F24000FB7B1946786803F097FD786800F086FA32
:10F25000FB7B002B04D07B68022283F89C2209E010
:10F260007B68012283F89C2204E03968786800F00A
:10F270009EF900BF00BF1037BD4680BD80B584B089
:10F2800000AF786039600023FB733B685B88DAB2BB
:10F290004E4B1A704D4B1B78012B05D93968786895
:10F2A00000F085F903238CE07B6893F89C32DBB295
:10F2B000022B02D0032B29D075E0444B1B78002B86
:10F2C00020D0424B1B781A467B685A603F4B1B7814
:10F2D00019467868FEF7B8FF0346FB73FB7B002BEB
:10F2E00008D03968786800F062F97B68022283F8F8
:10F2F0009C2265E0786800F031FA7B68032283F88D
:10F300009C225DE0786800F029FA59E02F4B1B78C9
:10F31000002B12D17B68022283F89C222B4B1B7896
:10F320001A467B685A60294B1B7819467868FEF7A5
:10F33000A7FF786800F012FA42E0244B1B781A46C7
:10F340007B685B689A422AD07B685B68DBB21946AF
:10F350007868FEF795FF1D4B1B781A467B685A604C
:10F360001A4B1B7819467868FEF76EFF0346FB734D
:10F37000FB7B002B0FD03968786800F018F97B68A8
:10F380005B68DBB219467868FEF77AFF7B68022279
:10F3900083F89C2214E0786800F0E0F910E07868C7
:10F3A00000F0DCF90CE03968786800F000F9074BF0
:10F3B0001B7819467868FEF763FF0323FB7300BFD1
:10F3C000FB7B18461037BD4680BD00BF20070020DC
:10F3D00080B582B000AF786039603B68DB88012B74
:10F3E00004D03968786800F0E2F823E07B6893F88D
:10F3F0009C32DBB2022B02DC002B03DC15E0032B7A
:10F400000BD012E07B6800229A607B6808330122EF
:10F410001946786800F048F90CE07B680433012253
:10F420001946786800F040F904E03968786800F01F
:10F43000BEF800BF00BF0837BD4680BD80B582B0B2
:10F4400000AF786039607B6893F89C32DBB2013B97
:10F45000022B1ED83B68DB88022B04D03968786801
:10F4600000F0A5F81AE07B680122DA607B68D3F827
:10F47000A432002B05D07B68DB6843F002027B6876
:10F48000DA607B680C3302221946786800F00CF9C8
:10F4900004E03968786800F08AF800BF00BF0837D8
:10F4A000BD4680BD80B582B000AF786039603B68F2
:10F4B0005B88012B07D17B680122C3F8A4227868FE
:10F4C00000F04CF913E03B685B88022B0BD13B68E2
:10F4D0009B881B0A9BB2DAB27B6883F8A02278680B
:10F4E00000F03CF903E03968786800F060F800BF8C
:10F4F0000837BD4680BD80B582B000AF7860396006
:10F500007B6893F89C32DBB2013B022B0BD83B6843
:10F510005B88012B0CD17B680022C3F8A422786899
:10F5200000F01CF904E03968786800F040F800E069
:10F5300000BF00BF0837BD4680BD80B584B000AFB6
:10F54000786039603B68FB60FB681A787B681A70EA
:10F55000FB680133FB60FB681A787B685A70FB68B4
:10F560000133FB60F868FFF715FA03461A467B681B
:10F570005A80FB680133FB60FB680133FB60F8686D
:10F58000FFF708FA03461A467B689A80FB68013346
:10F59000FB60FB680133FB60F868FFF7FBF903468B
:10F5A0001A467B68DA8000BF1037BD4680BD80B543
:10F5B00082B000AF786039608021786803F072FB18
:10F5C0000021786803F06EFB00BF0837BD4680BDA0
:10F5D00080B586B000AFF860B9607A600023FB7533
:10F5E000FB68002B42D0FB683B61386900F042F8B1
:10F5F000034601335B00B3F5007F08D8386900F09B
:10F6000039F8034601339BB25B009AB201E04FF434
:10F6100000727B681A80FB7DBA6813447A6812789E
:10F620001A70FB7D0133FB75FB7DBA68134403221E
:10F630001A70FB7D0133FB7513E0FB7DBA68134440
:10F640003A6912781A703B6901333B61FB7D0133E3
:10F65000FB75FB7DBA68134400221A70FB7D0133F1
:10F66000FB753B691B78002BE7D100E000BF183722
:10F67000BD4680BD80B485B000AF78600023FB73C9
:10F680007B68BB6005E0FB7B0133FB73BB68013328
:10F69000BB60BB681B78002BF5D1FB7B1846143789
:10F6A000BD465DF8047B704780B584B000AFF8605C
:10F6B000B9607A60FB680222C3F89422FB687A681A
:10F6C0009A61FB687A68DA617B68BA680021F86839
:10F6D00003F071FB002318461037BD4680BD80B58E
:10F6E00084B000AFF860B9607A607B68BA680021C6
:10F6F000F86803F060FB002318461037BD4680BD54
:10F7000080B584B000AFF860B9607A60FB6803220E
:10F71000C3F89422FB687A68C3F85821FB687A68BA
:10F72000C3F85C217B68BA680021F86803F064FBC9
:10F73000002318461037BD4680BD80B584B000AFA9
:10F74000F860B9607A607B68BA680021F86803F0F5
:10F7500053FB002318461037BD4680BD80B582B0EC
:10F7600000AF78607B680422C3F894220023002253
:10F770000021786803F01FFB002318460837BD46B8
:10F7800080BD80B582B000AF78607B680522C3F889
:10F790009422002300220021786803F02DFB00232F
:10F7A00018460837BD4680BD80B483B000AF03461D
:10F7B0003960FB7197F90730002B0ADB3B68DAB23E
:10F7C0000C4997F907301201D2B20B4483F8002399
:10F7D0000AE03B68DAB20849FB7903F00F03043B07
:10F7E0001201D2B20B441A7600BF0C37BD465DF849
:10F7F000047B704700E100E000ED00E080B500AF61
:10F80000054B1B6801F046FD0346012B01D002F0B9
:10F810003BFB00BF80BD00BF10E000E080B500AF43
:10F8200000216FF00400FFF7BFFF00BF80BD0000A4
:10F8300080B483B000AFEFF305833B603B68002BDF
:10F8400003D06FF005037B600CE00A4B1B68002BB4
:10F8500005D1084B01221A6000237B6002E04FF0C3
:10F86000FF337B607B6818460C37BD465DF8047B30
:10F87000704700BF2407002080B582B000AFEFF3CF
:10F8800005833B603B68002B03D06FF005037B6072
:10F8900010E00B4B1B68012B09D1FFF7BFFF084B92
:10F8A00002221A6001F092F800237B6002E04FF020
:10F8B000FF337B607B6818460837BD4680BD00BFBC
:10F8C0002407002080B58EB004AFF860B9607A607C
:10F8D00000233B61EFF305837B617B69002B7ED1C5
:10F8E000FB68002B7BD080233B621823FB61002345
:10F8F0007B624FF0FF33BB617B68002B45D07B6898
:10F900001B68002B02D07B681B687B627B689B694D
:10F91000002B02D07B689B69FB61FB69002B08D040
:10F92000FB69382B05D87B685B6803F00103002B6B
:10F9300001D0002354E07B685B69002B03D07B6817
:10F940005B699B083B627B689B68002B0ED07B68E1
:10F95000DB68A72B0AD97B681B69002B06D07B6864
:10F960005B69002B02D00123BB6110E07B689B68C0
:10F97000002B0CD17B68DB68002B08D17B681B69EE
:10F98000002B04D10023BB6101E00023BB61BB69F4
:10F99000012B10D17B681B697A68926802920193EF
:10F9A000FB690093BB683A6A796AF86800F01AFE4E
:10F9B00003463B6113E0BB69002B10D13B6A9AB24E
:10F9C00007F110030193FB690093BB68796AF8683B
:10F9D00000F068FE0346012B01D000233B613B6928
:10F9E00018462837BD4680BD80B584B000AF78602A
:10F9F000EFF30583BB60BB68002B03D06FF00503FA
:10FA0000FB6007E00023FB607B68002B02D0786876
:10FA100000F0A6FFFB6818461037BD4680BD000009
:10FA200080B485B000AFF860B9607A60FB68074ABF
:10FA30001A60BB68064A1A607B6880221A6000BFA1
:10FA40001437BD465DF8047B704700BF28070020CF
:10FA5000D007002080B485B000AFF860B9607A604C
:10FA6000FB68074A1A60BB68064A1A607B684FF455
:10FA700080721A6000BF1437BD465DF8047B704782
:10FA8000D0090020780A002080B483B000AF7860ED
:10FA90007B6803F108027B685A607B684FF0FF3295
:10FAA0009A607B6803F108027B68DA607B6803F187
:10FAB00008027B681A617B6800221A6000BF0C375D
:10FAC000BD465DF8047B704780B483B000AF7860BA
:10FAD0007B6800221A6100BF0C37BD465DF8047BCD
:10FAE000704780B485B000AF786039607B685B6830
:10FAF000FB603B68FA685A60FB689A683B689A60EA
:10FB0000FB689B683A685A60FB683A689A603B6891
:10FB10007A681A617B681B685A1C7B681A6000BF90
:10FB20001437BD465DF8047B704780B485B000AFE4
:10FB3000786039603B681B68BB60BB68B3F1FF3F0E
:10FB400003D17B681B69FB600CE07B680833FB60BA
:10FB500002E0FB685B68FB60FB685B681B68BA6877
:10FB60009A42F6D2FB685A683B685A603B685B6809
:10FB70003A689A603B68FA689A60FB683A685A602B
:10FB80003B687A681A617B681B685A1C7B681A603C
:10FB900000BF1437BD465DF8047B704780B485B064
:10FBA00000AF78607B681B69FB607B685B687A6884
:10FBB00092689A607B689B687A6852685A60FB68B2
:10FBC0005B687A689A4203D17B689A68FB685A60DE
:10FBD0007B6800221A61FB681B685A1EFB681A606A
:10FBE000FB681B6818461437BD465DF8047B7047F8
:10FBF00080B584B000AF786039607B68FB60FB68DB
:10FC0000002B0BD14FF0500383F31188BFF36F8F9C
:10FC1000BFF34F8FBB6000BF00BFFDE702F0A4F849
:10FC2000FB681A68FB68DB6BF968096C01FB03F37E
:10FC30001A44FB689A60FB6800229A63FB681A68A2
:10FC4000FB685A60FB681A68FB68DB6B013BF9686C
:10FC5000096C01FB03F31A44FB68DA60FB68FF22BE
:10FC600083F84420FB68FF2283F845203B68002B83
:10FC700014D1FB681B69002B1AD0FB68103318469F
:10FC800001F042F90346002B12D00D4B4FF0805289
:10FC90001A60BFF34F8FBFF36F8F09E0FB6810331B
:10FCA0001846FFF7F1FEFB6824331846FFF7ECFE19
:10FCB00002F08CF8012318461037BD4680BD00BF06
:10FCC00004ED00E080B58EB002AFF860B9607A60F4
:10FCD0003B60FB68002B0BD14FF0500383F311887E
:10FCE000BFF36F8FBFF34F8FBB6200BF00BFFDE755
:10FCF0003B68002B0BD14FF0500383F31188BFF307
:10FD00006F8FBFF34F8F7B6200BF00BFFDE77B6843
:10FD1000002B02D0BB68002B01D0012300E00023A0
:10FD2000002B0BD14FF0500383F31188BFF36F8F7B
:10FD3000BFF34F8F3B6200BF00BFFDE77B68002B26
:10FD400002D1BB68002B01D1012300E00023002B6E
:10FD50000BD14FF0500383F31188BFF36F8FBFF3C4
:10FD60004F8FFB6100BF00BFFDE750237B617B69C4
:10FD7000502B0BD04FF0500383F31188BFF36F8FDC
:10FD8000BFF34F8FBB6100BF00BFFDE77B693B68DE
:10FD9000FB62FB6A002B0DD0FB6A012283F8462030
:10FDA00097F83820FB6A009313467A68B968F868B8
:10FDB00000F005F8FB6A18463037BD4680BD80B5B7
:10FDC00084B000AFF860B9607A60FB70BB68002B4C
:10FDD00003D1BB69BA691A6002E0BB697A681A602C
:10FDE000BB69FA68DA63BB69BA681A640121B86949
:10FDF000FFF7FEFEBB69FA7883F84C2000BF10378E
:10FE0000BD4680BD80B58EB000AFF860B9607A6045
:10FE10003B6000237B63FB683B633B6B002B0BD198
:10FE20004FF0500383F31188BFF36F8FBFF34F8FF1
:10FE3000BB6200BF00BFFDE7BB68002B03D13B6B7B
:10FE40001B6C002B01D1012300E00023002B0BD100
:10FE50004FF0500383F31188BFF36F8FBFF34F8FC1
:10FE60007B6200BF00BFFDE73B68022B03D13B6B09
:10FE7000DB6B012B01D1012300E00023002B0BD110
:10FE80004FF0500383F31188BFF36F8FBFF34F8F91
:10FE90003B6200BF00BFFDE701F0FCF90346002B09
:10FEA00002D17B68002B01D1012300E00023002B4D
:10FEB0000BD14FF0500383F31188BFF36F8FBFF363
:10FEC0004F8FFB6100BF00BFFDE701F04DFF3B6BB3
:10FED0009A6B3B6BDB6B9A4202D33B68022B29D1B6
:10FEE0003A68B968386B00F00FFAF8623B6B5B6AEE
:10FEF000002B10D03B6B2433184601F005F8034665
:10FF0000002B13D03F4B4FF080521A60BFF34F8F3E
:10FF1000BFF36F8F0AE0FB6A002B07D0394B4FF01D
:10FF200080521A60BFF34F8FBFF36F8F01F04EFF07
:10FF3000012363E07B68002B03D101F047FF00231E
:10FF40005CE07B6B002B06D107F11403184601F02F
:10FF50003FF801237B6301F039FF00F0A7FD01F0BA
:10FF600003FF3B6B93F844305BB2B3F1FF3F03D127
:10FF70003B6B002283F844203B6B93F845305BB227
:10FF8000B3F1FF3F03D13B6B002283F8452001F022
:10FF90001DFF3A1D07F114031146184601F02EF813
:10FFA0000346002B24D1386B00F0A6FA0346002B41
:10FFB00018D03B6B10337A681146184600F052FF98
:10FFC000386B00F031FA00F07FFD0346002B7FF420
:10FFD0007CAF0C4B4FF080521A60BFF34F8FBFF3D2
:10FFE0006F8F72E7386B00F01FFA00F06DFD6CE761
:10FFF000386B00F019FA00F067FD00231846383717
:020000040801F1
:10000000BD4680BD04ED00E080B590B000AFF86063
:10001000B9607A603B60FB68BB63BB6B002B0BD1A4
:100020004FF0500383F31188BFF36F8FBFF34F8FEF
:10003000BB6200BF00BFFDE7BB68002B03D1BB6BF9
:100040001B6C002B01D1012300E00023002B0BD1FE
:100050004FF0500383F31188BFF36F8FBFF34F8FBF
:100060007B6200BF00BFFDE73B68022B03D1BB6B87
:10007000DB6B012B01D1012300E00023002B0BD10E
:100080004FF0500383F31188BFF36F8FBFF34F8F8F
:100090003B6200BF00BFFDE701F046FFEFF31182B6
:1000A0004FF0500383F31188BFF36F8FBFF34F8F6F
:1000B000FA61BB61FB697B63BB6B9A6BBB6BDB6BF0
:1000C0009A4202D33B68022B2FD1BB6B93F8453089
:1000D00087F83330BB6B9B6BFB623A68B968B86BCF
:1000E00000F012F997F93330B3F1FF3F12D1BB6B37
:1000F0005B6A002B16D0BB6B2433184600F004FF5C
:100100000346002B0ED07B68002B0BD07B680122AE
:100110001A6007E097F833300133DBB25AB2BB6B99
:1001200083F845200123FB6301E00023FB637B6B25
:100130007B617B6983F3118800BFFB6B18464037F6
:10014000BD4680BD80B58CB000AFF860B9607A6004
:100150000023FB62FB68BB62BB6A002B0BD14FF034
:10016000500383F31188BFF36F8FBFF34F8F3B6250
:1001700000BF00BFFDE7BB68002B03D1BB6A1B6C4F
:10018000002B01D1012300E00023002B0BD14FF005
:10019000500383F31188BFF36F8FBFF34F8FFB6161
:1001A00000BF00BFFDE701F075F80346002B02D148
:1001B0007B68002B01D1012300E00023002B0BD131
:1001C0004FF0500383F31188BFF36F8FBFF34F8F4E
:1001D000BB6100BF00BFFDE701F0C6FDBB6A9B6BC2
:1001E0007B627B6A002B1FD0B968B86A00F0F6F812
:1001F0007B6A5A1EBB6A9A63BB6A1B69002B0FD0CD
:10020000BB6A1033184600F07FFE0346002B07D070
:100210003C4B4FF080521A60BFF34F8FBFF36F8F8C
:1002200001F0D4FD012369E07B68002B03D101F0CC
:10023000CDFD002362E0FB6A002B06D107F110031D
:10024000184600F0C5FE0123FB6201F0BFFD00F07F
:100250002DFC01F089FDBB6A93F844305BB2B3F129
:10026000FF3F03D1BB6A002283F84420BB6A93F8A6
:1002700045305BB2B3F1FF3F03D1BB6A002283F884
:10028000452001F0A3FD3A1D07F110031146184661
:1002900000F0B4FE0346002B23D1B86A00F016F933
:1002A0000346002B17D0BB6A24337A6811461846E0
:1002B00000F0D8FDB86A00F0B7F800F005FC03467E
:1002C000002B89D10F4B4FF080521A60BFF34F8F34
:1002D000BFF36F8F80E7B86A00F0A6F800F0F4FB78
:1002E0007AE7B86A00F0A0F800F0EEFBB86A00F018
:1002F000EDF80346002B3FF46FAF0023184630376C
:10030000BD4680BD04ED00E080B586B000AFF8606A
:10031000B9607A6000237B61FB689B6B3B61FB6883
:100320001B6C002B0DD1FB681B68002B4DD1FB68AB
:100330009B68184600F0CCFF7861FB6800229A6049
:1003400043E07B68002B19D1FB685868FB681B6C85
:100350001A46B96804F002F8FB685A68FB681B6C1F
:100360001A44FB685A60FB685A68FB689B689A42AB
:100370002BD3FB681A68FB685A6026E0FB68D868D4
:10038000FB681B6C1A46B96803F0E8FFFB68DA6883
:10039000FB681B6C5B421A44FB68DA60FB68DA6836
:1003A000FB681B689A4207D2FB689A68FB681B6C63
:1003B0005B421A44FB68DA607B68022B05D13B691B
:1003C000002B02D03B69013B3B613B695A1CFB6837
:1003D0009A637B6918461837BD4680BD80B582B0E8
:1003E00000AF786039607B681B6C002B18D07B688D
:1003F000DA687B681B6C1A447B68DA607B68DA68B1
:100400007B689B689A4203D37B681A687B68DA60D2
:100410007B68D9687B681B6C1A46386803F09EFFBE
:1004200000BF0837BD4680BD80B584B000AF78609E
:1004300001F09AFC7B6893F84530FB7311E07B6810
:100440005B6A002B12D07B682433184600F05CFDF9
:100450000346002B01D000F035FEFB7B013BDBB2F5
:10046000FB7397F90F30002BE9DC00E000BF7B68DD
:10047000FF2283F8452001F0A9FC01F075FC7B68A0
:1004800093F84430BB7311E07B681B69002B12D0DA
:100490007B681033184600F037FD0346002B01D06F
:1004A00000F010FEBB7B013BDBB2BB7397F90E3053
:1004B000002BE9DC00E000BF7B68FF2283F84420CA
:1004C00001F084FC00BF1037BD4680BD80B584B00C
:1004D00000AF786001F048FC7B689B6B002B02D179
:1004E0000123FB6001E00023FB6001F06FFCFB686F
:1004F00018461037BD4680BD80B584B000AF786027
:1005000001F032FC7B689A6B7B68DB6B9A4202D10C
:100510000123FB6001E00023FB6001F057FCFB6856
:1005200018461037BD4680BD80B485B000AF7860F6
:1005300039600023FB6014E00F4AFB6852F8333047
:10054000002B0BD10C49FB683A6841F833200A4A6A
:10055000FB68DB0013447A685A6006E0FB680133ED
:10056000FB60FB68072BE7D900BF00BF1437BD460F
:100570005DF8047B704700BF780E002080B586B020
:1005800000AFF860B9607A60FB687B6101F0ECFB5A
:100590007B6993F844305BB2B3F1FF3F03D17B69D1
:1005A000002283F844207B6993F845305BB2B3F1B5
:1005B000FF3F03D17B69002283F8452001F006FC50
:1005C0007B699B6B002B06D17B6924337A68B96801
:1005D000184600F06DFC7869FFF726FF00BF18375A
:1005E000BD4680BD80B58EB004AFF860B9607A605A
:1005F0003B607B6B002B0BD14FF0500383F31188D2
:10060000BFF36F8FBFF34F8F3B6200BF00BFFDE7AB
:10061000BB6B002B0BD14FF0500383F31188BFF35A
:100620006F8FBFF34F8FFB6100BF00BFFDE7A823B3
:100630003B613B69A82B0BD04FF0500383F311882B
:10064000BFF36F8FBFF34F8FBB6100BF00BFFDE7EC
:100650003B69BB6B002B1ED07B6B002B1BD0BB6B95
:100660007B627B6A7A6B1A637B6A022283F8A5201D
:10067000002303937B6A029307F1140301933B6BFE
:1006800000933B687A68B968F86800F051F8786AB6
:1006900000F0F6F801E000237B617B6918462837FB
:1006A000BD4680BD80B58CB004AFF860B9603B60DA
:1006B0001346FB80FB889B00184601F077FC7861AD
:1006C0007B69002B0ED0A82001F070FCF861FB695B
:1006D000002B03D0FB697A691A6305E0786901F0A1
:1006E00033FD01E00023FB61FB69002B17D0FB69A0
:1006F000002283F8A520FA8800230393FB69029364
:10070000FB6A0193BB6A00933B68B968F86800F024
:100710000FF8F86900F0B4F80123BB6102E04FF074
:10072000FF33BB61BB6918462037BD4680BD000062
:1007300080B588B000AFF860B9607A603B603B6B11
:10074000186B7B689B001A46A52103F0DDFC3B6B10
:100750001A6B7B6803F18043013B9B001344BB6130
:10076000BB6923F00703BB61BB6903F00703002BE0
:100770000BD04FF0500383F31188BFF36F8FBFF39B
:100780004F8F7B6100BF00BFFDE7BB68002B1FD010
:100790000023FB6112E0BA68FB69134419783A6BD5
:1007A000FB69134434330A461A70BA68FB69134470
:1007B0001B78002B06D0FB690133FB61FB690F2B13
:1007C000E9D900E000BF3B6B002283F8432003E03F
:1007D0003B6B002283F83420BB6A372B01D93723C7
:1007E000BB623B6BBA6ADA623B6BBA6ADA643B6B38
:1007F00000221A653B6B04331846FFF765F93B6B23
:1008000018331846FFF760F93B6B3A6B1A61BB6A05
:10081000C3F138023B6B9A613B6B3A6B5A623B6B9C
:100820000022C3F8A0203B6B002283F8A4203B6B7E
:1008300054334C220021184603F066FC3B6B0D4AF2
:100840009A653B6B0C4ADA653B6B0C4A1A663A6850
:10085000F968B86901F05AF902463B6B1A60FB6A05
:10086000002B02D0FB6A3A6B1A6000BF2037BD46EE
:1008700080BD00BFF42F01205C300120C430012076
:1008800080B582B000AF786001F06EFA2D4B1B6826
:1008900001332C4A13602C4B1B68002B09D12A4AC8
:1008A0007B681360274B1B68012B10D100F02EFCD6
:1008B0000DE0264B1B68002B09D1234B1B68DA6A1D
:1008C0007B68DB6A9A4202D81F4A7B681360204B20
:1008D0001B6801331E4A13601D4B1A687B685A64FB
:1008E0007B68DA6A1B4B1B689A4203D97B68DB6A18
:1008F000184A13607B68DA6A13469B0013449B0016
:10090000154A1A447B68043319461046FFF7E9F884
:1009100001F05CFA0D4B1B68002B0ED00A4B1B68D4
:10092000DA6A7B68DB6A9A4207D20C4B4FF080523E
:100930001A60BFF34F8FBFF36F8F00BF0837BD46FC
:1009400080BD00BF8C130020B80E0020981300203B
:10095000A813002094130020BC0E002004ED00E03A
:1009600080B584B000AF78600023FB607B68002B0B
:1009700018D0144B1B68002B0BD04FF0500383F39F
:100980001188BFF36F8FBFF34F8FBB6000BF00BFF5
:10099000FDE700F08BF80021786800F009FD00F019
:1009A00093F8F860FB68002B07D1074B4FF080529B
:1009B0001A60BFF34F8FBFF36F8F00BF1037BD4674
:1009C00080BD00BFB413002004ED00E080B58AB004
:1009D00004AF0023BB6000237B603A46391D07F15A
:1009E00008031846FFF71CF839687B68BA6802925A
:1009F00001930023009300230A4624492448FFF76B
:100A0000F1FD0346234A1360224B1B68002B02D0E2
:100A100001237B6101E000237B617B69012B02D113
:100A200000F01AFD78617B69012B1BD14FF0500358
:100A300083F31188BFF36F8FBFF34F8F3B6100BF0C
:100A4000154B1B685433154A1360154B4FF0FF329A
:100A50001A60144B01221A60134B00221A6001F035
:100A6000DFF80FE07B69B3F1FF3F0BD14FF050038C
:100A700083F31188BFF36F8FBFF34F8FFB6000BF0D
:100A800000BFFDE700BF1837BD4680BD9C7101085F
:100A9000DD100108B0130020B80E0020FC02002079
:100AA000AC130020981300209013002080B400AFF6
:100AB000044B1B680133034A136000BFBD465DF859
:100AC000047B7047B413002080B584B000AF0023CE
:100AD000FB600023BB60424B1B68002B0BD14FF027
:100AE000500383F31188BFF36F8FBFF34F8F3B60C9
:100AF00000BF00BFFDE701F037F9394B1B68013B30
:100B0000374A1360364B1B68002B62D1354B1B688C
:100B1000002B5ED02FE0344BDB68DB68FB60FB68AA
:100B200018331846FFF73AF8FB6804331846FFF706
:100B300035F8FB68DA6A2D4B1B689A4203D9FB68CB
:100B4000DB6A2A4A1360FB68DA6A13469B00134487
:100B50009B00274A1A44FB68043319461046FEF7E7
:100B6000C0FFFB68DA6A234B1B68DB6A9A4202D338
:100B7000214B01221A601C4B1B68002BCBD1FB6858
:100B8000002B01D000F066FB1C4B1B687B607B6870
:100B9000002B10D000F046F80346002B02D0164B75
:100BA00001221A607B68013B7B607B68002BF1D1DE
:100BB000124B00221A60104B1B68002B09D0012336
:100BC000BB600F4B4FF080521A60BFF34F8FBFF3E3
:100BD0006F8F01F0FBF8BB6818461037BD4680BD2B
:100BE000B41300208C1300204C1300209413002019
:100BF000BC0E0020B80E0020A01300209C13002083
:100C000004ED00E080B483B000AF054B1B687B604F
:100C10007B6818460C37BD465DF8047B704700BF03
:100C20009013002080B586B000AF00237B614F4B4E
:100C30001B68002B40F090804D4B1B6801333B61DB
:100C40004B4A3B6913603B69002B21D1494B1B6820
:100C50001B68002B0BD04FF0500383F31188BFF3B8
:100C60006F8FBFF34F8F3B6000BF00BFFDE7414B6D
:100C70001B68FB60404B1B683E4A13603E4AFB68A2
:100C800013603E4B1B6801333C4A136000F0E2FAEC
:100C90003B4B1B683A699A4249D3364B1B681B6829
:100CA000002B04D1364B4FF0FF321A603FE0314B3E
:100CB0001B68DB68DB68BB60BB685B687B603A69AC
:100CC0007B689A4203D22E4A7B6813602FE0BB6890
:100CD00004331846FEF762FFBB689B6A002B04D002
:100CE000BB6818331846FEF759FFBB68DA6A254B14
:100CF0001B689A4203D9BB68DB6A224A1360BB684F
:100D0000DA6A13469B0013449B001F4A1A44BB68CF
:100D1000043319461046FEF7E4FEBB68DA6A1B4B43
:100D20001B68DB6A9A42B8D301237B61B5E7174B96
:100D30001B68DA6A144913469B0013449B000B445A
:100D40001B68012B01D901237B61114B1B68002B10
:100D500007D001237B6104E00E4B1B6801330D4A71
:100D600013607B6918461837BD4680BDB413002058
:100D7000901300204413002048130020A4130020E7
:100D8000AC13002094130020BC0E0020B80E0020ED
:100D9000A01300209C13002080B485B000AF2B4B23
:100DA0001B68002B03D02A4B01221A6047E0284B16
:100DB00000221A60274B1B68FB6011E0FB68002BC8
:100DC0000BD14FF0500383F31188BFF36F8FBFF344
:100DD0004F8F7B6000BF00BFFDE7FB68013BFB60FE
:100DE0001D49FA6813469B0013449B000B441B6883
:100DF000002BE3D0FA6813469B0013449B00164A6D
:100E00001344BB60BB685B685A68BB685A60BB68C8
:100E10005A68BB6808339A4204D1BB685B685A6859
:100E2000BB685A60BB685B68DB680C4A1360094AA0
:100E3000FB681360094B1B685433094A136000BFF9
:100E40001437BD465DF8047B704700BFB413002023
:100E5000A013002094130020BC0E0020B80E002028
:100E6000FC02002080B584B000AF786039607B68F8
:100E7000002B0BD14FF0500383F31188BFF36F8F1A
:100E8000BFF34F8FFB6000BF00BFFDE7074B1B6840
:100E9000183319467868FEF748FE0121386800F0DB
:100EA00087FA00BF1037BD4680BD00BFB80E0020D6
:100EB00080B586B000AFF860B9607A60FB68002B3F
:100EC0000BD14FF0500383F31188BFF36F8FBFF343
:100ED0004F8F7B6100BF00BFFDE70A4B1B681833D3
:100EE0001946F868FEF7FDFD7B68002B02D04FF035
:100EF000FF33BB607968B86800F05AFA00BF183752
:100F0000BD4680BDB80E002080B586B000AF7860C9
:100F10007B68DB68DB683B613B69002B0BD14FF0E2
:100F2000500383F31188BFF36F8FBFF34F8FFB60C4
:100F300000BF00BFFDE73B6918331846FEF72EFEE1
:100F40001D4B1B68002B1DD13B6904331846FEF76F
:100F500025FE3B69DA6A194B1B689A4203D93B6943
:100F6000DB6A164A13603B69DA6A13469B00134436
:100F70009B00134A1A443B69043319461046FEF796
:100F8000B0FD05E03B69183319460E48FEF7A9FD90
:100F90003B69DA6A0C4B1B68DB6A9A4205D901236C
:100FA0007B610A4B01221A6001E000237B617B69AF
:100FB00018461837BD4680BDB41300209413002096
:100FC000BC0E00204C130020B80E0020A0130020FF
:100FD00080B483B000AF7860064B1A687B681A60F3
:100FE000054B1A687B685A6000BF0C37BD465DF838
:100FF000047B7047A41300209013002080B588B0B4
:1010000000AF786039607B68002B0BD14FF0500344
:1010100083F31188BFF36F8FBFF34F8F3B6100BF26
:1010200000BFFDE73B68002B0BD14FF0500383F36B
:101030001188BFF36F8FBFF34F8FFB6000BF00BFFE
:10104000FDE700F091FE1D4B1B68BB617B685B6890
:10105000BA69D31A7B613B681B68B3F1FF3F02D1C9
:101060000023FB6123E07B681A68154B1B689A42DA
:1010700007D07B685B68BA699A4202D30123FB619F
:1010800015E03B681B687A699A420BD23B681A6884
:101090007B69D21A3B681A607868FFF799FF0023D2
:1010A000FB6104E03B6800221A600123FB6100F051
:1010B0008DFEFB6918462037BD4680BD9013002089
:1010C000A413002080B400AF034B01221A6000BFBC
:1010D000BD465DF8047B7047A013002080B582B048
:1010E00000AF786000F052F8064B1B68012BF9D96D
:1010F000054B4FF080521A60BFF34F8FBFF36F8FD5
:10110000F0E700BFBC0E002004ED00E080B582B027
:1011100000AF00237B600CE07A6813469B00134409
:101120009B00124A13441846FEF7AEFC7B6801335D
:101130007B607B68372BEFD90D48FEF7A5FC0D4887
:10114000FEF7A2FC0C48FEF79FFC0C48FEF79CFC47
:101150000B48FEF799FC0B4B054A1A600A4B054AEF
:101160001A6000BF0837BD4680BD00BFBC0E00201E
:101170001C130020301300204C13002060130020AB
:1011800078130020441300204813002080B582B05B
:1011900000AF19E000F0E8FD104BDB68DB687B6016
:1011A0007B6804331846FEF7F9FC0D4B1B68013BC6
:1011B0000B4A13600B4B1B68013B0A4A136000F09B
:1011C00005FE786800F010F8064B1B68002BE1D193
:1011D00000BF00BF0837BD4680BD00BF60130020C0
:1011E0008C1300207413002080B584B000AF7860A9
:1011F0007B685433184602F0E3FF7B6893F8A53010
:10120000002B08D17B681B6B184600F09DFF7868A7
:1012100000F09AFF19E07B6893F8A530012B03D109
:10122000786800F091FF10E07B6893F8A530022BFE
:101230000BD04FF0500383F31188BFF36F8FBFF3D0
:101240004F8FFB6000BF00BFFDE700BF1037BD46FA
:1012500080BD000080B483B000AF0C4B1B681B68DE
:10126000002B04D10A4B4FF0FF321A6008E0074B05
:101270001B68DB68DB687B607B685B68044A136023
:1012800000BF0C37BD465DF8047B70474413002057
:10129000AC13002080B483B000AF0B4B1B68002B55
:1012A00002D101237B6008E0084B1B68002B02D1B0
:1012B00002237B6001E000237B607B6818460C37CB
:1012C000BD465DF8047B704798130020B4130020DE
:1012D00080B586B000AF78607B683B6100237B619E
:1012E0007B68002B58D02F4B1B683A699A420BD071
:1012F0004FF0500383F31188BFF36F8FBFF34F8F0D
:10130000FB6000BF00BFFDE73B691B6D002B0BD1ED
:101310004FF0500383F31188BFF36F8FBFF34F8FEC
:10132000BB6000BF00BFFDE73B691B6D5A1E3B69F8
:101330001A653B69DA6A3B69DB6C9A422CD03B69DF
:101340001B6D002B28D13B6904331846FEF726FCA1
:101350003B69DA6C3B69DA623B69DB6AC3F13802EC
:101360003B699A613B69DA6A0F4B1B689A4203D961
:101370003B69DB6A0C4A13603B69DA6A13469B00DF
:1013800013449B00094A1A443B690433194610462A
:10139000FEF7A7FB01237B617B6918461837BD4622
:1013A00080BD00BFB80E002094130020BC0E0020AA
:1013B00080B584B000AF78603960214B1B68FB605A
:1013C000204B1B6804331846FEF7E8FB7B68B3F13B
:1013D000FF3F0AD13B68002B07D01A4B1B68043330
:1013E00019461948FEF77DFB26E0FA687B6813442E
:1013F000BB60144B1B68BA685A60BA68FB689A42B3
:1014000009D2124B1A680F4B1B6804331946104659
:10141000FEF78BFB10E00E4B1A680A4B1B68043377
:1014200019461046FEF781FB0A4B1B68BA689A42C0
:1014300002D2084ABB68136000BF1037BD4680BDAA
:1014400090130020B80E00207813002048130020CD
:1014500044130020AC13002080B58AB004AF0023F1
:101460007B6100F013FB1D4B1B68002B21D0002378
:10147000FB600023BB603A1D07F1080107F10C0374
:101480001846FEF7E7FA7968BB68FA68029201939A
:101490000223009300230A4611491248FFF7A2F8DD
:1014A0000346114A1360104B1B68002B01D0012327
:1014B0007B617B69002B0BD14FF0500383F31188C4
:1014C000BFF36F8FBFF34F8F3B6100BF00BFFDE7DE
:1014D0007B6918461837BD4680BD00BFE813002061
:1014E000A471010825160108EC13002080B58AB00C
:1014F00000AFF860B9607A603B6000237B62FB68F4
:10150000002B0BD14FF0500383F31188BFF36F8F83
:10151000BFF34F8F3B6200BF00BFFDE7194B1B6855
:10152000002B2AD0BB683B617B687B61FB68BB6199
:10153000BB68052B18DCFFF7ADFE0346022B09D173
:10154000104B186807F1100100233A6BFEF75AFCA4
:10155000786212E00B4B186807F11001002300229B
:10156000FEF750FC786208E0064B186807F110019E
:1015700000233A68FEF748FD78627B6A18462837F0
:10158000BD4680BDE813002080B588B002AF78600A
:101590003960234B1B68DB68DB687B617B69043344
:1015A0001846FEF7FBFA7B6993F8283003F0040332
:1015B000002B23D07B699A697B68D1187B683A68D5
:1015C000786900F0D5F80346002B20D00023009363
:1015D00000237A6800217869FFF788FF38613B694A
:1015E000002B14D14FF0500383F31188BFF36F8F9A
:1015F000BFF34F8FFB6000BF00BFFDE77B6993F82F
:10160000283023F00103DAB27B6983F828207B6954
:101610001B6A7869984700BF1837BD4680BD00BF78
:10162000E013002080B584B000AF786007F10803B4
:10163000184600F059F8F860BB681946F86800F0E1
:1016400005F800F0D7F800BFF0E7000080B584B0DF
:1016500000AF78603960FFF729FA07F108031846F0
:1016600000F066F8F860BB68002B30D13B68002BB7
:101670000AD17A68FB689A4206D8FFF725FAF9681A
:101680007868FFF781FF24E03B68002B08D0134BFC
:101690001B681B68002B01D1012300E000233B6085
:1016A0000F4B18687A68FB68D31A3A681946FEF738
:1016B00065FFFFF709FA0346002B0AD1094B4FF0EB
:1016C00080521A60BFF34F8FBFF36F8F01E0FFF7B7
:1016D000FBF900BF1037BD4680BD00BFE4130020FA
:1016E000E813002004ED00E080B485B000AF78601E
:1016F0000E4B1B681B68002B01D1012200E0002269
:101700007B681A607B681B68002B05D1074B1B6840
:10171000DB681B68FB6001E00023FB60FB68184688
:101720001437BD465DF8047B704700BFE01300200E
:1017300080B584B000AF7860FFF764FAF8600B4BB7
:101740001B68FA689A4205D200F03AF97B680122D8
:101750001A6002E07B6800221A60044AFB6813608A
:10176000FB6818461037BD4680BD00BFF01300204F
:1017700080B586B000AFF860B9607A603B60002346
:101780007B61FB68BA685A60FB68FA681A61BA68DC
:101790007B689A4212D87A683B68D21AFB689B69C8
:1017A0009A4202D301237B611BE0104B1A68FB684D
:1017B000043319461046FEF7B8F912E07A683B6820
:1017C0009A4206D2BA683B689A4202D301237B61EF
:1017D00007E0074B1A68FB68043319461046FEF70A
:1017E000A4F97B6918461837BD4680BDE413002074
:1017F000E013002080B58EB002AFCEE07B68002BF6
:1018000019DA3B1D0433FB62FB6A002B0BD14FF04E
:10181000500383F31188BFF36F8FBFF34F8FFB61CA
:1018200000BF00BFFDE7FB6A1B68FA6A5068FA6AEE
:101830009268114698477B68002BC0F2AE80FB6827
:10184000BB62BB6A5B69002B04D0BB6A04331846D9
:10185000FEF7A4F93B461846FFF76AFF78627B68FB
:10186000092B00F2978001A252F823F09518010885
:1018700095180108951801080B1901081F1901088E
:101880006B19010895180108951801080B19010832
:101890001F190108BB6A93F8283043F00103DAB23C
:1018A000BB6A83F82820BA68BB6A9B69D118BB68F9
:1018B0007A6AB86AFFF75CFF0346002B6CD0BB6AFC
:1018C0001B6AB86A9847BB6A93F8283003F0040390
:1018D000002B61D0BA68BB6A9B691A44002300934D
:1018E00000230021B86AFFF701FE38623B6A002B33
:1018F00052D14FF0500383F31188BFF36F8FBFF3C2
:101900004F8FBB6100BF00BFFDE7BB6A93F8283073
:1019100023F00103DAB2BB6A83F828203DE0BB6AFA
:1019200093F8283043F00103DAB2BB6A83F8282029
:10193000BA68BB6A9A61BB6A9B69002B0BD14FF0F6
:10194000500383F31188BFF36F8FBFF34F8F7B6119
:1019500000BF00BFFDE7BB6A9A697B6AD1187B6A4A
:101960007A6AB86AFFF704FF17E0BB6A93F8283079
:1019700003F00203002B03D1B86A00F0E5FB0CE092
:10198000BB6A93F8283023F00103DAB2BB6A83F80C
:10199000282002E000BF00E000BF084B1B68391D93
:1019A00000221846FEF7CEFB0346002B7FF426AF3D
:1019B00000BF00BF3037BD4680BD00BFE813002028
:1019C00080B588B002AF49E02E4B1B68DB681B680E
:1019D0003B612C4B1B68DB68DB68FB60FB680433F6
:1019E0001846FEF7DBF8FB681B6AF8689847FB6847
:1019F00093F8283003F00403002B2FD0FB689B6979
:101A00003A691344BB60BA683B699A420ED9FB68D5
:101A1000BA685A60FB68FA681A611A4B1A68FB6860
:101A2000043319461046FEF780F817E000230093B0
:101A300000233A690021F868FFF758FD78607B6859
:101A4000002B0BD14FF0500383F31188BFF36F8F3E
:101A5000BFF34F8F3B6000BF00BFFDE7094B1B6822
:101A60001B68002BB0D1074B1B687B61064B1B68C2
:101A7000044A1360044A7B69136000BF1837BD46EF
:101A800080BD00BFE0130020E413002080B582B0C9
:101A900002AF00F069F9154B1B68002B20D11448E8
:101AA000FDF7F2FF1348FDF7EFFF134B104A1A60E2
:101AB000124B104A1A6000230093114B114A102157
:101AC0000A20FEF7FFF80346084A1360074B1B681D
:101AD000002B05D0054B1B680B491846FEF724FD6B
:101AE00000F074F900BFBD4680BD00BFE8130020C0
:101AF000B8130020CC130020E0130020E4130020D2
:101B000094140020F4130020AC71010880B485B057
:101B100000AFF860B9607A60FB68043BFB60FB686B
:101B20004FF080721A60FB68043BFB60BB6823F0D7
:101B30000102FB681A60FB68043BFB600C4AFB680F
:101B40001A60FB68143BFB607A68FB681A60FB68EC
:101B5000043BFB60FB686FF002021A60FB68203BED
:101B6000FB60FB6818461437BD465DF8047B704780
:101B7000751B010880B485B000AF00237B60134B58
:101B80001B68B3F1FF3F0BD04FF0500383F3118874
:101B9000BFF36F8FBFF34F8FFB6000BF00BFFDE748
:101BA0004FF0500383F31188BFF36F8FBFF34F8F54
:101BB000BB6000BF00BF7B68002BFCD000BF00BF34
:101BC0001437BD465DF8047B704700BF0C01002050
:101BD000074B19680868B0E8F04F80F30988BFF335
:101BE0006F8F4FF0000080F311887047AFF30080D3
:101BF000B80E002000BF00BF08480068006880F3EE
:101C000008884FF0000080F3148862B661B6BFF315
